:020000040000FA
:200000000207B60200800402003F000200081B22FFFFFF02008014FFFFFFFF0200801CFFE7
:20002000FFFFFF020080244753373136542020202020202020204C56312E30EB7002E722DA
:2000400089828A831410E704F593E022F593E49322BB0002F722BB8000500989828A838BC1
:20006000931593F022BC000BBE0029EF8DF084FFADF022E4CCF875F008EF2FFFEE33FEEC9A
:2000800033FCEE9DEC984005FCEE9DFE0FD5F0E9E4CEFD22EDF8F5F0EE008420D21CFEADD5
:2000A000F075F008EF2FFFED33FD4007985006D5F0F222C398FD0FD5F0EA22A3F8E0C5F033
:2000C00025F0F0E582158270021583E0C838F0E822BB0006F709A7F01922BB8000500D8985
:2000E000828A838B931593F0E5F0A3F022E88FF0A4CC8BF0A42CFCE98EF0A42CFC8AF0ED79
:20010000A42CFCEA8EF0A4CDA8F08BF0A42DCC3825F0FDE98FF0A42CCD35F0FCEB8EF0A40D
:20012000FEA9F0EB8FF0A4CFC5F02ECD39FEE43CFCEAA42DCE35F0FDE43CFC22EB9FF5F0F0
:20014000EA9E42F0E99D42F0E89C45F022E8600FEFC333FFEE33FEED33FDEC33FCD8F122D5
:20016000BB0006E9F802000332BB8000500C89828A838B9315930200017B22ECF0A3EDF035
:20018000A3EEF0A3EFF022EB700C87F009E608B5F019DFF6801589828A831410E70FF59383
:2001A000E0F5F0A3E608B5F002DFF5806AF593E493F5F0A3E608B5F05EDFF4805ACB701311
:2001C00088828C838B9387F009E493A3B5F048DFF580441410E71F88848C858B9589828ACD
:2001E00083F593758620E0F5F0E493A3A3B5F024DFF4DEF2801E88848C858B9589828A83F8
:20020000F593758620E493F5F0E493A3A3B5F004DFF3DEF17586007FFFB5F0020F22400245
:200220007F012202000187809488F0EF60010E4E60F0ED60EE1410E7EECB701288828C8370
:20024000F59387F009E0A3B5F0CDDFF680C91410E71E88848C858B9589828A83F593758682
:2002600020E0F5F0E0A3A3B5F0AADFF5DEF380A488848C858B9589828A83F593758620E47F
:2002800093F5F0E0A3A3B5F08BDFF4DEF28085EB7008E709F608DFFA801B89828A831410E7
:2002A000E70AF593E0A3F608DFFA8009F593E493A3F608DFF9ECFAA9F0EDFB2288F0EF601A
:2002C000010E4E60F088F0ED60C51410E7E7CB700E88828C838B93E709F0A3DFFA80D614AF
:2002E00010E71C88848C858B9589828A83F593758620E0F0A3A3DFFADEF875860080B68875
:20030000848C858B9589828A83F593758620E493F0A3A3DFF9DEF77586008099C5F0F8A3AF
:20032000E028F0C5F0F8E582158270021583E038F022ECF608EDF608EEF608EFF62290008E
:200340007004E0F54090007005E0F541854082854183E020E7077E007F00C2D72289428A6E
:20036000435407F54512000539E02402F54450020545120003E0053AE53A7002053BE54050
:200380002544F540E541354530E604C2E6242DF5411200040090007004E540F090007005A2
:2003A000E541F0AE45AF44D2D72290007010E020E61EA3EDF0A3E9F0A3EAF0EC5407D2E6EA
:2003C00090007010F00538E53870020539D2D7227C007D00C2D72290007010E0A2E6B32247
:2003E00075F001800375F0041200040078407F06900070921200052190007090E5F0F02217
:2004000090007090E0540770F7221200046D90007008742DF0900070107508101200045861
:20042000E490007004F090007006F0742D90007005F090007007F0751D10751C10751E008B
:20044000751F2D75832D758200E4F0753800753900753A00753B0022E4A808F0A3D8FC22F2
:20046000120005171200040A120004AB22900004A175080A79707860120005287518C075CD
:2004800019A8751A00751B647510C07511A87512007513017514FF7515FF7516FF7517006E
:2004A00022000B78667788C0A800649000706AE0440CF0229000706AE054F3F02290007017
:2004C0006AE04401F0229000706AE054FEF0229000706AE04402F0229000706AE054FDF0A0
:2004E000229000706AE04440F0229000706AE054BFF02290007000E04410F0229000700045
:20050000E054EFF02290007000E04420F02290007000E05420F0229000700AF000000000F0
:2005200022E6F008A3DFFA2289A0E493A3F208B800030989A0D508F222A3E58330E6037569
:20054000832D22754300754200754100754000754508754400120003E5754308754200758E
:200560004108754000754508754400120003E51200040090000000750910750800750B00D7
:20058000750A0012000638400B9000706CE04408F0D2D722C2D7227543007542007541000E
:2005A000754000754508754400120003E5754308754200754108754000754508754400129A
:2005C0000003E51200040090000000750910750800750B00750A00120006384051754310DA
:2005E000754200754110754000754508754400120003E575431875420075411875400075D5
:200600004508754400120003E51200040090001000750910750800750B10750A00120006F2
:2006200038400B9000706CE04418F0D2D722C2D722E6F008A3DFFA22A90B89A0A80AE49397
:20064000F5F0A3E265F0701008B800030989A01200067D50E9C2D722D2D722A90B89A0A88D
:200660000AE0F5F0A3E265F0701008B800030989A01200067D50EAC2D722D2D722E50860BA
:200680000A14F50845097007D2D72215091508C2D7229000700B7418F09000700C7420F0A2
:2006A00075A06022120006927824E2E2B408157400F21200072912000721120007071200B4
:2006C000070E802E22120006927816E2E2703708E2E2B4013178281200079C5029120007F9
:2006E0003912000779120007411200078178177402F27800E2E2FC4480F208E2E2FD7918FC
:200700007A20120003AA22781AE4F208F222782680F7E2E2F5F0E3E3F2E5F0F30809DAF2BF
:20072000227A04781C792080E9790878027A0680E1E2E2F30809DAF922780879027A0680EF
:20074000F0780879227A0680E8E4F309F3227A08E480037A04E4F309DAFC22E0F3A309E013
:20076000F3227A04E0F3A309DAFA227A0280027A04E2E2F0A308DAF922900070607A068041
:20078000E3781879227A0A8089E0F5F0E2E265F0700708A3DAF3D2D722C2D7229000706605
:2007A0007A0480E59000200AE0FEA3E08E8375820075814F732275C7AA75C755759D027856
:2007C0007FE4F6D8FD900000007F007E607D01E4F0A3DFFCDEFADDF875815012000517D23B
:2007E0000D120004B41200040A12001D6F12001D8B12000F7BEF700402000807020008157B
:200800001200000FEF700EC20D120004AB1200000702000C17D20D02008000300D040200D8
:20082000800CC0E0C0D075D00012001D24D0D0D0E0320D0A20426C616E6B20436865636BC5
:20084000696E67002E2E2E5B6661696C5D0A002E2E2E5B6F6B5D0A000D0A205446333331E4
:2008600046553A536563746F722D62617365642832353620736563746F72732920466C61C3
:2008800073682045726173652028314D29002E2E2E5B6F6B5D2E004387049000555574AA0E
:2008A000F090002AAA7455F09000555574A0F08F828E838D93E52EF05387FB224387049053
:2008C000200AAA74AAF0902005557455F090200AAA74A0F08F828E838D93E52EF05387FBF1
:2008E000220D0A2849503D200025752E00257529000D0A284D41433D200025782E00257841
:2009000029000D0A54463333313A205446545020646F6E652E204A756D7020746F20307853
:2009200025782E0A00496C6C6567616C206669726D77617265002E000D0A20496E76616C4C
:200940006964206669726D776172652021000D0A20466C617368206572726F722021001B41
:200960005B324A000D0A436865636B204D6167696320436F64652E2E2E004F4B2121004663
:2009800061696C2121009000262FEEF0A3EFF0E4784FF608F6D390002630E0940090002618
:2009A0002FE094005003010C1690002620E0FF94094003010AD2EF705E9000262FE0FEA389
:2009C000E0FFD39400EE94004031784FE6FC08E67B012448F974203CFA1200003B643A6051
:2009E0001A90002630E024FFF09000262FE034FFF0785006E61870C10680BEEF4E7003012A
:200A00000C16784C7601900026207401F0785006E618704F06804C90002620E0784CF678F9
:200A20004CE6C39409504E90002630E094009000262FE09400403E784F0806E61886067086
:200A40000106147B012448F974203EFA1200003BFF784CE6062423F582E43426F583759356
:200A600000EFF090002630E024FFF09000262FE034FFF080AA784CE690002620F0C39409DC
:200A80005003010C169000261A7426F0A37423F012001885EF64014E700690002620F022AD
:200AA00012001885EF64044E7003010BC77D027F01120018899000261CEFF07D067C007FBB
:200AC000037E001200188D90002614EEF0A3EFF0807E9000261DE0FFA3E090002614CFF0F8
:200AE000A3EFF090002621E06066D390002630E094009000262FE0940040559000261A7498
:200B000026F0A37421F0784F0806E6188606700106147B012448F974203EFA1200003B9023
:200B2000002622F090002630E024FFF09000262FE034FFF07D017C00E4FFFE1200188D1218
:200B40000014EFE490002621F09000261CE014F09000261A7420F0A37448F0A3E0FF784D47
:200B6000760008A607D3784EE6940018E694004049D390002630E094019000262FE0940095
:200B80004038784FE6FE08E6FF2401FDE43EFC1200188D120014EF7850740226F618E436AD
:200BA000F618E6161870011690002630E024FEF09000262FE034FFF080AB784EE69000263F
:200BC0001CF0E61846700890002620F00109959000262FE07004A3E064017026784F08065C
:200BE000E6188606700106147B012448F974203EFA1200003B90002621F0E49000262FF066
:200C0000A3F090002614E0FFA3E09000261DCFF0A3EFF00109952275B0FB7F0A7E00120007
:200C20001A31EF784BF612001D4C900070FFE0784BF6120012407E087FE1E4FDFC12000E67
:200C400013E4784BF6784BE6FDC39403501E7E087FE974042DF582E43420F583759300E0D4
:200C6000FD7C0012000E13784B0680D97E087FED90002007E0FD7C0012000E137E087FF17B
:200C8000E4FDFC12000E13E4784BF6784BE6FDC39405501E7E087FFA74122DF582E43420D6
:200CA000F583759300E0FD7C0012000E13784B0680D97E087FFE90002017E0FD7C001200D1
:200CC0000E137B017A2079181200033E90002608EEF0A3EFF0D39424EE940040E5900020F9
:200CE00026E0B4081FA3E0B4061A90002609E024F0F090002608E034FFF0120006C5784BB8
:200D0000A60780BE90002026E0B408B6A3E0B400B19000202AE0FFA3E090002608CFF0A37C
:200D2000EFF090002034E0FCA3E0FDA3E0FEA3E0FF900020001200017BE4784BF6784BE60D
:200D4000FF7C007B012420F9EC3420FA1200003BFE740C2FF582E43420F583759300EEF01E
:200D600006E6B406D890002028E064456003010CC29000202EE0543F6003010CC29000202F
:200D800031E0B4010E120006A4E490002608F0A3F0805190002031E0B411499000203EE030
:200DA0007004A3E06445701690002609E024E4F090002608E034FFF0120010DE802690007F
:200DC000203EE064FC7004A3E064036003010CC290002609E024E4F090002608E034FFF08D
:200DE000120015FB9000264DE07003010CC212001DB19000200A741FF0A374FCF07E097F86
:200E000002FD7C1F12000E13C2A9C2AF120007A4010CC290002638EEF0A3EFF0A3ECF0A32D
:200E2000EDF090002638E475F001120000BB85F082F583759300E4939000263DF07003018B
:200E40000F7AE064256003010F5B9000263C740AF090002638E475F001120000BB85F08276
:200E6000F583759300E49324DB7003010F5B800090002639E024FFF090002638E034FFF04B
:200E800090002638E475F001120000BB85F082F583759300E4939000263DF0E0249D601467
:200EA00024EE601924FD6003010F5B9000263C7410F080099000263BE0FF010F73900026C0
:200EC0003E740AF09000263AE07002A3E0605A9000263CE0FBFD7C009000263AE0FEA3E050
:200EE000FF12000065AA059000263AE0FEA3E0FFEBFD7C00120000659000263AEEF0A3EF42
:200F0000F0D3EA64809489EA40052457FF80032430FF9000263EE014F0244EF582E43426A5
:200F2000F583759300EFF0809B9000263EE0B40A047F30803E9000263EE0C3940A400301BB
:200F40000E22E0FF04F0744E2FF582E43426F583759300E0FF12001DBA80DA9000263DE073
:200F6000FF12001DBA9000263DE0640A6003010E227F0D12001DBA010E2222E4FFFEFDFC12
:200F80009000262F1200017BE490002633F07F0AFE12001A31EF12001D4C7E097F5FE4FD8D
:200FA000FC12000E137E097F64E4FDFC12000E137FFC7EFF7D0F7C00900026341200017B10
:200FC0009000262FE0F8A3E0F9A3E0FAA3E0FBC000C001C002C003A3E0FFE4FDFEA3A3E050
:200FE000F9A3E0FAA3E02FFFEE3AFEED39FDE42FFFE43EFEED3481FDA907AA06AB0512008E
:20100000003BFFD003D002D001D000EB4FFFEAFEE9FDE8FC9000262F1200017B9000262F0D
:20102000E0FCA3E0FDA3E0FEA3E0FF78081200014D9000262F1200017B90002633E004F041
:20104000E0C394035003010FC09000262FE0F8A3E0F9A3E0FAA3E0FBC000C001C002C003F9
:20106000A3E0FFE4FDFEA3A3E0F9A3E0FAA3E02FFFEE3AFEED39FDE42FFFE43EFEED3481A5
:20108000FDA907AA06AB051200003BFFD003D002D001D000EB4FFFEAFEE9FDE8FC90002610
:2010A0002F1200017B7F557EAA7D557CAA9000262FE0F8A3E0F9A3E0FAA3E0FBC312000175
:2010C0003C700D7E097F7AFDFC12000E137F01227E097F7FE4FDFC12000E137F0022900043
:2010E0002044E0FEA3E0FFEE600301123FEF24FD606404600301123F12001C049000203CDE
:20110000E0FFA3E090002643CFF0A3EFF09000203EE0FEA3E0FF90002641EEF0A3EFF090FE
:20112000002044E4F0A37404F0E4A3F0A3F09000203CEEF0A3EFF090002643E0FFA3E0902B
:2011400000203ECFF0A3EFF090002608E4F0A37404F0020013989000203EE0FEA3E0FF90C8
:20116000002641E06E7003A3E06F60030112379000263FE0FEA3E0FF90002046E0B50608BA
:20118000A3E0B5070301123390002640E02401FF9000263FE03400FE90002046E06E70030F
:2011A000A3E06F60030112379000203CE0FFA3E090002643CFF0A3EFF07E097F36E4FDFCEF
:2011C00012000E13C390002609E09404FF90002608E09400FE120009869000262EE0702BB3
:2011E00090002617E0C3941450067E097F3880047E097F4EE4FDFC12000E137F047E001248
:20120000001B989000264D7401F02290002640E004F070079000263FE004F0C39000260905
:20122000E0940490002608E0940250079000264D7401F002001CEAE490002608F0A3F022F4
:20124000D2A9D2AFE49000262FF0A3F09000262FE0FEA3E0FFC39402EE9400505BEF240464
:20126000FFE43EFE12001A3190002631EEF0A3EFF0E0FD90002630E025E0FB9000262FE043
:2012800033FA74042BF58274203AF583759300EDF090002631E0FF74052BF58274203AF538
:2012A00083759300EFF090002630E004F0709D9000262FE004F08094E49000262FF0A3F0E4
:2012C0009000262FE0FEA3E0FFC39403EE9400505412001A3190002631EEF0A3EFF0E0FDC8
:2012E00090002630E025E0FB9000262FE033FA74122BF58274203AF583759300EDF0900053
:201300002631E0FF74132BF58274203AF583759300EFF090002630E004F070A49000262F8E
:20132000E004F0809BE4784CF6784CE6FF2404F582E43420F583759300E0FEEF2466FDE4E8
:2013400034708D82F583759300EEF006E6B404D9E4784CF6784CE6FF2412F582E43420F5DE
:2013600083759300E0FEEF2460FDE434708D82F583759300EEF006E6B406D99000706CE0D4
:2013800054FDF090007001743FF0900070007410F0900070DAE4F02290002609E02408FE5B
:2013A00090002608E0340090002040F0A3CEF0E4A3F0A3F090002000E0FCA3E0FDA3E0FE83
:2013C000A3E0FF900020381200017B90002004E0FCA3E0FDA3E0FEA3E0FF9000203412000C
:2013E000017B90002609E0241CF090002608E03400F0900020287445F0E4A3F09000202E0A
:201400007440F0E4A3F0A37410F0A304F090002608E0FFA3E09000202ACFF0A3EFF0900038
:201420002009E004F0700790002008E004F090002008E09000202CF090002009E0900020FF
:201440002DF0E490002032F0A3F0900020187490F090002609E02412F090002608E03400D3
:20146000F0C3A3E0944090002608E094005006E4F0A37440F090002018E054F8FE90002617
:2014800008E04EFFA3E090002018CFF0A3EFF0E4FF740C2FF582E43420F583759300E0FEEC
:2014A000EF7C007B01241AF9EC3420FAEE120000510FEFB406DBE4FF74122FF582E43420A9
:2014C000F583759300E0FE74202FF582E43420F583759300EEF00FEFB406DD9000202674FF
:2014E00008F0A3E4F07B017A207918020003AA90002618EEF0A3EFF090002614E475F001E5
:20150000120000BBAFF090002631F0A3EFF090002619E0FF9000262CF090002046E070043C
:20152000A3E0640160030115AA90002631E0FCA3E0FDC39427EC9400403CD3ED943AEC94D5
:2015400000503390002617E004F08D828C83759300E4936F6006E49000262DF09000261771
:20156000E0B414129000262DE07004A3F080079000262E7401F090002616E0702DA3E064E7
:201580001470279000262EE06020E4F52F12000597120016E7120017C4EF70069000262E61
:2015A000F022900026167401F02290002631E0FEA3E04E7002052F9000262EE06401703AB7
:2015C00090002616E0640170319000262CE0FDF46028E52F7011C3EE9440401E90002631BF
:2015E000E0FEA3E0FF800F90002631E0FEA3E0FF9000262CE0FD12001B2A227FF27ED27D3F
:20160000077C0C90002054E0F8A3E0F9A3E0FAA3E0FBC31200013C60030116E69000204680
:20162000E0FEA3E0FF64014E6007EF4E60030116E6E490002052F0A3F090002050E0FEA3A9
:20164000E0FFEE60030116E6EF24FB600B24FB6009240960030116E6802D78127C207D017E
:201660007B017A2079487E007F0612000229EF707590002608E4F0A37428F090002050E4DA
:20168000F0A3740BF0800E12001C5790002050E4F0A3740CF078487C207D017B017A2079E5
:2016A000127E007F06120002BC90002044E4F0A37402F0A3E4F0A304F09000204EE4F0A3F1
:2016C00004F09000203EE0FEA3E0FF9000203CE0FDA3E0A3CDF0A3EDF09000203CEEF0A32F
:2016E000EFF012001398227E087F58E4FDFC12000E13E4F52FF523752408AE23AF24E4FC7A
:20170000FDFB7A10F9F8120000ED8F288E278D268C25A2AFE433F522C2AF4387047B217AB3
:201720000A79AA74AA120000517A0579557455120000517A0A79AA74801200005174AA1254
:201740000000517A057955745512000051E47FFF7EFFFDFCAB28AA27A926A825D3120001C1
:201760003C401BE42528FFE43527FEE5263401FDA907AA06AB05745012000051800C8528B7
:20178000828527837593007450F05387FBE52224FF92AFAE23AF24E4FCFDFB7A10F9F81293
:2017A0000000ED120019AF0524E52470020523C3E523940150030116FA7E087F8EE4FDFC62
:2017C00002000E137E087F32E4FDFC12000E13E4752502F524F523F522E47F3FFEFDFCAB93
:2017E00025AA24A923A822D31200013C4003011877E4F526F527E4FF7E40FDFCAB25AA2418
:20180000A923A822120000ED8F2B8E2A8D298C28E4FCFDE52B2527F52BE52A3526F52AED88
:201820003529F529EC3528F528E4252BFFE4352AFEE5293481FDA907AA06AB051200003B35
:20184000F4600D7E087F44E4FD12000E137F00220527E52770020526C3E52694404097E5F6
:20186000252401F525E43524F524E43523F523E43522F5220117D97E087F4FE4FDFC1200D4
:201880000E137F01227D087F077C007E0090002631ECF0A3EDF0E4A3F0A3F0AD07AC06C30A
:2018A00090002632E09D90002631E09C40629000261AE0FEA3E08E837593002DF582E58368
:2018C0003CF583759300E0F990002634E0C4F8540FC868F090002633E0C454F048F0E9D3A5
:2018E0009439500BE9C39430FFE49400FE8013C3E99441FFE49400CF240ACF3400FE9000C2
:201900002633E04EF0A3E04FF00DBD00010C808F90002633E0FEA3E0FF229000263AEEF06F
:20192000A3EFF09000265C7408F0F5C84402F0F5C87F327E0012001DB09000265CE04404AF
:20194000F0F5C87F647E0012001DB012001DA29000265A7408F0A3E4F09000265AE0FCA347
:20196000E0FD4C6043A3E054FAF09000263AE0FEA3E0FFEC5EFEED5F4E60089000265CE04E
:201980004404F09000265CE012001DAA12001DAC9000265CE04401F0F5C89000265AE0C3D2
:2019A00013F0A3E013F080B19000265CE0FF22900026361200017B752901E4F52CF52D908A
:2019C000002636A3E0FDA3E0FEA3E02400FFE43EFEED3481FDA907AA06AB051200003BF5F3
:2019E0002A532A40E529604090002636A3E0FDA3E0FEA3E02400FFE43EFEED3481FDA90750
:201A0000AA06AB051200003BF52B532B40E52AB52B03E4F529852B2A052DE52D7002052C86
:201A2000B4FFC1E52CB4FFBCE5297F0060027F0122C2AFEE4408FE1200191A9000265CEF32
:201A4000F0E490002638F0A3F09000265A7480F0A3E4F09000265AE07002A3E060379000CA
:201A6000265CE054FA12001DA912001DA2AFC8EF30E3149000265AE0FEA3E0FF9000263822
:201A8000E04EF0A3E04FF09000265AE0C313F0A3E013F080BE9000265CE054F8F0F5C87F82
:201AA000907E0112001DB0D2AF90002638E0FEA3E0FF229000262FEBF0A3EAF0A3E9F0E4AA
:201AC00090002637F0A3F09000263574FFF5F0120000BB45F0604690002632E0FBA3E0FA6B
:201AE000A3E0F91200003BFF9000262FE0FBA3E0FAA3E0F990002637E475F001120000BB61
:201B0000FCE925F0F9EA3CFAEF1200005160B890002633E475F0011200031C80AA90002604
:201B20002FE0FBA3E0FAA3E0F92290002633EEF0A3EFF0A3EDF0AF2FE4FCFDFEFBFA79018F
:201B4000F8120000ED8F268E258D248C2390002633E0FEA3E0FFE4FCFDE5262FF526E52541
:201B60003EF525ED3524F524EC3523F523A3E0F52EA2AFE433F522C2AFAF26AE25AD24AC97
:201B800023120008BCAF26AE25AD24AC23120019AFE52224FF92AF22900070007429F09080
:201BA000002044E4F0A37405F0A3EEF0A3EFF064044E7020900026327481F0A37409F0A318
:201BC0007425F0A3E4F0A37411F07B017A20794812001AB390002641E0FFA3E09000203CF2
:201BE000CFF0A3EFF090002643E0FFA3E09000203ECFF0A3EFF090002608E4F0A37415F06C
:201C000002001398E49000263FF0A3F090002000E0FCA3E0FDA3E0FEA3E0FF90002645129F
:201C200000017BE490002641F0A3F0A3F0A3F09000264DF09000262EF090002617F0900090
:201C40002616F09000262D04F0900070007421F0900070DAE4F0227B017A20796CE475F0E8
:201C600004120000D1740229F9E43AFAE475F008120000D1740229F9E43AFA90002004E055
:201C8000FCA3E0FDA3E0FEA3E0FF12000160740429F9E43AFEC3E99444FFEE9420900026C1
:201CA00008F0A3EFF0229000265EEEF0A3EFF0E4F54AD3ED9400EC9400402C9000265EE0BD
:201CC000FEA3E0AA06F97B811200003B254AF54AED1D70011C9000265FE004F070D490008F
:201CE000265EE004F080CBAF4A2290002044E4F0A37404F090002641E0FFA3E09000203C0E
:201D0000CFF0A3EFF090002643E0FFA3E09000203ECFF0A3EFF090002608E4F0A37404F05B
:201D200002001398C0D0C2A9C2AFE5492401F549E43548F548E43547F547E43546F54675B0
:201D40008C5D758A3DD2AFD2A9D0D0227598504387805389CF438920EFB40108758DF3754C
:201D60008CF38006758DE5758CE5D28ED29922E58954F04401F589758C5D758A3DE4F54973
:201D8000F548F547F546D2B9D28C227598504387805389CF438920758DE5758CE5D28ED247
:201DA00099229000265CE04401F0F5C87FF47E01229000706CE054E7F0223099FDC2998F27
:201DC0009922FFFFFFFFFFFFFFFFFFFFFFFFFFFFFFFFFFFFFFFFFFFFFFFFFFFFFFFFFFFF66
:201DE000FFFFFFFFFFFFFFFFFFFFFFFFFFFFFFFFFFFFFFFFFFFFFFFFFFFFFFFFFFFFFFFF03
:201E0000FFFFFFFFFFFFFFFFFFFFFFFFFFFFFFFFFFFFFFFFFFFFFFFFFFFFFFFFFFFFFFFFE2
:201E2000FFFFFFFFFFFFFFFFFFFFFFFFFFFFFFFFFFFFFFFFFFFFFFFFFFFFFFFFFFFFFFFFC2
:201E4000FFFFFFFFFFFFFFFFFFFFFFFFFFFFFFFFFFFFFFFFFFFFFFFFFFFFFFFFFFFFFFFFA2
:201E6000FFFFFFFFFFFFFFFFFFFFFFFFFFFFFFFFFFFFFFFFFFFFFFFFFFFFFFFFFFFFFFFF82
:201E8000FFFFFFFFFFFFFFFFFFFFFFFFFFFFFFFFFFFFFFFFFFFFFFFFFFFFFFFFFFFFFFFF62
:201EA000FFFFFFFFFFFFFFFFFFFFFFFFFFFFFFFFFFFFFFFFFFFFFFFFFFFFFFFFFFFFFFFF42
:201EC000FFFFFFFFFFFFFFFFFFFFFFFFFFFFFFFFFFFFFFFFFFFFFFFFFFFFFFFFFFFFFFFF22
:201EE000FFFFFFFFFFFFFFFFFFFFFFFFFFFFFFFFFFFFFFFFFFFFFFFFFFFFFFFFFFFFFFFF02
:201F0000FFFFFFFFFFFFFFFFFFFFFFFFFFFFFFFFFFFFFFFFFFFFFFFFFFFFFFFFFFFFFFFFE1
:201F2000FFFFFFFFFFFFFFFFFFFFFFFFFFFFFFFFFFFFFFFFFFFFFFFFFFFFFFFFFFFFFFFFC1
:201F4000FFFFFFFFFFFFFFFFFFFFFFFFFFFFFFFFFFFFFFFFFFFFFFFFFFFFFFFFFFFFFFFFA1
:201F6000FFFFFFFFFFFFFFFFFFFFFFFFFFFFFFFFFFFFFFFFFFFFFFFFFFFFFFFFFFFFFFFF81
:201F8000FFFFFFFFFFFFFFFFFFFFFFFFFFFFFFFFFFFFFFFFFFFFFFFFFFFFFFFFFFFFFFFF61
:201FA00075C7AA75C755759D02787FE4F6D8FD900000007F007E607D01E4F0A3DFFCDEFA5B
:201FC000DDF875815012000517C20D120004B41200040A12001D6F12001D8BC20D120004C2
:201FE000AB02000C17FFFFFFFFFFFFFFFFFFFFFFFFFFFFFFFFFFFFFFFFFFFFFF020007B669
:20200000020021EEEB7002E72289828A831410E704F593E022F593E49322BB0002F722BBE6
:202020008000500989828A838B931593F022BC000BBE0029EF8DF084FFADF022E4CCF8755E
:20204000F008EF2FFFEE33FEEC33FCEE9DEC984005FCEE9DFE0FD5F0E9E4CEFD22EDF8F5F0
:20206000F0EE008420D21CFEADF075F008EF2FFFED33FD4007985006D5F0F222C398FD0F39
:20208000D5F0EA22A3F8E0C5F025F0F0E582158270021583E0C838F0E822EB7007E7F5F02A
:2020A00009E7192289828A831410E708F593E0F5F0A3E022F593E493F5F074019322BB000F
:2020C00006F709A7F01922BB8000500D89828A838B931593F0E5F0A3F022EB9FF5F0EA9E41
:2020E00042F0E99D42F0E89C45F022E8600FECC313FCED13FDEE13FEEF13FFD8F122E860D6
:202100000FEFC333FFEE33FEED33FDEC33FCD8F122EB7006E9F80200217289828A83141077
:20212000E706F5930200217EF5930200218ABB0006E9F8020021C3BB8000500C89828A831D
:202140008B9315930200216622EB7006E9F80200219A89828A831410E706F593020021A794
:20216000F593020021B3ECF0A3EDF0A3EEF0A3EFF022E6FC08E6FD08E6FE08E6FF22E0FCDC
:20218000A3E0FDA3E0FEA3E0FF22E493FC740193FD740293FE740393FF22E6FB08E6F90820
:2021A000E6FA08E6CBF822E0F8A3E0F9A3E0FAA3E0FB22E493F8740193F9740293FA740311
:2021C00093FB22ECF608EDF608EEF608EFF6220D0A5B4D41435F49443D25785D000D0A5BAF
:2021E0005048595F49442578003D25785D0002002F2F9000200EEDF0A3EBF0A3EAF0A3E9AC
:20220000F0AE07EE7F0030E7027F01EF60037F0422EEC4135403FF90002013F0EE541FA34A
:20222000F012002EFEEF70037F042290002013E0FFA3E0FD7B017A20791512002DCCEF6049
:20224000037F0122E47F01FEFDFC900020161200216690002016E0FCA3E0FDA3E0FEA3E0F9
:20226000FF7805120020FE900020161200216690002016E0F8A3E0F9A3E0FAA3E0FB9000AE
:20228000200EE0FFEB4FFFEAFEE9FDE8FC900020161200216690002016E0FCA3E0FDA3E042
:2022A000FEA3E0FF7805120020FE900020161200216690002016E0F8A3E0F9A3E0FAA3E078
:2022C000FB90002015E0FFEB4FFFEAFEE9FDE8FCA31200216690002016E0FCA3E0FDA3E093
:2022E000FEA3E0FF7810120020FE900020161200216690002014E0FF12002ED19000201AC9
:20230000120021669000201AE0FCA3E0FDA3E0FEA3E0FF900020231200216690002016E0E9
:20232000FCA3E0FDA3E0FEA3E0FF900020271200216690002013E0FF12002C1190002012FB
:20234000EFF06003E0FF229000201AE0FCA3E0FDA3E0FEA3E0FF9000202312002166900015
:2023600020277401F0A37420F0A37416F090002013E0FF12002B5B90002012EFF06003E04F
:20238000FF22E4FFFEFD7C089000201E120021669000201EE0FCA3E0FDA3E0FEA3E0FF9096
:2023A000002016E0F8A3E0F9A3E0FAA3E05FFFEA5EFEE95DFDE85CFC781B120020EB90002C
:2023C000201E120021669000201EE0FCA3E0FDA3E0FEA3E0FFEC4D4E4F70030123479000B5
:2023E0002016A3A3E0FEA3E0FF9000200FE0FBA3E0FAA3E0F9EE8FF0120020BE900020124F
:20240000E0FF229000200EEEF0A3EFF0A3ECF0A3EDF09000200EE475F0011200208485F06B
:2024200082F583759300E49390002013F0700301256AE06425600301254B90002012740AF0
:20244000F09000200EE475F0011200208485F082F583759300E49324DB700301254B80007D
:202460009000200FE024FFF09000200EE034FFF09000200EE475F0011200208485F082F53F
:2024800083759300E49390002013F0E0249D601424EE601924FD600301254B9000201274BC
:2024A00010F0800990002011E0FF01256390002014740AF090002010E07002A3E0605A9059
:2024C000002012E0FBFD7C0090002010E0FEA3E0FF1200202EAA0590002010E0FEA3E0FF27
:2024E000EBFD7C001200202E90002010EEF0A3EFF0D3EA64809489EA40052457FF800324EA
:2025000030FF90002014E014F02450F582E43420F583759300EFF0809B90002014E0B40AE5
:20252000047F30803E90002014E0C3940A4003012412E0FF04F074502FF582E43420F583BE
:20254000759300E0FF12002F5780DA90002013E0FF12002F5790002013E0640A60030124CF
:20256000127F0D12002F570124122212002E8812002AA2E490002000F0A3F0A3F0A3F09059
:20258000002002E0FEA3E0FFC394C9EE940040030126C6EF7803C333CE33CED8F924BAF910
:2025A000742F3EFA7B81120021117B547A4079007804C3120020DA602D90002002E0FEA3F3
:2025C000E07803C333CE33CED8F924BAF9742F3EFA7B81120021117B547A4079007805C3D6
:2025E000120020DA706D90002001E0FFC007A3E0FEA3E07803C333CE33CED8F924BAF9743B
:202600002F3EFA7B8112002111900020061200216690002002E0FEA3E07803C333CE33CE71
:20262000D8F924BEF9742F3EFA7B81120021119000200A12002166D007120028F2900020CD
:2026400004EFF0E4FFFE0FBF00010EBE27F8BF10F5805D90002001E0FFC007A3E0FEA3E000
:202660007803C333CE33CED8F924BAF9742F3EFA7B8112002111900020231200216690005B
:202680002002E0FEA3E07803C333CE33CED8F924BEF9742F3EFA7B811200211190002027D9
:2026A00012002166D00712002C1190002004EFF090002003E004F0600301257F9000200287
:2026C000E004F001257F229000202DEFF0FBA3E0FCA3E0FDA3A3E4FFFEEC7810120020EBF1
:2026E00090002035EEF0A3EFF09000202EE0FCA3A3E0FEA3E0FF90002037EEF0A3EFF0AF3F
:202700000390002035E0FAA3E0FB7D0412002E2BEF6001229000202DE0FF90002037E0FA9E
:20272000A3E0FB7D0512002E2BEF6001229000203B7464F09000202DE0FF7B017A20793985
:202740007D1F120029D4EF6001229000203BE014F0C3940150037F01229000203AE030E066
:20276000D39000202DE0FF7B017A2079357D06120029D4EF6001229000202DE0FF7B017A50
:202780002079377D07120029D4EF60012290002035E0FEA3E0FFE4FCFD90002032E0FBA3E2
:2027A000E0FAA3E0F91200212E90002032E0FBA3E0FAA3E0F9120021117810120020FE129E
:2027C00000212E90002032E0FBA3E0FAA3E0F9C003C002C0011200214990002037E0FEA3CA
:2027E000E0FFEB4FFFEA4EFEE9FDE8FCD001D002D0031200212E7F00229000202EEFF0FB91
:20280000A3E0FCA3E0FDA3A3E4FFFEEC7810120020EB90002037EEF0A3EFF09000202FE0FB
:20282000FCA3A3E0FEA3E0FF90002039EEF0A3EFF0AF0390002037E0FAA3E0FBE4FD1200C9
:202840002E2BEF6001229000202EE0FF90002039E0FAA3E0FB7D0112002E2BEF60012290C4
:20286000002033E0FCA3E0FDA3A3E4FFFEEC7810120020EBA3EEF0FAA3EFF0FB9000203316
:20288000E0FCA3A3E0FEA3E0FF90002039EEF0A3EFF09000202EE0FF7D0212002E2BEF6077
:2028A00001229000202EE0FF90002039E0FAA3E0FB7D0312002E2BEF6001229000203D7439
:2028C00064F09000202EE0FF7B017A20793B7D1F120029D4EF6001229000203DE014F0C36C
:2028E000940150037F01229000203CE030E1D37F002290002005EFF0C007A3E0FCA3E0FDA3
:20290000A3E0FEA3E0FF90002023120021669000200AE0FCA3E0FDA3E0FEA3E0FF9000207F
:202920002712002166D00712002C119000200EEFF06003E0FF2290002006E0FCA3E0FDA3FB
:20294000E0FEA3E0FF9000202312002166900020277401F0A37420F0A3740AF09000200582
:20296000E0FF12002B5B9000200EEFF06003E0FF22E4FFFEFD7C109000200F12002166908D
:2029800000200FE0FCA3E0FDA3E0FEA3E0FF9000200AE0F8A3E0F9A3E0FAA3E05FFFEA5EF5
:2029A000FEE95DFDE85CFC781C120020EB9000200F120021669000200FE0FCA3E0FDA3E0EF
:2029C000FEA3E0FFEC4D4E4F60030129369000200EE0FF229000203EEFF0A3EDF0A3EBF054
:2029E000A3EAF0A3E9F0E4F5F0120020BE900020457405F090007080E054FEF09000203E37
:202A0000E090007082F09000203FE090007083F07DE87C0390007080E0FF20E709ED1D7055
:202A2000011C144C70EEED4C606990007085E090002043F090007084E090002044F0900099
:202A40002043E0FF90002040E0FBA3E0FAA3E0F9E48FF0120020BE90002040E0FBA3E0FAD5
:202A6000A3E0F91200209A75F000120020BE90002040E0FBA3E0FAA3E0F91200209AFF909A
:202A8000002044E0FDEF4DFFE5F08FF0120020BE7F002290002045E014F060030129F47FFC
:202AA0000122E490002009F0A3F090002005F0A3F090002005E0FEA3E0FFC39410EE64804D
:202AC00094805075E49000200CF0A3F09000200AE0C43354E0FDEF4DA3F0E490002007F0DE
:202AE000A3F09000200CE064017004A3E0644160359000200BE0FF7B017A20790C7D02124B
:202B00000021F290002008E004F0700790002007E004F0C390002008E0940A90002007E084
:202B20006480948040BC90002006E004F0708290002005E004F0012AB17E217FDD90002015
:202B400005E0FCA3E0FD120024037E217FE99000200CE0FCA3E0FD0200240390002032743D
:202B600001F0A37420F0A3742CF07B017A20792B12002CC7EF60037F01229000202BE0702C
:202B80003A90002023E0FCA3E0FDA3E0FEA3E0FF9000202E1200216690002027E0F9A3E01F
:202BA000FAA3E090002032C9F0A3EAF0A3E9F09000202CE0FF12002F1780409000202BE076
:202BC000B4014090002023E0FCA3E0FDA3E0FEA3E0FF9000202E1200216690002027E0F9A7
:202BE000A3E0FAA3E090002032C9F0A3EAF0A3E9F09000202CE0FF120026C79000202AEFBE
:202C0000F080079000202A7401F09000202AE0FF22900020327401F0A37420F0A3742DF081
:202C20007B017A20792C12002CC7EF60037F01229000202CE0703A90002023E0FCA3E0FD4B
:202C4000A3E0FEA3E0FF9000202F1200216690002027E0FCA3E0FDA3E0FEA3E0FF90002013
:202C600033120021669000202DE0FF12002F6780409000202CE0B4014090002023E0FCA361
:202C8000E0FDA3E0FEA3E0FF9000202F1200216690002027E0FCA3E0FDA3E0FEA3E0FF9016
:202CA000002033120021669000202DE0FF120027F99000202BEFF080079000202B7401F0B9
:202CC0009000202BE0FF229000202EEFF0A3EBF0A3EAF0A3E9F09000202EE075F072A42487
:202CE00008F9743635F0FA7B811200200470037F012290003674E493700F9000202FE0FBD9
:202D0000A3E0FAA3E0F9E4801790003674E493B4013D9000202FE0FBA3E0FAA3E0F9740174
:202D20001200201A9000202EE075F072A42407F9743635F0FA7B8112002004FF900020320E
:202D4000E0FBA3E0FAA3E0F9EF1200201A80037F01227F0022E490002004F090002003F073
:202D600090002000F090002000E0FFC394015041900020327401F0A37420F0A37402F07B49
:202D8000017A20790112002CC7EF60037F012290002001E0FF70069000200304F0EFB401D4
:202DA00007900020047401F090002000E004F080B490002004E0B4010412002F5F9000209E
:202DC00003E0B4010412002F647F002290002022EFF0A3EDF0A3EBF0A3EAF0A3E9F09000D9
:202DE0002022E075F072A4FDACF02408F974363CFA7B811200200470037F0122742A2DF98D
:202E000074363CFA7B8190002023E07E0029F9EE3AFA12002004FF90002024E0FBA3E0FA00
:202E2000A3E0F9EF1200201A7F0022A907EA9000203EF0EBA3F0A37405F09000203FE090D9
:202E4000007084F09000203EE090007085F090007080E04401F090007082E9F0A3EDF07B60
:202E6000E87A0390007080E0FF20E709EB1B70011A144A70EEEB4A60037F00229000204008
:202E8000E014F070B57F0122E4FFC0077F4CFEFDFC9000202312002166900020277401F073
:202EA000A37420F0A37405F0D00712002B5B90002005E0FCA3E0FDA3E0FEA3E0FF780412CE
:202EC0000020EBE4AD07AC067E217FCF1200240322EFC3940C5008E490002022F0800790EE
:202EE0000020227401F090002022E075F004A42475F9743635F0FA7B811200211122EF754B
:202F0000F072A42408F9743635F0FA7B81120020047F017001FF22E4FFFEFDFC90002032BD
:202F2000E0FBA3E0FAA3E0F91200212E7F012212002D55E4FFFE0FBF00010EBE4EF8BF2085
:202F4000F50200256B90007080E054FBF0A3E054F84402F07F00223099FDC2998F99221228
:202F6000002F45227F01227F0122040040540324055505004054032405550400410061247A
:202F8000FF9B0400410C0000A00004004104111100000480410422223434050041006124FB
:202FA000FF9B0500410C0000A000050041041111000005804104222234340000000000069D
:202FC000600A050040340000014C06000000000060A10204000009000011000000A02603D1
:202FE000803F000000A400010019078000040200000004004030128398A4048040301EE68A
:20300000B16A050040300149CA300400405402C40001040040540004014004004054000404
:2030200081400400405402C400000400405402C50001040040540005014004004054000596
:2030400081400400405402C500000400405402C60001040040540006014004004054000672
:2030600081400400405402C600000400405402C7000104004054000701400400405400074E
:2030800081400400405402C700000400405402C8000104004054000801400400405400082A
:2030A00081400400405402C800000400405402C90001040040540009014004004054000906
:2030C00081400400405402C900000400405402CA000104004054000A014004004054000AE2
:2030E00081400400405402CA00000400405402CB000104004054000B014004004054000BBE
:2031000081400400405402CB00000400405402CC000104004054000C014004004054000C99
:2031200081400400405402CC00000400405402CD000104004054000D014004004054000D75
:2031400081400400405402CD00000400405402CE000104004054000E014004004054000E51
:2031600081400400405402CE00000400405402CF000104004054000F014004004054000F2D
:2031800081400400405402CF00000500405402D00002050040540010004005004054001006
:2031A00080400500405402D000000500405402D080000500405402D10002050040540011E1
:2031C000004005004054001180400500405402D100000500405402D180000500405402D280
:2031E0000003050040540212711E050040540232441005004054025242050500405402D2CE
:2032000000020500405400120040050040540012804004004054021205880500405402D2B0
:2032200000000500405402D280000500405402D30003050040540213711E05004054023325
:20324000441005004054025342050500405402D300020500405400130040050040540013DD
:20326000804004004054021305880500405402D300000500405402D3800004004040000173
:203280009015048040400001901505004040000190150580404000019015040000100000F5
:2032A00078CC04000110000078CC04000210000078CC04000310000078CC040004100000A4
:2032C00078CC04000510000078CC04800010000078CC04800110000078CC04800210000006
:2032E00078CC04800310000078CC04800410000078CC04800510000078CC050000100000E1
:2033000078CC05000110000078CC05000210000078CC05000310000078CC0500041000003F
:2033200078CC05000510000078CC05800010000078CC05800110000078CC058002100000A1
:2033400078CC05800310000078CC05800410000078CC05800510000078CC04004028001016
:203360000000048040280010000005004028001000000580402800100000040000001403BC
:2033800002010400010014030203040002001403020504000300140302070400040014039F
:2033A0000209040005001403020B048000001403020D048001001403020F048002001403E1
:2033C00002110480030014030213048004001403021504800500140302170500000014039C
:2033E0000219050001001403021B050002001403021D050003001403021F050004001403DB
:2034000002210500050014030223058000001403022505800100140302270580020014031C
:203420000229058003001403022B058004001403022D058005001403022F01800500080462
:2034400002010181050008040201020400040000FA500200000040000000020010004000EB
:20346000000002002000400000000200300040000000020040004000000002005000400064
:20348000000002006000400000000200700040000000020080004000000002009000400044
:2034A00000000200A000400000000200B000400000000200C000400000000200D000400024
:2034C00000000200E000400000000200F00040000000020100004000000002011000400002
:2034E0000000020120004000000002013000400000000201400040000000020150004000E0
:2035000000000201600040000000020170004000000004004054032405550500405403247C
:203520000555040041006124FF9B0400410C0000A000040041041111000004804104222264
:203540003434050041006124FF9B0500410C0000A000050041041111000005804104222232
:203560003434030000007FCFF7FC0300003000FFFFFF018000040392FBF3030000200780BD
:20358000C826030000240400740E01800C800000310801810C800000310801800C00000076
:2035A000310901800C100000310901800C200000310901800C300000310901810C0000008E
:2035C000310901810C100000310901810C200000310901810C3000003109000000000006F3
:2035E000600B0500405400128940050040540013894005004054001291400500405400134F
:2036000091400D1411AB0110181F000102030405060708090A0B0C0D0E0F101112131415CD
:20362000161700000000000000000405060708090A0B0C0D0E0F1011121308090A0B0C0D66
:203640000E0F140000000000000003030303030303030303030303030303030303030303F7
:20366000030300000000000000020000000000000000FFFF010400405405004054FFFFFF15
:20368000FFFFFFFFFFFFFFFFFFFFFFFFFFFFFFFFFFFFFFFFFFFFFFFFFFFFFFFFFFFFFFFF4A
:2036A000FFFFFFFFFFFFFFFFFFFFFFFFFFFFFFFFFFFFFFFFFFFFFFFFFFFFFFFFFFFFFFFF2A
:2036C000FFFFFFFFFFFFFFFFFFFFFFFFFFFFFFFFFFFFFFFFFFFFFFFFFFFFFFFFFFFFFFFF0A
:2036E000FFFFFFFFFFFFFFFFFFFFFFFFFFFFFFFFFFFFFFFFFFFFFFFFFFFFFFFFFFFFFFFFEA
:203F0000120021EE22FFFFFFFFFFFFFFFFFFFFFFFFFFFFFFFFFFFFFFFFFFFFFFFFFFFFFF79
:203F2000FFFFFFFFFFFFFFFFFFFFFFFFFFFFFFFFFFFFFFFFFFFFFFFFFFFFFFFFFFFFFFFFA1
:203F4000FFFFFFFFFFFFFFFFFFFFFFFFFFFFFFFFFFFFFFFFFFFFFFFFFFFFFFFFFFFFFFFF81
:203F6000FFFFFFFFFFFFFFFFFFFFFFFFFFFFFFFFFFFFFFFFFFFFFFFFFFFFFFFFFFFFFFFF61
:203F8000FFFFFFFFFFFFFFFFFFFFFFFFFFFFFFFFFFFFFFFFFFFFFFFFFFFFFFFFFFFFFFFF41
:208000000200C77D286E756C6C29002202051BD67400740002072ACF25730056312E312E5E
:208020003800740002073DA2716F73747970653D00716F73747970653D256400516F73202C
:20804000547970652053657474696E6700546F20656E61626C65203830322E317020516FCD
:20806000532C20596F75206E656564206368616E676520746F203830322E315120564C4172
:208080004E2E006367695F716F730070253032643D002564005761726E696E6700546F20A5
:2080A00073657420516F5320737570706F7274206F6E20616E7920706F72742C204A756D42
:2080C000626F204672616D6520737570706F7274206D7573742062652064697361626C65C3
:2080E000642E00706F72743D00706F72743D253032640073706565643D0073706565643D63
:208100002564007365745F666C6F773D007365745F666C6F773D2564006367695F7365742F
:20812000706F72743D256400506F72742053657474696E67004D656469612074797065202F
:208140006973206368616E6765642E3C62723E43757272656E74207370656564207365745D
:2081600074696E67206973206E6F74207375697461626C652E00766C616E5F69643D0076A9
:208180006C616E5F69643D256400646573633D002600564C414E2064657363726970746998
:2081A0006F6E206D75737420626520302D25642063686172616374657273006367695F61D9
:2081C0006464766C616E3F6E756D3D256400564C414E2053657474696E67007663623D002A
:2081E0007663623D25303264006367695F736574766C616E3D25640054686520766C616ED5
:208200002067726F757020706F7274206D7573742073657420746F207468652073616D65AD
:20822000207472756E6B2073657474696E67006E756D3D006E756D3D2564007663623D258C
:2082400064006367695F64656C766C616E0076747970653D0076747970653D25303264006D
:2082600044656661756C74007379733D006C6F633D006C6F67696E3D0053797374656D2027
:208280006E616D65206D75737420626520302D2564206368617261637465727300537973E8
:2082A00074656D2053657474696E67006367695F737973004C6F636174696F6E206E616DF4
:2082C00065206D75737420626520302D2564206368617261637465727300496E76616C69C0
:2082E00064206C6F67696E2074696D656F75742076616C756500646863703D006468637002
:208300003D25640069703D00496E76616C69642049502061646472657373006D6B3D00499D
:208320006E76616C6964207375626E6574206D61736B0067773D00496E76616C69642067D9
:20834000617465776179204950004950207375626E6574206D75737420657175616C2074DA
:208360006F2067617465776179207375626E65740061636C5F69643D0061636C5F69643D99
:20838000256400495020416363657373204C6973742053657474696E67006367695F616339
:2083A0006C00495020616464726573732063616E6E6F74206265207468652073616D6520E1
:2083C00061732053776974636800495020616464726573732063616E206E6F7420626520CE
:2083E0006475706C696361746564006F6C645F706173733D006E65775F706173733D0072BD
:20840000656E65775F706173733D004368616E67652050617373776F726400706173737773
:208420006F7264206C656E6774682063616E6E2774206265207A65726F006367695F7061D0
:2084400073730050617373776F72642053657474696E67004E65772050617373776F726448
:20846000206D75737420626520302D32302063686172616374657273006F6C64207061736A
:2084800073776F72642069732077726F6E67006E65772070617373776F7264206973206902
:2084A0006E636F6E73697374656E7400656E61626C65253032643D00746B70253032643DFE
:2084C000002530326426005472756E6B2053657474696E67005468652073656C6563746553
:2084E00064207472756E6B20706F72742073657474696E67206D7573742073657420746F69
:20850000207468652073616D652056414C4E2047726F7570006367695F7472756E6B006D83
:208520006F64653D006D6F64653D2530326400736E69666665723D00736E69666665723DA5
:2085400025303264006D63623D006D63623D2530326400647669643D005056494420536578
:208560007474696E6700496E76616C6964205649442076616C7565006367695F7076696489
:20858000005649442025303264206973206E6F742065786973742C6F7220506F727420251C
:2085A000303264206973206E6F7420746865206D656D626572206F662056494420253032F0
:2085C000642E00276367695F7076696427007669643D005649442053657474696E670056BF
:2085E0004944206D757374206265206265747765656E203220616E642034303934006367B4
:20860000695F6164647669640054686520564944207461626C652069732066756C6C0054B7
:2086200068652056494420697320657869737420696E20564944207461626C650070256406
:208640003D007461675F69643D007461675F69643D25640054686520564944206973206565
:208660007869737420564944207461626C65007669645F6D656D3D00546865206465666118
:20868000756C7420766964206F6620706F727420253032642069732025642C20736F2069E1
:2086A000742063616E6E277420626520756E73656C65637465642E00276367695F73657485
:2086C0007669643D2564270054686520766964206973207468652064656661756C742076EE
:2086E0006964206F6620706F727420253032642C20736F2069742063616E6E27742062655B
:208700002064656C657465642E006367695F7365747669643D25640052656D6F7665205669
:208720004C414E00506C65617365206D616B652073757265207468657265206973206E6F36
:2087400020656E74727920696E207468652074727573746564204D414320746861742075ED
:20876000736573207468652073616D6520564C414E2049442E007061737377643D00666CBA
:2087800061673D00666C61673D256400666173743D00666173743D256400627072693D002B
:2087A0005370616E6E696E6720547265652053657474696E6700496E76616C696420427232
:2087C00069646765205072696F72697479006367695F73747000626167653D00496E76613B
:2087E0006C696420427269646765204D617820416765006268656C6C6F3D00496E76616CB3
:208800006964204272696467652048656C6C6F2054696D650062646C61793D00496E766184
:208820006C69642042726964676520466F72776172642044656C61790064633D00496E765D
:20884000616C6964205061746820436F73742076616C75650064703D00496E76616C696403
:20886000205072696F726974792076616C75650000534E4D502053657474696E6700496E46
:2088800076616C696420534E4D5020486F73742049502E006367695F6E6577736E6D705FCC
:2088A000686F737400636F6D6D25643D00436F6D6D756E697479206E616D65206D75737419
:2088C00020626520302D25642063686172616374657273006367695F736E6D7000707269D0
:2088E00025643D0030007431616C6C3D0061646D696E007431616C6C3D25640028256429E0
:20890000543174726170323A25640A00747225643D0025732525640061646D696E25643D5B
:2089200000486F73742049702063616E206E6F74206265206475706C696361746564006D6A
:208940006163616464723D00667764706F72743D00667764706F72743D2530326400706634
:208960005F69643D0054727573746564204D41432053657474696E67006367695F736574D6
:2089800066776400564C414E2049442076616C7565206D757374206265206265747765650F
:2089A0006E203120616E64203430393400496E76616C696420564C414E2049442076616C8C
:2089C000756500506C6561736520696E70757420746865204D414320616464726573732E8D
:2089E00000506C6561736520636F727265637420746865204D414320616464726573732093
:208A0000666F726D61742E005468652074727573746564204D414320616C72656164792040
:208A200065786973747320696E20746865207461626C652E00546865204D414320697320BA
:208A40007468652073616D65206173207377697463682773204D41432E0054686520564CCD
:208A6000414E204944206D7573742062652063726561746564206265666F726520747275E4
:208A800073746564204D41432073657474696E672E006677623D006677623D256400627096
:208AA000747970653D006270747970653D256400656E61626C65645F666C61673D00656E89
:208AC00061626C65645F666C61673D256400546F20736574204A756D626F204672616D6588
:208AE000207374617475732C516F5320506F72742D426173656420737570706F72742073D2
:208B00007461747573206D757374206265207468652073616D65206F6E20616E7920706FC9
:208B200072742E006367695F6A756D626F00546F20736574204A756D626F204672616D651B
:208B4000207374617475732C516F532049454545203830322E315120737570706F72742013
:208B6000737461747573206D757374206265207468652073616D65206F6E20616E79207065
:208B80006F72742E00696E67726573734374726C3D00696E67726573734374726C3D25642F
:208BA00000696E6772657373526174653D00696E6772657373526174653D256C75004425BE
:208BC000643D00E5252407F582E4348BF583759308E005252290088B0430170490088B0755
:208BE000E475F0011200BCAC0200B31F2010E57F2ED2108018EF540F2490D43440D4FF3050
:208C0000140BEF24BFB41A0050032461FFE526600215260529E5297002052830171190084B
:208C20008B04E475F0011200BCACEF0200B3700200CA1A7403D2178003E4C217F525900895
:208C40008B041200BCDAE4F526F528F529E52660087F2012008C0D80F47527FFC211C21032
:208C6000C212C213C215C216C21812008BD5FF700E3017067F0012008C1EAF29AE2822B4C7
:208C80002563C2D5C21412008BD5FF24D0B40A00501A75F00A782630D50508B6FF0106C6B1
:208CA000A426F620D5047002D21380D824CFB41A00EF5004C2E5D21402008E4BD21180C4B9
:208CC000D21080BED21280BAD2D580B8D21580B27F2012008C0D2012077401B5260040F05B
:208CE00012008BC3FF12008C0D02008C4DD218D216808F12008BC3FB12008BC3FA12008B5C
:208D0000C3F94A4B700679227A8F7B8120123DE52660397E00E9C0E02EF9EAC0E03400FAF3
:208D20001200B31FF9D0E0FAD0E0C960060EEE652770E2C2D5EBC0E0EAC0E0E9C0E0EE12BE
:208D4000008E93D0E0F9D0E0FAD0E0FB1200B31FFF6096EBC0E0EAC0E0E9C0E012008C0DD2
:208D6000D0E02401F9D0E03400FAD0E0FBE5270460DAD527D702008CE97BFF7A8E798FD2AC
:208D8000128089791080027908C216C2188008D2D5790A8004790AC2D5E527047002F5278C
:208DA000E4FAFDFEFF12008BC3FC7B0820111612008BC3FD7B1030100C12008BC3FE120011
:208DC0008BC3FF7B20EC3382D592D55013C3E43010069FFFE49EFEE42011039DFDE49CFC32
:208DE000E4CBF8C211EC700CCFCECDCCE824F8F870F38017C3EF33FFEE33FEED33FDEC3326
:208E0000FCEB33FB994002FB0FD8E9EB301105F8D0E0C448B211C0E00AEC4D4E4F78207B5C
:208E20000070C2EAB5270040BCC0E012008E95D0F0D0E0201104C4C0E0C4B211C0F0120017
:208E40008BF6D0F0D5F0EA02008C4D1200B7F18CF3538D83588CC04C8CBC428D874F8D8FB2
:208E6000448D8F498CD6438D95558D79468D79458D79478F3F508CC42D8CC82E8CEF2B8CFA
:208E8000CC238CED208F2B2A8C824800008CE53F3F3F00790AA2D5201314301509B9100288
:208EA0000404B9080104A2D520160250010420126D9212B526005036C0E07F2030131A7F21
:208EC00030A21272167215501012008EEEC212C216C215C2187F308010301503E9C0E01232
:208EE000008C0D301503D0E0F9D0E0B526CA3015197F30B9100D12008C0D7F583014077F64
:208F0000788003B9080412008C0D3012067F2D02008C0D7F202018F77F2B2016F2229212F1
:208F200080CC286E756C6C2900D21112008BC33011F7C211782630D50108F602008C8212C7
:208F4000008BC37F4960087F4310E7027F5814C0E0EF12008BFE743A12008BFED0E0600D5D
:208F6000C0E0C412008BF6D0E012008BF6D21375260402008D836C6F676F2E6769660069A3
:208F80006E6465782E68746D006C6566742E68746D00746F702E68746D0068656C702E6880
:208FA000746D00666F6C642E67696600666F726D2E637373006C6566742E637373006865AD
:208FC0006C702E637373006461726B626C75652E676966006E6574676561722E6A7067003B
:208FE0006D6F64656C2E6A706700752E67696600622E67696600742E676966007400740092
:209000004753373136540000000000000000000000000000000000000000000000000000C4
:209020000000000000000000004753373136540000000000000000000000000000000000A4
:2090400000000000000000000000000000000000000056312E312E38000000000000740050
:2090600074000000000000000000000000000000000056312E312E3800001223344566001C
:2090800000000000000180C200000F74000A5B4D41435F49443D25785D0A000A5B50485951
:2090A0005F494425643D25785D0A00740088D89288D89A88D89D88D8A088DBC788DBCF88B9
:2090C000DBD588DBDC88DBE488DBEC61007400203C74643E0A203C73656C656374206E61EF
:2090E0006D653D25733E0A203C6F7074696F6E2076616C75653D25643E25730A003C747287
:209100003E3C746820636F6C7370616E3D343E25730A3C74723E0A203C74643E3C623E429E
:20912000797465730A203C746420636F6C7370616E3D333E256C750A0A003C74723E0A20CA
:209140003C74643E3C623E25730A203C74643E256C750A203C74643E3C623E25730A203C71
:2091600074643E256C750A0A007400740074000000000000007400740074007400740062BD
:209180007267436C656172566C616E506F7274735461626C6500000000000000000000007E
:2091A000000000000000000000000000000000000000000000000000000000000000008827
:2091C00003E7000062726744656C657465566C616E506F72747354626C456E74727900003A
:2091E00000000000000000000000000000000000000000000000000000000000000000006F
:209200000000000087385F00086272674765744D414346646254626C4669727374456E749F
:20922000727900000000000000000000000000000000000000000000000000000000000043
:2092400000000000000000000086F10B00006272674765744D414346646254626C4E657807
:2092600074456E747279000000000000000000000000000000000000000000000000000068
:20928000000000000000000000000000000087CB970000627267476574566C616E506F72C8
:2092A000747354626C4669727374456E74727900000000000000000000000000000000008B
:2092C00000000000000000000000000000000000000000882FE50000627267476574566CD5
:2092E000616E506F72747354626C4E657874456E74727900000000000000000000000000B4
:2093000000000000000000000000000000000000000000000000000087986C000062726787
:209320005365744D756C7469706C65566C616E496E7365727454626C456E7472790000007B
:209340000000000000000000000000000000000000000000000000000000000000853853FD
:20936000000F627267536574566C616E506F72747354626C456E747279000000000000009A
:209380000000000000000000000000000000000000000000000000000000000000000000CD
:2093A00000008712860008636F73476574546332557365725072696F54626C4669727374D5
:2093C000456E7472790000000000000000000000000000000000000000000000000000007B
:2093E00000000000000000883A4A0000636F73476574546332557365725072696F54626CB8
:209400004E657874456E74727900000000000000000000000000000000000000000000009B
:209420000000000000000000000000008793D60000636F73476574557365724E657750724C
:20944000696F32546354626C4669727374456E74727900000000000000000000000000000F
:209460000000000000000000000000000000000000883A3F0100636F7347657455736572E6
:209480004E65775072696F32546354626C4E657874456E747279000000000000000000004C
:2094A00000000000000000000000000000000000000000000000878F320100636F73476572
:2094C00074557365725072696F32546354626C4669727374456E74727900000000000000BA
:2094E000000000000000000000000000000000000000000000000000000000883A34000076
:20950000636F73476574557365725072696F32546354626C4E657874456E747279000000F1
:2095200000000000000000000000000000000000000000000000000000000000000000002B
:209540008799130000636F73536574546332557365725072696F54626C456E747279000011
:209560000000000000000000000000000000000000000000000000000000000000000000EB
:209580000000000000882DC20002636F73536574557365724E65775072696F3254635462DF
:2095A0006C456E74727900000000000000000000000000000000000000000000000000002D
:2095C00000000000000000000000882AA80102636F73536574557365725072696F3254639B
:2095E00054626C456E74727900000000000000000000000000000000000000000000000037
:20960000000000000000000000000000000000882D3B000267636F73476574506F72745592
:20962000703254635461626C654964780000000000000000000000000000000000000000C4
:20964000000000000000000000000000000000000000000087C7CA040067636F7353657416
:20966000506F727444656661756C74557365725072696F0000000000000000000000000047
:209680000000000000000000000000000000000000000000000000000087E9E205006763A9
:2096A0006F73536574506F727455703254635461626C65496478000000000000000000003C
:2096C00000000000000000000000000000000000000000000000000000000000000087EA19
:2096E00056050067666462466C75736800000000000000000000000000000000000000007A
:20970000000000000000000000000000000000000000000000000000000000000000000049
:20972000000000882A81020067766C6E536574506F72744163634672616D655479706500D8
:20974000000000000000000000000000000000000000000000000000000000000000000009
:20976000000000000000000087E8FA050067766C6E536574506F7274496E677265737346D2
:20978000696C746572696E670000000000000000000000000000000000000000000000006B
:2097A0000000000000000000000000000087E96E050067766C6E5365745076696400000050
:2097C000000000000000000000000000000000000000000000000000000000000000000089
:2097E00000000000000000000000000000000000000087E63D050067766C6E536574566918
:209800006452616E67650000000000000000000000000000000000000000000000000000F7
:209820000000000000000000000000000000000000000000000000882FC70100687750700A
:20984000526561645265674269744D61736B000000000000000000000000000000000000C3
:20986000000000000000000000000000000000000000000000000000000000008797C50302
:20988000006877507057726974655265674269744D61736B00000000000000000000000055
:2098A0000000000000000000000000000000000000000000000000000000000000000000A8
:2098C000008795CF0400706F7274476574506F727453746174757354626C4669727374451C
:2098E0006E747279000000000000000000000000000000000000000000000000000000009B
:2099000000000000000088389E0000706F7274476574506F727453746174757354626C4E6B
:20992000657874456E747279000000000000000000000000000000000000000000000000C4
:209940000000000000000000000000859E2C0000706F7274476574706F7274734D61634347
:209960006F756E7465727354626C4669727374456E7472790000000000000000000000009B
:209980000000000000000000000000000000000088388E0000706F7274476574706F7274CF
:2099A000734D6163436F756E7465727354626C4E657874456E7472790000000000000000FD
:2099C00000000000000000000000000000000000000000000086BFCE0000706F72745365F7
:2099E00074506F72744374726C54626C456E74727900000000000000000000000000000085
:209A0000000000000000000000000000000000000000000000000000000085997E00237017
:209A2000736D6952656164506F7274536D695068795265676973746572000000000000001D
:209A400000000000000000000000000000000000000000000000000000000000000000877F
:209A6000B90F050070736D695772697465506F72745068795265676973746572000000003A
:209A80000000000000000000000000000000000000000000000000000000000000000000C6
:209AA0000000000087DC3506007472756E6B44656C6574655472756E6B47727054626C45DD
:209AC0006E74727900000000000000000000000000000000000000000000000000000000B9
:209AE000000000000000000000878BD600077472756E6B4765745472756E6B477270546230
:209B00006C4669727374456E747279000000000000000000000000000000000000000000BF
:209B2000000000000000000000000000000088362900007472756E6B4765745472756E6BD6
:209B400047727054626C4E657874456E747279000000000000000000000000000000000009
:209B60000000000000000000000000000000000000000087CA8200007472756E6B536574B2
:209B80005472756E6B47727054626C456E7472790000000000000000000000000000000054
:209BA000000000000000000000000000000000000000000000000000870C7300077663744B
:209BC0004765744361626C6544696167000000000000000000000000000000000000000019
:209BE000000000000000000000000000000000000000000000000000000000000086844219
:209C0000040000000000000000000000000000000000000000000000000000000000000040
:209C2000000000000000000000000000000000000000000000000000000000000000000024
:209C400000000000000000447EDB0000012C417EB50042A6700000438C03FFFFFF4AA21C97
:209C60000000000000000000000041A684FF41ABF201428DEA000A428DF20000428DE60062
:209C800000428DE80000428DE20000428DF40000428DECFFFF428DE48000448DDE000000FE
:209CA00000428DD80000428DDA0000428DDC0000416AC9004699EFFFFFFFFFFFFF4699E5A9
:209CC0000180C200000043926681908B42925E7F7F4692690180C20000004692580180C243
:209CE0000000024692600180C2000003428B7700004F97FE88CF6C88CF7888CF8988CF9B58
:209D000088CF894C9ECC8983BB8983C38983C68983C94C7CD389000789000E89001289008A
:209D200019587CBB89001E89002689002E890037890040890049890050890057587D1289EA
:209D4000005F89006789007189007B89008489008D89001E89009260277CEB89009789003A
:209D6000A18900AB8900B78900C38900CF8900DB8900E68900F18900FC89010789010C89A8
:209D80000092467CDF89010C890114467CE589011B89011F43AAC989DE0B4890C2000100A4
:209DA00009001100194890D2000800100018001A43746F00000063534559883D7E6367698C
:209DC0005F64756D7900000000000000000000000085B9056367695F6C6F67696E00000077
:209DE0000000000000000000864B0A6367695F706F727400000000000000000000000082AF
:209E0000D8A16367695F736574706F727400000000000000000084F7C76367695F766C610F
:209E20006E0000000000000000000000008581BF6367695F736574766C616E000000000060
:209E40000000000084ACE76367695F64656C766C616E000000000000000000875AC7636701
:209E6000695F667764000000000000000000000000008603CA6367695F7365746677640067
:209E80000000000000000000008491D56367695F64656C66776400000000000000000000D0
:209EA00087EF316367695F64756D7066776400000000000000000083F82C6367695F707653
:209EC000696400000000000000000000000082C7F36367695F7669640000000000000000A4
:209EE0000000000000837A6B6367695F61646476696400000000000000000000829B61631B
:209F000067695F64657669636500000000000000000000827F246367695F64657461696C78
:209F2000000000000000000000008435776367695F73746174697374000000000000000053
:209F4000008590136367695F7472756E6B00000000000000000000008355C56367695F6D77
:209F60006972726F7200000000000000000000881A0D6367695F6A756D626F000000000055
:209F800000000000000086A4566367695F73746F726D6374726C00000000000000865830B7
:209FA0006367695F7061737300000000000000000000000082BF316367695F7379730000F5
:209FC0000000000000000000000000880D406367695F6261636B75700000000000000000A4
:209FE0000000865CF26367695F62616B5F646174610000000000000000880D8D6367695F20
:20A0000072657365740000000000000000000000882D186367695F716F730000000000006B
:20A0200000000000000000872C1B6367695F7170626173650000000000000000000087239A
:20A040005F6367695F71746F7300000000000000000000000086B3006367695F71647363D2
:20A060007000000000000000000000008741866367695F713170000000000000000000007E
:20A080000000008362376367695F7374700000000000000000000000000082F6D963676937
:20A0A0005F736E6D7000000000000000000000000082FDD86367695F61636C00000000006A
:20A0C00000000000000000008698046367695F61646461636C0000000000000000000085EE
:20A0E000E2E86367695F64656C61636C00000000000000000000000000000000000000009F
:20A100000000000000000000000000000042A9FE0000427D920000427D9400004231D80067
:20A120000042366500004233CB00044933AA81C63181C63F81C66752359581C67E81C6956F
:20A1400081C6AB81C6C181C6D981C6F54C363D81C71281C72F81C74D81C7646032366700A9
:20A160000000000000000000000000000000000000000000000000000000000000000000DF
:20A18000000000000000000000000000000000000060643174000100030006000100040047
:20A1A0000111AE000B000500010000000000000000000000000000000000000000000000CE
:20A1C0000000000000000B0000000000000000000000000000000000000000000000000074
:20A1E000000000000000000000000000000000000000000000000000006064334600010021
:20A2000003000600010004000111AE000B000500020000000000000000000000000000005E
:20A2200000000000000000000000000000000B000000000000000000000000000000000013
:20A240000000000000000000000000000000000000000000000000000000000000000000FE
:20A2600000609632B0000100030006000100020001000200020001000100FF0000000000F3
:20A28000000000000000000000000000000000000000000000000B000100030006000100A8
:20A2A00004000111AE000B00050003000000000000000000000000000000000000000000C7
:20A2C00000000000000000000B000000000000000000000000000000000000000000000073
:20A2E000000000000000000000000000000000000000000000000000000000609635A7008C
:20A300000100030006000100020001000200020001000100FF00000000000000000000002A
:20A32000000000000000000000000000000000000B00010003000600010004000111AE0043
:20A340000B00050004000000000000000000000000000000000000000000000000000000E9
:20A3600000000B0000000000000000000000000000000000000000000000000000000000D2
:20A380000000000000000000000000000000000000000000006064310C00010003000600B2
:20A3A000010004000111AE000B0005000500000000000000000000000000000000000000C3
:20A3C000000000000000000000000B00000000000000000000000000000000000000000072
:20A3E000000000000000000000000000000000000000000000000000000000000060643069
:20A40000A800010003000600010004000111AE000B000500060000000000000000000000AF
:20A420000000000000000000000000000000000000000B0000000000000000000000000011
:20A440000000000000000000000000000000000000000000000000000000000000000000FC
:20A4600000000000006064304200010003000600010004000111AE000B00050007000000C0
:20A4800000000000000000000000000000000000000000000000000000000B0000000000B1
:20A4A00000000000000000000000000000000000000000000000000000000000000000009C
:20A4C00000000000000000000000000000606431DE00010003000600010004000111AE00DA
:20A4E0000B0005000800000000000000000000000000000000000000000000000000000044
:20A5000000000B000000000000000000000000000000000000000000000000000000000030
:20A520000000000000000000000000000000000000000000006064324200010003000600D9
:20A54000010004000111AE000B00050009000000000000000000000000000000000000001D
:20A56000000000000000000000000B000000000000000000000000000000000000000000D0
:20A5800000000000000000000000000000000000000000000000000000000000004432AC99
:20A5A000093174004433C7093346004433C30932B00144364D0935A7014432A609310C00F8
:20A5C0004431DA0930A800443170093042004433BB0931DE004433BF09324200423040003C
:20A5E000004AA2A8FC06FC03FC0400A120004241DB000143AAEA89DE0D43AAED89DE0F43C8
:20A60000AAF089DE114C913089C9E289C9E989C9ED89C9F44C912489C9F989CA0889CA1E0F
:20A6200089CA284C9EF089BD1D89BD2489BD2889BD2F43AAF389DE1343A95A89DE15604059
:20A64000847100081018202830380A121A220C141C240E161E262E01020304050607090BA7
:20A660000D0F11131517191B1D1F21232527292A2B2C2D2F31323334353637393A3B3C3DD5
:20A680003E3F46A85B893E8D893E8E42A2B4000142A2B2000042A2B8000042A2BA0001429F
:20A6A000A2B60000427C49000454712F00010003000600010004000111AE00640004000309
:20A6C00043AAFC818010427EB3740060597E5A4E6F74653A3C62723E0A54313A20617574B7
:20A6E00068656E7469636174696F6E206661696C3C62723E0A54323A206465766963652040
:20A70000626F6F7475703C62723E0A54333A206C696E6B207570202F206C696E6B20646FA4
:20A72000776E3C62723E0A004F9B3089278889279089279689279D8927A643416881906004
:20A7400060283C8700000000000000000000000000000000000000000000000000000000AE
:20A7600000000000000000000000000062103F5200000000000000000000000000000000D6
:20A780000000000000000000000000000000000000000000000000000000000000000000B9
:20A7A000000000000000000000000000000000000000000000000000000000000000000099
:20A7C000000000000000000000000000000000000000000000000000000000000000000079
:20A7E000000000000000000000000000000000000000000000000000000000000000000059
:20A80000000000000000000000000000000000000000000000000000000000000000000038
:20A82000000000000000000000000000000000000000000000000000000000000000000018
:20A840000000000000000000000000000000000000000000000000000000000000000000F8
:20A860000000000000000000000000000000000000000000000000000000000000000000D8
:20A880000000000000000000000000000000000000000000000000000000000000000000B8
:20A8A000000000000000000000000000000000000000000000000000000000000000000098
:20A8C000000000000000000000000000000000000000000000000000000000000000000078
:20A8E000000000000000000000000000000000000000000000000000000000000000000058
:20A90000000000000000000000000000000000000000000000000000000000000000000037
:20A92000000000000000000000000000000000000000000000000000000000000000000017
:20A940000000000000000000000000000000000000000000000000000000000000000000F7
:20A960000000000000000000000000000000000000000000000000000000000000000000D7
:20A9800062103CAF000000000000000000000000000000000000000000000000000000005A
:20A9A000000000000000000000000000000000000000000000000000000000000000000097
:20A9C000000000000000000000000000000000000000000000000000000000000000000077
:20A9E000000000000000000000000000000000000000000000000000000000000000000057
:20AA0000000000000000000000000000000000000000000000000000000000000000000036
:20AA2000000000000000000000000000000000000000000000000000000000000000000016
:20AA40000000000000000000000000000000000000000000000000000000000000000000F6
:20AA60000000000000000000000000000000000000000000000000000000000000000000D6
:20AA80000000000000000000000000000000000000000000000000000000000000000000B6
:20AAA000000000000000000000000000000000000000000000000000000000000000000096
:20AAC000000000000000000000000000000000000000000000000000000000000000000076
:20AAE000000000000000000000000000000000000000000000000000000000000000000056
:20AB0000000000000000000000000000000000000000000000000000000000000000000035
:20AB2000000000000000000000000000000000000000000000000000000000000000000015
:20AB40000000000000000000000000000000000000000000000000000000000000000000F5
:20AB60000000000000000000000000000000000000000000000000000000000000000000D5
:20AB80000000000000000000000000000000000000000000503F42000000000000000000E4
:20ABA00000000000000000602041AC00000000000000000000000000000000000000000028
:20ABC00000000000000000000000006020416B000000000000000000000000000000000049
:20ABE00000000000000000000000000000000060203EC800000000000000000000000000CF
:20AC0000000000000000000000000000000000000000006020418C000000000000000000E7
:20AC2000000000000000000000000000000000000000000000000060503EEE000000000038
:20AC40000000000000000000000000000000000000000000000000000000000000000000F4
:20AC60000000000000000000000000000000000000000000000000000000000000000000D4
:20AC80000000000000000000000000413EC3014641620180C200000041418B00423EEC00CC
:20ACA0000043AB1189DE1743AB148191754496780000000044967C00000014449674000084
:20ACC000000143AB2081801243AB2381802243AB26818FFC43AB29818FFE43AB2C81CB4D26
:20ACE00043AB2F81CB4F419DD600449DD700000000624059580000000000000000000000DD
:20AD0000000000000000000000000000000000000000000000000000000000000000000033
:20AD2000000000000000000000000000000000000000000000000000000000000000000013
:20AD40000000000000000000000000000000000000000000000000000000000000000000F3
:20AD60000000000000000000000000000000000000000000000000000000000000000000D3
:20AD80000000000000000000000000000000000000000000000000000000000000000000B3
:20ADA000000000000000000000000000000000000000000000000000000000000000000093
:20ADC000000000000000000000000000000000000000000000000000000000000000000073
:20ADE000000000000000000000000000000000000000000000000000000000000000000053
:20AE0000000000000000000000000000000000000000000000000000000000000000000032
:20AE2000000000000000000000000000000000000000000000000000000000000000000012
:20AE40000000000000000000000000000000000000000000000000000000000000000000F2
:20AE60000000000000000000000000000000000000000000000000000000000000000000D2
:20AE80000000000000000000000000000000000000000000000000000000000000000000B2
:20AEA000000000000000000000000000000000000000000000000000000000000000000092
:20AEC000000000000000000000000000000000000000000000000000000000000000000072
:20AEE000000000000000000000000000000000000000000000000000000000000000000052
:20AF0000000000000000000000000000000000000000000000000000000000000000000031
:20AF20000000000000000000000000000000000000000000004E984A09984A09984A09986A
:20AF40004A0000000000489A550000000000000000489A5D000000000000000041AC130031
:20AF600041A9A70044A9A3000000006040040000000000000000000000000000000000000C
:20AF80000000000000000000000000000000000000000000000000000000000000000000B1
:20AFA00000000000000000000000000000000062C00440000000000000000000000000002B
:20AFC000000000000000000000000000000000000000000000000000000000000000000071
:20AFE000000000000000000000000000000000000000000000000000000000000000000051
:20B00000000000000000000000000000000000000000000000000000000000000000000030
:20B02000000000000000000000000000000000000000000000000000000000000000000010
:20B040000000000000000000000000000000000000000000000000000000000000000000F0
:20B060000000000000000000000000000000000000000000000000000000000000000000D0
:20B080000000000000000000000000000000000000000000000000000000000000000000B0
:20B0A000000000000000000000000000000000000000000000000000000000000000000090
:20B0C000000000000000000000000000000000000000000000000000000000000000000070
:20B0E000000000000000000000000000000000000000000000000000000000000000000050
:20B1000000000000000000000000000000000000000000000000000000000000000000002F
:20B1200000000000000000000000000000000000000000000000000000000000000000000F
:20B140000000000000000000000000000000000000000000000000000000000000000000EF
:20B160000000000000000000000000000000000000000000000000000000000000000000CF
:20B180000000000000000000000000000000000000000000000000000000000000000000AF
:20B1A00000000000000000000000000000000000000000000000000000000000000000008F
:20B1C00000000000000000000000000000000000000000000000000000000000000000006F
:20B1E00000000000000000000000000000000000000000000000000000000000000000004F
:20B2000000000000000000000000000000000000000000000000000000000000000000002E
:20B2200000000000000000000000000000000000000000000000000000000000000000000E
:20B240000000000000000000000000000000000000000000000000000000000000000000EE
:20B260000000000000000000000000000000000000000000EB7008E709F608DFFA801B8980
:20B28000828A831410E70AF593E0A3F608DFFA8009F593E493A3F608DFF9ECFAA9F0EDFBC0
:20B2A0002288F0EF60010E4E60F088F0ED60C51410E7E7CB700E88828C838B93E709F0A379
:20B2C000DFFA80D61410E72A89828A83F593ECFAE0A3C8C582C8CCC583CCCBC593CBF0A3C9
:20B2E000C8C582C8CCC583CCCBC593CBDFE2DEE080AA89828A83F593ECFAE493A3C8C58251
:20B30000C8CCC583CCCBC593CBF0A3C8C582C8CCC583CCCBC593CBDFE1DEDF0200B29CEBA7
:20B320007002E72289828A831410E704F593E022F593E49322F8EB7006E7C828F3E822890A
:20B34000828A831410E708F593E0C828F0E822F593E49322BB000327F722F8EB89828A83DF
:20B360001410E706F593E028F022F593E4932822BB0002F722BB8000500989828A838B9331
:20B380001593F022EF8DF0A4A8F0CF8CF0A428CE8DF0A42EFE22BC000BBE0029EF8DF08459
:20B3A000FFADF022E4CCF875F008EF2FFFEE33FEEC33FCEE9DEC984005FCEE9DFE0FD5F0B6
:20B3C000E9E4CEFD22EDF8F5F0EE008420D21CFEADF075F008EF2FFFED33FD4007985006F2
:20B3E000D5F0F222C398FD0FD5F0EA22C2D5EC30E709B2D5E4C39DFDE49CFCEE30E716B288
:20B40000D5E4C39FFFE49EFE1200B396C3E49DFDE49CFC80041200B39630D507C3E49FFF4A
:20B42000E49EFE22C5F0F8A3E028F0C5F0F8E582158270021583E038F022A3F8E0C5F025EE
:20B44000F0F0E582158270021583E0C838F0E822EB7007E7F5F009E7192289828A83141095
:20B46000E708F593E0F5F0A3E022F593E493F5F074019322F8EB700C09E5F027C7F5F019B4
:20B48000E837C72289828A831410E707F593E80200B43AF593E4740193F5F0E49322BB006D
:20B4A0000B09C5F027F7C5F01937F722F8EB89828A831410E707F593E80200B424F5937434
:20B4C000019325F0F5F0E4933822BB0006F709A7F01922BB8000500D89828A838B93159304
:20B4E000F0E5F0A3F022E88FF0A4CC8BF0A42CFCE98EF0A42CFC8AF0EDA42CFCEA8EF0A442
:20B50000CDA8F08BF0A42DCC3825F0FDE98FF0A42CCD35F0FCEB8EF0A4FEA9F0EB8FF0A48C
:20B52000CFC5F02ECD39FEE43CFCEAA42DCE35F0FDE43CFC2275F008758200EF2FFFEE33AE
:20B54000FECD33CDCC33CCC58233C5829BED9AEC99E58298400CF582EE9BFEED9AFDEC999B
:20B56000FC0FD5F0D6E4CEFBE4CDFAE4CCF9A88222B800C1B90059BA002DEC8BF084CFCEDE
:20B58000CDFCE5F0CBF97818EF2FFFEE33FEED33FDEC33FCEB33FB10D703994004EB99FBE6
:20B5A0000FD8E5E4F9FA227818EF2FFFEE33FEED33FDEC33FCC933C910D7059BE99A4007AC
:20B5C000EC9BFCE99AF90FD8E0E4C9FAE4CCFB2275F010EF2FFFEE33FEED33FDCC33CCC8D0
:20B5E00033C810D7079BEC9AE899400AED9BFDEC9AFCE899F80FD5F0DAE4CDFBE4CCFAE40E
:20B60000C8F922CFF4CFCEF4CECDF4CDCCF4CC22C3E49FFFE49EFEE49DFDE49CFC22EB9F7E
:20B62000F5F0EA9E42F0E99D42F0EC6480C864809845F022EB9FF5F0EA9E42F0E99D42F067
:20B64000E89C45F022E8600FECC313FCED13FDEE13FEEF13FFD8F122E8600FEFC333FFEEE9
:20B6600033FEED33FDEC33FCD8F122EB7006E9F80200BC2489828A831410E706F59302009F
:20B68000BC30F5930200B6C0BB0006E9F80200BC85BB8000500C89828A838B931593020062
:20B6A000B75722EB7006E9F80200BC6E89828A831410E706F5930200B72BF5930200B6C057
:20B6C000E493FC740193FD740293FE740393FF22EB7006E9F80200BC3C89828A831410E761
:20B6E00006F5930200BC49F5930200BC557401FF3395E0FEFDFCA3A3A3E0CF2FF0E58215D4
:20B700008270021583E0CE3EF0E582158270021583E0CD3DF0E582158270021583E0CC3CEF
:20B72000F0227401FF3395E0FEFDFCA3A3A3E02FFFF0E582158270021583E03EFEF0E58282
:20B74000158270021583E03DFDF0E582158270021583E03CFCF022ECF0A3EDF0A3EEF0A38C
:20B76000EFF022F5F0C582A4C582C5F0C583A42583F58322A42582F582E5F03583F58322E5
:20B78000EB7006E9F80200BC9189828A831410E706F5930200BCA3F5930200BCE3BB001C06
:20B7A000D093D0F0D0E0F8D0E0C9FBD0E0FAD0E0CBC8C0E0C0F0C0930200BC9ABB800050D7
:20B7C00022D093D0F0D0E0F8D0E0C9F582D0E0CAF583D0E0CB14C8C0E0C0F0C09388930283
:20B7E00000BCDAD093D083D082D0E0D0E0D0E0E473D093D083D082F8E493701274019370D3
:20B800000DA3A393F8740193F5828883E4737402936860EFA3A3A380DFD093D083D082F861
:20B82000E4937012740193700DA3A393F8740193F5828883E473740293B5F00674039368B2
:20B8400060E9A3A3A3A380D8D093D083D082E4937012740193700DA3A393F8740193F582E5
:20B860008883E4737402936C70127403936D700C7404936E70067405936F60DDA3A3A3A349
:20B88000A3A380CA8B938A838982159353937FE473759308E5512582F582E5503583F583B5
:20B8A000B550048582512210AF06858251F55022858251F550D2AF22759308E5512582F55F
:20B8C00082E5503583F58322EB700C87F009E608B5F041603F80F489828A831410E70FF56A
:20B8E00093E0F5F0A3E608B5F02A602880F3F593E493F5F0A3E608B5F01A601880F2CB703C
:20B900001588828C838B9387F009E493A3B5F004600280F380611410E72E89828A83F59309
:20B92000ECFAE0F5F0A3C8C582C8CCC583CCCBC593CBE493A3C8C582C8CCC583CCCBC59320
:20B94000CBB5F033603180DA89828A83F593ECFAE493F5F0A3C8C582C8CCC583CCCBC593FA
:20B96000CBE493A3C8C582C8CCC583CCCBC593CBB5F004600280D97F00F845F0600EE86374
:20B98000F0806480D395F01F40027F01220200B8C80200B8FEED60F51410E7F5CB701488A5
:20B9A000828C83F59387F009E0A3B5F0CA60C880F480C41410E72D89828A83F593ECFAE07E
:20B9C000F5F0A3C8C582C8CCC583CCCBC593CBE0A3C8C582C8CCC583CCCBC593CBB5F097D6
:20B9E000609580DB89828A83F593ECFAE493F5F0A3C8C582C8CCC583CCCBC593CBE0A3C882
:20BA0000C582C8CCC583CCCBC593CBB5F0A360A180DAEB7008E709F60870FA801B89828ABB
:20BA2000831410E70AF593E0A3F60870FA8009F593E493A3F60870F9ECFAA9F0EDFB228858
:20BA4000F0ED60CE1410E7F0CB700E88828C83F593E709F0A370FA80DF1410E72889828AE2
:20BA600083F593ECFAE0A3C8C582C8CCC583CCCBC593CBF0A3C8C582C8CCC583CCCBC59340
:20BA8000CB70E280B589828A83F593ECFAE493A3C8C582C8CCC583CCCBC593CBF0A3C8C5EF
:20BAA00082C8CCC583CCCBC593CB70E1808CEB700C87F009E608B5F019DFF6801589828A7F
:20BAC000831410E711F593E0F5F0A3E608B5F002DFF50200BB5FF593E493F5F0A3E608B528
:20BAE000F07DDFF48079CB701388828C838B9387F009E493A3B5F067DFF580631410E730F0
:20BB000089828A83F593ECFAE0F5F0A3C8C582C8CCC583CCCBC593CBE493A3C8C582C8CCD5
:20BB2000C583CCCBC593CBB5F035DFDCDEDA802F89828A83F593ECFAE493F5F0A3C8C58273
:20BB4000C8CCC583CCCBC593CBE493A3C8C582C8CCC583CCCBC593CBB5F004DFDBDED97FF7
:20BB6000FFB5F0020F2240027F01220200BAAE0200BAE688F0EF60010E4E60EEED60EC143F
:20BB800010E7ECCB701288828C83F59387F009E0A3B5F0CBDFF680C71410E72F89828A83F3
:20BBA000F593ECFAE0F5F0A3C8C582C8CCC583CCCBC593CBE0A3C8C582C8CCC583CCCBC540
:20BBC00093CBB5F09ADFDDDEDB809489828A83F593ECFAE493F5F0A3C8C582C8CCC583CC03
:20BBE000CBC593CBE0A3C8C582C8CCC583CCCBC593CBB5F004DFDCDEDA0200BB5FEF4E605A
:20BC000022EF60010EEDBB0007F709DFFCA9F022BB8000500E89828A838B931593F0A3DF76
:20BC2000FCDEFA22E6FC08E6FD08E6FE08E6FF22E0FCA3E0FDA3E0FEA3E0FF22E6FB08E6F6
:20BC4000F908E6FA08E6CBF822E0F8A3E0F9A3E0FAA3E0FB22E493F8740193F9740293FA4C
:20BC6000740393FB227401FF3395E0FEFDFC080808E62FFFF618E63EFEF618E63DFDF618F2
:20BC8000E63CFCF622ECF608EDF608EEF608EFF622E6FB08E6FA08E6F922EBF608EAF60803
:20BCA000E9F622E0FBA3E0FAA3E0F922F8E0FBA3A3E0F925F0F0E582158270021583E0FAB4
:20BCC00038F022F8E0FBA3A3E025F0F9F0E582158270021583E038FAF022EBF0A3EAF0A3FC
:20BCE000E9F022E493FB740193FA740293F922E52A301C0104F8232824D8F582E43489F505
:20BD00008375930822900889D5301C04900889D8E475F0011200BCAC0200B31F60E6C52E5E
:20BD20007002152D14C52E201C05FF0200CB37900889D574FFF5F00200BCC3FF0207363DBA
:20BD4000E52B6006D52B037F0022201C101200CAECEF6008052EE52E7002052D2290088931
:20BD6000D51200BCA31200B31FFF60E5900889D5E475F0011200BCAC80D71200BD4AEFC07C
:20BD8000E01200BD3BD0E040F18091D21C8002C21C900889D51200BCDAE4F52CF52AF52D95
:20BDA000F52E752B00C21BC219C21AC21D1200BD05FF7005AF2C7E0022B425321200BD05AB
:20BDC000FF24D0B40A00500C75F00AC52BA4252BF52B80E824CFB41A00EF5002C2E50200D0
:20BDE000C025D21A80D6D21980D2D21D80CEEF1200BD3B50091200BD7AEF600F80A4EFC0D6
:20BE0000E01200BD4AD0E06F6098EF70040200BE951200BD1C809D1200BD4AEF6077E52B63
:20BE20007008052B80041200BD4AEF6017201D111200BCEFE475F0011200BCACEF1200B3D4
:20BE400070D52BE2201D04052A052C80AF1200BD40EFC0E01200BD3BD0E050051200BD1C28
:20BE6000E4FF201D111200BCEFE475F0011200BCACEF1200B370EF70D4201D04052A052C18
:20BE80000200BDFCE52B6002052B1200BD7A1200BD40EF70BD301C05E41200BD1CE52C6040
:20BEA000030200BDB47EFF7FFF22201D1474FFFCFDFEFF1200BCEF1200BCA31200B68805B2
:20BEC0002A0200BDA2D0E080CC7900800A7910800679088002790AD21EE52B6002052BE9C8
:20BEE000C0E01200BD7AEF60DC1200BD4ABF2D04D21B8003BF2B0B1200BD7AEF60C712004F
:20BF0000BD40D0E0B40A028034B40802802FBF302870027408C21EC0E01200BD40D0E0BF90
:20BF200078028003BF5816052BD52B028007D52B04D21E800B7410801B7002740ABF000BC6
:20BF4000EFF8E4FCFDFEFF0200BFCDC0E0EF1200BD1CD0E0F9E4FCFDFEFFE9C0E0ECC0E080
:20BF6000EDC0E0EEC0E0EFC0E01200BD40EFF8D0E0FFD0E0FED0E0FDD0E0FCD0F0E8604D16
:20BF8000B461004007B47B005002C2E524D0503DFA24F6500724F95034240AFAEAB5F000D9
:20BFA000502BCFA9F0A42FFF92D5E9C5F0CEA4A2D53EFE92D5E9C5F0CDA4A2D53DFD92D514
:20BFC000E9C5F0CCA4A2D53CFCC21E808DE8C0E0201D30201E09052C301B041200B6101211
:20BFE00000BCEF1200BCA3052A20190C201A0FEE8FF01200B4CA800B1200B6888005EF120A
:20C0000000B370D0E01200BD1C0200BDA2201D131200BCEF1200BCA3052AE52D852EF0128D
:20C0200000B4CA80E41200B7F1BE8453BECD58BDE64CBDE242BDBC48BED14FBED544BE17D1
:20C0400043BEC949BED555BEAA46BEAA45BEAA47BDEA2AC00D4E0000BDEE474554200069DB
:20C060006E6465782E68746D00706F73745F75726C3D002E006367695F6C6F676F7574008B
:20C08000636F6E6669672E62696E006367695F62616B5F64617461006367695F006661763B
:20C0A00069636F6E2E69636F006367695F6C6F67696E004C6F67696E004F6E6C79206F6E2B
:20C0C0006520757365722063616E206C6F67696E006367695F6465766963650077726F6EC9
:20C0E000672070617373776F726400496E76616C69642061636365737320495020616464EB
:20C1000072657373006C6F67696E2074696D656F7574006367695F706F7274006367695F39
:20C1200064656C766C616E006367695F766C616E006367695F667764006367695F64656C3C
:20C14000667764006367695F7472756E6B006367695F6D6972726F72006367695F6A756DCD
:20C16000626F5F656E61626C6564006367695F73746F726D6374726C006367695F73797357
:20C18000006367695F737470006367695F70617373006367695F716F73006367695F717015
:20C1A00062617365006367695F713170006367695F71746F73006367695F7164736370003A
:20C1C0006367695F736E6D70006367695F61636C006367695F64656C61636C006367695FC4
:20C1E0007365747674797065006367695F70766964006367695F7365747669640063676922
:20C200005F766964006367695F64656C766964006367695F7265736574006367695F736553
:20C2200074627074797065006367695F636C7273746174006367695F7374617469737400C9
:20C240006367695F616464766C616E006367695F736574766C616E006367695F61646466C2
:20C260007764006367695F736574667764006367695F7365747669643D25640090007004D9
:20C28000E0F54090007005E0F541854082854183E020E7077E007F00C2D72289428A43544C
:20C2A00007F5451200C477E02402F544500205451200C31E053AE53A7002053BE540254484
:20C2C000F540E541354530E604C2E6242FF5411200C33E90007004E540F090007005E541E7
:20C2E000F0AE45AF44D2D72290007010E020E61EA3EDF0A3E9F0A3EAF0EC5407D2E6900081
:20C300007010F00538E53870020539D2D7227C007D00C2D72290007010E0A2E6B32275F072
:20C3200001800375F0041200C33E78407F06900070921200C45F90007090E5F0F0229000F2
:20C340007090E0540770F7221200C3AB90007008742FF0900070107508101200C396E49082
:20C36000007004F090007006F0742F90007005F090007007F0751D10751C10751E00751F6A
:20C380002F75832F758200E4F0753800753900753A00753B0022E4A808F0A3D8FC22120071
:20C3A000C4551200C3481200C3E9229000C3DF75080A797078601200C4667518C07519A82E
:20C3C000751A00751B647510C07511A87512007513017514FF7515FF7516FF75170022000E
:20C3E0000B78667788C0A800649000706AE0440CF0229000706AE054F3F0229000706AE0F0
:20C400004401F0229000706AE054FEF0229000706AE04402F0229000706AE054FDF0229038
:20C4200000706AE04440F0229000706AE054BFF02290007000E04410F02290007000E054C3
:20C44000EFF02290007000E04420F02290007000E05420F0229000700AF00000000022E61D
:20C46000F008A3DFFA2289A0E493A3F208B800030989A0D508F222A3E58330E60375832FC0
:20C48000220A0A776562207365727665722072756E6E696E672E2E2E205B25645D0A000A51
:20C4A00053797374656D20696E6974206661696C7572652E0A00496E69742066696E697316
:20C4C0006865642E0A005B54494D4525643A2044256420204825643A4D25643A5325645D25
:20C4E0000A002E005B456E74727925643D256C785D202000537461727421210A00476574B1
:20C5000054696D65203A202564202025643A25643A25640A0053746F7021210A00436F7517
:20C520006E742054696D65203A202564202025643A25643A25640A00436F756E7420416C38
:20C540006C2054696D65203A202564202025643A25643A25640A0020456E747279204E754F
:20C560006D62657220202020756C76616C75650A002D2D2D2D2D2D2D2D2D2D2D2D2D2D2DEA
:20C580002D2D2D2D2D2D2D2D2D2D2D2D2D0A002020202025642020202020202025382E389C
:20C5A0007825342E3478200A0053746172742074696D65203D20257520286D696E69207429
:20C5C00069636B73290A0069203D2025640A0053746F702074696D65203D20257520286DC4
:20C5E000696E69207469636B73290A00546F74616C207365617263682074696D65203D20A4
:20C60000257520286D696E69207469636B73290A00546F74616C2073656172636820746983
:20C620006D65203D202575207365636F6E64730A0053797374656D20626F6F747570004C6E
:20C640006F67696E20696E76616C69642070617373776F72642066726F6D2025642E25645F
:20C660002E25642E25640052656D6F74652049503A2025642E25642E25642E256400506F60
:20C68000727420256420666962657220696E73657274656400506F727420256420666962C6
:20C6A00065722072656D6F76656400506F7274202564206669626572206C696E6B20757048
:20C6C00000506F7274202564206669626572206C696E6B20646F776E00506F7274202564F0
:20C6E0002066696265722072656365697665206572726F7200506F72742025642066696226
:20C700006572207472616E736D6974206572726F7200506F727420256420636F707065726F
:20C720002072656365697665206572726F7200506F727420256420636F70706572207472AF
:20C74000616E736D6974206572726F7200506F727420256420636F70706572206C696E6B3E
:20C7600020757000506F727420256420636F70706572206C696E6B20646F776E0075C7AA31
:20C7800075C755759D0275C7AA75C75575C600787FE4F6D8FD755004755100758151D20DE7
:20C7A0000200C7CE02030007E493A3F85407240CC8C333C4540F4420C8834004F456800196
:20C7C00046F6DFE4800C010204081020408090009C47E47E019360CCA3FF543F30E5095493
:20C7E0001FFEE493A360010ECF54E0B4E02AE493FBA3E493FAA3E493F9A3E493C083C0829A
:20C80000C0931200B370D093D082D083A309E970010ADFE6DEE480BA54C025E0602B40884B
:20C82000E493A3FAE493A3F8E493A3C8C582C8CAC583CA759308F0759300A3C8C582C8CAB9
:20C84000C583CADFE3DEE18089E493A3F8E493A34003F68001F208DFF40200C7D22A2A2A70
:20C860002A2A2A2A2A2A2A2A2A2A2A2A2A2A2A2A2A2A2A2A2A2A2A2A2A2A2A2A2A2A2A2A78
:20C880002A2A2A2A0A20507265737465726120636F6D6D616E646572207368656C6C2073DF
:20C8A0006572766572207265616479200A2A2A2A2A2A2A2A2A2A2A2A2A2A2A2A2A2A2A2AD7
:20C8C0002A2A2A2A2A2A2A2A2A2A2A2A2A2A2A2A2A2A2A2A0A0A002D3E000A0A0068656C44
:20C8E0006C6F3F3F3F0068696869232323006D616320777269746500676F206C6F6164651E
:20C900007200636C6F7365746D006D61632072656164002573006D6163006D6F64656C20C7
:20C9200072656164006D6F64656C3A00667776657220726561640066777665723A007262F2
:20C9400063686B004661696C004F6B009008A8FDE0FFA3E0FEA3E0CF90088B07F0A3EEF0E1
:20C96000A3EFF09008A900E0CBF0A3E0CAF0A3E0C9F07F2290088B0AAD82AC831200B31FD0
:20C980008D828C83F0A309E970010ADFEB9008A900E0FBA3E0FAA3E0F902008C337365748D
:20C9A00020766964783D25640A00736574206669656C642066616C6564200A006D63566987
:20C9C000647847726F7570536861646F775B695D2E76696478203D25642C2025640A0044F5
:20C9E000656661756C740070617373776F726400004D444C3A4753373136542D56312E318D
:20CA00002E38202020202020202020202020202020202020202020202000EFB40A08740D9A
:20CA20001200CA26740A309811A899B8130CC2983098FDA899C298B811F63099FDC299F5F6
:20CA4000992240404025782121210023232300253032780025303478002530386C7800255C
:20CA60006C6400256C78000D0A2047616C746973206167656E742072756E6E696E672E2E96
:20CA80002E0D0A00E94A4B7001221200B31FFF6D700122EF7004FBFAF92209E970EC0A8012
:20CAA000E946455F2564004762455F256400566C616E31007075626C69630062797465331C
:20CAC000203D256C78200A0076696478202E2E2E3D25640A00256C640077726974652D6FD5
:20CAE0006E6C790044656661756C740010200D1200CB2DBF0D027F0A0200CA1A9008AC2135
:20CB0000E0FF22E4FFFE1200B31F600C0FEF70010E09E970F10A80EE2225732025730047E2
:20CB200053373136540056312E312E38003098FDAF99C2987E00229008AC21EFF0D2202205
:20CB4000257800256C7800082008000A00740074009000FFFD1200B891EBF0A3EAF0A3E942
:20CB6000F09000FFCD1200B8919000003F1200B8B8E0FEA3E0FF9000003F1200B8B8EEF02E
:20CB8000A3EFF0900000391200B8B8E0FBA3E0FAA3E0F91200B450FDACF0C3940DEC648011
:20CBA0009480500301E3F4900000361200B8B8E0FBA3E0FAA3E0F9C003C002C001C3ED9490
:20CBC00001FDEC9400FC900000331200B8B8E0F9A3E0FAA3E090089F19C9F0A3EAF0A3E9AB
:20CBE000F0900000331200B8B8E0FBA3E0FAA3E02434F9E43AFA1200B450C39401FEE5F07B
:20CC0000940090089F1CF0A3CEF0D001D002D0031206054BEF4E600301E3F47C007D0290FB
:20CC20000000391200B8B8E0FBA3E0FAA3E0F91200B45025E0FFE5F033FE9000003612006D
:20CC4000B8B8E0FBA3E0FAA3E02FF9EA3EFAC3E99DF9EA9CFA1200B450FFAEF085508385ED
:20CC60005182759308EEF0A3EFF0855083855182759308E0FEA3E0FFC39401EE6480948013
:20CC8000400BD3EF9401EE64809480400301E3F485508385518275930874FFF5F01200B413
:20CCA00024900000331200B8B8E0FBA3E0FAA3E02437F9E43AFA1200B450FFAEF0E5F060DC
:20CCC0000301E3F4EF24FD700301D30C14700301D8DB14700301E0662403600301E3F48526
:20CCE0005083855182759308E0FEA3E0FF90087E5975F00E1200B774EE75F00EA42583F5D8
:20CD000083759308E0FD900000321200B8B8EDF090087E5975F00EEF1200B774EE75F00E13
:20CD2000A42583F583759308ED54FEF09000003C1200B8B8E0FBA3E0FAA3E0F91200B66B9B
:20CD40001200B848CD6000000000CD8B00000001CDB600000002CDE2000000030000CE2B0B
:20CD6000855083855182759308E0FEA3E0FF90087E4C75F00E1200B774EE75F00EA42583D4
:20CD8000F583759308E4F0A301CE0C855083855182759308E0FEA3E0FF90087E4C75F00EC4
:20CDA0001200B774EE75F00EA42583F583759308E4F0A3048056855083855182759308E010
:20CDC000FEA3E0FF90087E4C75F00E1200B774EE75F00EA42583F583759308E4F0A374029F
:20CDE000802A855083855182759308E0FEA3E0FF90087E4C75F00E1200B774EE75F00EA452
:20CE00002583F583759308E4F0A37403F090087E5975F00EEF1200B774EE75F00EA4258349
:20CE2000F583759308E04401F0803A900000321200B8B8E020E00301E3EE855083855182F2
:20CE4000759308E0FEA3E090087E5975F00E1200B774EE75F00EA42583F583759308E044E9
:20CE600001F001E3EE855083855182759308E0FEA3E090087E5775F00E1200B774EE75F05E
:20CE80000EA42583F583759308E0FEA3E064014E600301E3FAFE7F04FD7B099000000A12AD
:20CEA00000B8B8A982AA831200BBFD7E007F047D007B099000000E1200B8B8A982AA831254
:20CEC00000BBFD7B099000000A1200B8B8A982AA83C001855083855182759308E0FEA3E0C0
:20CEE000FF7C007D0E1200B38474532FF9747E3EA801FC7D09D0017E007F041200BB73EF98
:20CF00006048855083855182759308E0FEA3E0FF7C007D0E1200B38474532FF9747E3EFAE0
:20CF20007B09C003C002C0017B099000000E1200B8B8A982AA83A801AC02AD03D001D00281
:20CF4000D0037E007F041200B2A17B099000000A1200B8B8A982AA83C0018550838551822F
:20CF6000759308E0FEA3E0FF7C007D0E1200B384744F2FF9747E3EA801FC7D09D0017E005C
:20CF80007F041200BB73EF6048855083855182759308E0FEA3E0FF7C007D0E1200B3847453
:20CFA0004F2FF9747E3EFA7B09C003C002C0017B099000000E1200B8B8A982AA83A801ACB5
:20CFC00002AD03D001D002D0037E007F041200B2A1855083855182759308E0FEA3E090080A
:20CFE0007E5975F00E1200B774EE75F00EA42583F583759308E054FEF09000003C1200B8BD
:20D00000B8E0FBA3E0FAA3E0F91200B66B1200B848D02D00000000D03400000001D1070065
:20D02000000002D1DA000000030000D2D51206B45E01D2AA855083855182759308E0FEA3B1
:20D04000E090087E4E75F00E1200B774EE75F00EA42583F583759308E0FF131313541FFE1E
:20D060009000000E1200B8B8E5822EF582E43583F583759308E0FEEF5407FF7401A807080D
:20D080008002C333D8FC5E600301E3EE7B099000000A1200B8B8A982AA83C001855083851B
:20D0A0005182759308E0FEA3E0FF7C007D0E1200B38474532FF9747E3EA801FC7D09D001C2
:20D0C0007E007F041200B2A17B099000000E1200B8B8A982AA83C001855083855182759375
:20D0E00008E0FEA3E0FF7C007D0E1200B384744F2FF9747E3EA801FC7D09D0017E007F0460
:20D100001200B2A101D2AA855083855182759308E0FEA3E090087E4E75F00E1200B774EE0A
:20D1200075F00EA42583F583759308E0FF131313541FFE9000000E1200B8B8E5822EF582F3
:20D14000E43583F583759308E0FEEF5407FF7401A807088002C333D8FC5E600301E3EE7BFE
:20D16000099000000E1200B8B8A982AA83C001855083855182759308E0FEA3E0FF7C007D54
:20D180000E1200B38474532FF9747E3EA801FC7D09D0017E007F041200B2A17B09900000A3
:20D1A0000A1200B8B8A982AA83C001855083855182759308E0FEA3E0FF7C007D0E1200B3DE
:20D1C00084744F2FF9747E3EA801FC7D09D0017E007F041200B2A101D2AA85508385518221
:20D1E000759308E0FEA3E090087E4E75F00E1200B774EE75F00EA42583F583759308E0FF96
:20D20000131313541FFE9000000E1200B8B8E5822EF582E43583F583759308E0FEEF5407EC
:20D22000FF7401A807088002C333D8FC5E600301E3EE7B099000000E1200B8B8A982AA83E8
:20D24000C001855083855182759308E0FEA3E0FF7C007D0E1200B384744F2FF9747E3EA8DA
:20D2600001FC7D09D0017E007F041200B2A17B099000000E1200B8B8A982AA83C001855062
:20D2800083855182759308E0FEA3E0FF7C007D0E1200B38474532FF9747E3EA801FC7D09A9
:20D2A000D0017E007F041200B2A1855083855182759308E0FEA3E090087E5975F00E120022
:20D2C000B774EE75F00EA42583F583759308E04401F001DFBF900000321200B8B8E030E006
:20D2E00028855083855182759308E0FEA3E090087E5975F00E1200B774EE75F00EA4258319
:20D30000F583759308E04401F001E3EE855083855182759308E0FEA3E0FF90087E5975F0AA
:20D320000E1200B774EE75F00EA42583F583759308E0FD900000321200B8B8EDF090087E59
:20D340005975F00EEF1200B774EE75F00EA42583F583759308ED54FDF0855083855182754D
:20D360009308E0FEA3E090087E4C75F00E1200B774EE75F00EA42583F583759308E0FEA3E9
:20D38000E04E700301D4409000003C1200B8B8E0FBA3E0FAA3E0F91200B66BE47B01FAF92F
:20D3A000F8D31200B634506190087EFFE02401FF90087EFEE03400FE90087ECCE02FFF9036
:20D3C000087ECBE03EFE90087EC2E02FFF90087EC1E03EFE90087F08E02FFF90087F07E0DC
:20D3E0003ECFC39401CF9400FE3395E0FDFC9000003C1200B8B8E0FBA3E0FAA3E0F9120092
:20D40000B6D0D31200B6344037900000321200B8B8E030E128855083855182759308E0FE45
:20D42000A3E090087E5975F00E1200B774EE75F00EA42583F583759308E04402F001E3EE2D
:20D44000855083855182759308E0FEA3E0FF90087E4C75F00E1200B774EE75F00EA42583ED
:20D46000F583759308E0FCA3E0FDEC600301D871ED14603314700301D5AA14700301D6AD89
:20D480002403600301D8711206B46C855083855182759308E0FEA3E090087E5975F00E126B
:20D4A00000B774EE01D8609000003C1200B8B8E0FBA3E0FAA3E0F91200B66BC3EF9401FF7F
:20D4C000EE9400FEED9400FDEC9400FCEF5407FFE404A807088002C333D8FCFFC0071200C6
:20D4E000B66BC3EF9401FFEE9400FEED9400FDEC9400FC78031200B645855083855182759E
:20D500009308E0FCA3E0FD90087E4F75F00E1200B774EC75F00EA42583F583E5822FF582CF
:20D52000E5833EF583759308E0FED0E05E602B900000321200B8B8E030E11C90087E597511
:20D54000F00EED1200B774EC75F00EA42583F583759308E04402F001E3EE9000003C1200AA
:20D56000B8B8E0FBA3E0FAA3E0F91200B66BC3EF9401FF855083855182759308E0FCA3E0CF
:20D58000FD90087E4E75F00E1200B774EC75F00EA42583F583759308EFF090087E5975F094
:20D5A0000EED1200B774EC01D8609000003C1200B8B8E0FBA3E0FAA3E0F91200B66BC3EF07
:20D5C0009401FFEE9400FEED9400FDEC9400FCEF5407FFE404A807088002C333D8FCFFC04A
:20D5E000071200B66BC3EF9401FFEE9400FEED9400FDEC9400FC78031200B64585508385CC
:20D600005182759308E0FCA3E0FD90087E5375F00E1200B774EC75F00EA42583F583E58228
:20D620002FF582E5833EF583759308E0FED0E05E602B900000321200B8B8E030E11C9008B6
:20D640007E5975F00EED1200B774EC75F00EA42583F583759308E04402F001E3EE900000AB
:20D660003C1200B8B8E0FBA3E0FAA3E0F91200B66BC3EF9401FF855083855182759308E0FF
:20D68000FCA3E0FD90087E4E75F00E1200B774EC75F00EA42583F583759308EFF090087ED2
:20D6A0005975F00EED1200B774EC01D8609000003C1200B8B8E0FBA3E0FAA3E0F91200B665
:20D6C0006BC3EF9401FFEE9400FEED9400FDEC9400FCEF5407FFE404A807088002C333D8E7
:20D6E000FCFFC0071200B66BC3EF9401FFEE9400FEED9400FDEC9400FC78031200B6458568
:20D700005083855182759308E0FCA3E0FD90087E4F75F00E1200B774EC75F00EA42583F5BD
:20D7200083E5822FF582E5833EF583759308E0FED0E05E602B900000321200B8B8E030E17F
:20D740001C90087E5975F00EED1200B774EC75F00EA42583F583759308E04402F001E3EE86
:20D760009000003C1200B8B8E0FBA3E0FAA3E0F91200B66BC3EF9401FFEE9400FEED94000D
:20D78000FDEC9400FCEF5407FFE404A807088002C333D8FCFFC0071200B66BC3EF9401FF9D
:20D7A000EE9400FEED9400FDEC9400FC78031200B645855083855182759308E0FCA3E0FD4B
:20D7C00090087E5375F00E1200B774EC75F00EA42583F583E5822FF582E5833EF5837593DA
:20D7E00008E0FED0E05E602B900000321200B8B8E030E11C90087E5975F00EED1200B7744D
:20D80000EC75F00EA42583F583759308E04402F001E3EE9000003C1200B8B8E0FBA3E0FA47
:20D82000A3E0F91200B66BC3EF9401FF855083855182759308E0FCA3E0FD90087E4E75F00E
:20D840000E1200B774EC75F00EA42583F583759308EFF090087E5975F00EED1200B774EC73
:20D8600075F00EA42583F583759308E04402F08037900000321200B8B8E030E128855083DF
:20D88000855182759308E0FEA3E090087E5975F00E1200B774EE75F00EA42583F583759373
:20D8A00008E04402F001E3EE855083855182759308E0FEA3E090087E5775F00E1200B7743A
:20D8C000EE75F00EA42583F583759308E0FEA3E064014E600301E3FA01DFBF8550838551F1
:20D8E00082759308E0FEA3E0FF90087E5975F00E1200B774EE75F00EA42583F583759308E2
:20D90000E0FD900000321200B8B8EDF090087E5975F00EEF1200B774EE75F00EA42583F559
:20D9200083759308ED54FBF0855083855182759308E0FEA3E0FF90087E4C75F00E1200B76A
:20D9400074EE75F00EA42583F583759308E0FCA3E04C605490087E5975F00EEF1200B774B1
:20D96000EE75F00EA42583F583759308E0FF20E137900000321200B8B8E030E228855083A5
:20D98000855182759308E0FCA3E090087E5975F00E1200B774EC75F00EA42583F583759376
:20D9A00008EF4404F001E3EE7E007F047D007B09900000121200B8B8A982AA831200BBFD1E
:20D9C0009000003F1200B8B8E0FEA3E0FF9000003C1200B8B8E0FBA3E0FAA3E0F9C003C0F1
:20D9E00002C0017B09900000121200B8B8A982AA83A801AC02AD03D001D002D0031200B223
:20DA0000A17B09900000121200B8B8A982AA837D047C001205A5B2EFF47002EEF47037908C
:20DA20000000321200B8B8E030E228855083855182759308E0FEA3E090087E5975F00E1203
:20DA400000B774EE75F00EA42583F583759308E04404F001E3EE7B09900000121200B8B8D4
:20DA6000A982AA83C003C002C0017B099000000E1200B8B8A982AA839008A5B3EBF0A3EAB4
:20DA8000F0A3E9F0D001D002D003120607547E007F047D007B099000000A1200B8B8A982E8
:20DAA000AA831200BBFD855083855182759308E0FEA3E090087E4C75F00E1200B774EE75D9
:20DAC000F00EA42583F583759308E0FEA3E04E60707B099000000A1200B8B8A982AA83C03D
:20DAE00003C002C0017B099000000E1200B8B8A982AA83A801AC02AD03D001D002D0037EA9
:20DB0000007F041200BB73EF7037900000321200B8B8E030E228855083855182759308E0AE
:20DB2000FEA3E090087E5975F00E1200B774EE75F00EA42583F583759308E04404F001E314
:20DB4000EE855083855182759308E0FEA3E090087E4C75F00E1200B774EE75F00EA42583F7
:20DB6000F583759308E0FEA3E0FF64024E6009EF64034E600301DC76855083855182A3A350
:20DB8000759308E4F0A3F0900000041200B8B8E4F0A3F0C390087ED4E09401FF90087ED387
:20DBA000E09400FE855083855182A3A3759308E0FCA3E0FDC39FEE6480F8EC648098506944
:20DBC000EDAE047803CEA2E713CE13D8F8FF9000000E1200B8B8E5822FF582E5833EF583C6
:20DBE000759308E0FF855083855182A3A3759308A3E05407FE7401A806088002C333D8FCDD
:20DC00005F6010900000041200B8B8E475F0011200B424855083855182A3A3759308E4758C
:20DC2000F0011200B42401DB93900000041200B8B8E0FEA3E0D39404EE64809480403790CB
:20DC40000000321200B8B8E030E228855083855182759308E0FEA3E090087E5975F00E12E1
:20DC600000B774EE75F00EA42583F583759308E04404F001E3EE7E007F04C006C0077F004D
:20DC8000C007855083855182759308E0FEA3E0FF7C007D0E1200B384744F2FF9747E3EFA38
:20DCA0007B09D005D007D0061200BBFD7E007F04C006C0077F00C007855083855182759308
:20DCC00008E0FEA3E0FF7C007D0E1200B38474532FF9747E3EFA7B09D005D007D00612005B
:20DCE000BBFD855083855182759308E0FEA3E0FF90087E4C75F00E1200B774EE75F00EA435
:20DD00002583F583759308E0FCA3E0FDEC600301DF58ED14601A14700301DDC714700301C1
:20DD2000DE5E2403600301DF581206B46C01DF2E855083855182759308E0FEA3E090087E68
:20DD40004E75F00E1200B774EE75F00EA42583F583759308E0FF131313541FFE9000000E69
:20DD60001200B8B8E5822EF582E43583F583759308E0FEEF5407FF7401A807088002C33326
:20DD8000D8FC5E600301E3EE7B099000000E1200B8B8A982AA83C0018550838551827593A7
:20DDA00008E0FEA3E0FF7C007D0E1200B384744F2FF9747E3EA801FC7D09D0017E007F0493
:20DDC0001200B2A101DF2E855083855182759308E0FEA3E090087E4E75F00E1200B774EEAD
:20DDE00075F00EA42583F583759308E0FF131313541FFE9000000E1200B8B8E5822EF58227
:20DE0000E43583F583759308E0FEEF5407FF7401A807088002C333D8FC5E600301E3EE7B31
:20DE2000099000000E1200B8B8A982AA83C001855083855182759308E0FEA3E0FF7C007D87
:20DE40000E1200B38474532FF9747E3EA801FC7D09D0017E007F041200B2A101DF2E855007
:20DE600083855182759308E0FEA3E090087E4E75F00E1200B774EE75F00EA42583F58375A8
:20DE80009308E0FF131313541FFE9000000E1200B8B8E5822EF582E43583F583759308E02E
:20DEA000FEEF5407FF7401A807088002C333D8FC5E600301E3EE7B099000000E1200B8B86C
:20DEC000A982AA83C001855083855182759308E0FEA3E0FF7C007D0E1200B384744F2FF9CE
:20DEE000747E3EA801FC7D09D0017E007F041200B2A17B099000000E1200B8B8A982AA8394
:20DF0000C001855083855182759308E0FEA3E0FF7C007D0E1200B38474532FF9747E3EA809
:20DF200001FC7D09D0017E007F041200B2A1855083855182759308E0FEA3E090087E597522
:20DF4000F00E1200B774EE75F00EA42583F583759308E04404F08037900000321200B8B83E
:20DF6000E030E228855083855182759308E0FEA3E090087E5975F00E1200B774EE75F00EE6
:20DF8000A42583F583759308E04404F001E3EE855083855182759308E0FEA3E090087E5735
:20DFA00075F00E1200B774EE75F00EA42583F583759308E0FEA3E064014E600301E3FA85A2
:20DFC0005083855182759308E0FEA3E0FF90087E4E75F00E1200B774EE75F00EA42583F5F0
:20DFE00083759308E0FDC0057C007D0E1200B38474532FF9747E3EFA7B098550838551824F
:20E00000759308A3E0FF900892E77402F0D00512048B5C855083855182759308E0FEA3E004
:20E02000FF90087E4E75F00E1200B774EE75F00EA42583F583759308E0FDC0057C007D0EEF
:20E040001200B384744F2FF9747E3EFA7B09855083855182759308A3E0FF900892E7740116
:20E06000F0D00501E3E49000003C1200B8B8E0FBA3E0FAA3E0F91200B66B90000006120016
:20E08000B8B81200B757900000061200B8B8E0FCA3E0FDA3E0FEA3E0FF1200B848E0BF00C8
:20E0A000000001E1B600000002E1B600000004E1B900000005E245000000060000E1B68543
:20E0C0005083855182759308E0FEA3E0900000161206E09B900000161200B8B8E0FEA3E0E2
:20E0E0004E701B900000211200B8B8E0FEA3E04E7006FE7F0301E3FD1206B45E8012900042
:20E1000000231200B8B8E054076407600301E3EE900000211200B8B8E4F0A304F07B0990CD
:20E120000000161200B8B8A982AA83C001855083855182759308E0FEA3E0FF7C007D0E12F5
:20E1400000B384744C2FF9747E3EA801FC7D09D0017E007F0E1200B2A185508385518275DF
:20E160009308A3E0FF900000181200B8B8E0FD7B099000001D1200B8B8A982AA8390089246
:20E18000E77402F012048B5C855083855182759308A3E0FF900000181200B8B8E0FD7B0968
:20E1A000900000191200B8B8A982AA83900892E77401F001E3E401E3EE85508385518275A7
:20E1C0009308E0FEA3E0900000241206E09BEF4E600301E3EE7E007F0E7D007B09900000EE
:20E1E000241200B8B8A982AA831200BBFD900000261200B8B87480F09000002F1200B8B8FA
:20E20000E4F0A37403F07B09900000241200B8B8A982AA83C001855083855182759308E0AD
:20E22000FEA3E0FF7C007D0E1200B384744C2FF9747E3EA801FC7D09D0017E007F0E1200DD
:20E24000B2A101E3FA855083855182759308E0FEA3E090087E5775F00E1200B774EE75F0FC
:20E260000EA42583F583759308E0FEA3E04E7002802D855083855182759308E0FEA3E0903D
:20E28000087E5775F00E1200B774EE75F00EA42583F583759308E0FEA3E064034E7076FEC2
:20E2A0007F0EFD7B09900000161200B8B8A982AA831200BBFD900000181200B8B87480F0F8
:20E2C000900000211200B8B8E4F0A3F0900000231200B8B8E4F07B09900000161200B8B8EF
:20E2E000A982AA83C001855083855182759308E0FEA3E0FF7C007D0E1200B384744C2FF9AD
:20E30000747E3EA801FC7D09D0017E007F0E1200B2A101E3FA7E007F0E7D007B09900000E7
:20E32000161200B8B8A982AA831200BBFD900000181200B8B87480F0900000211200B8B8E2
:20E34000E4F0A3F0900000231200B8B8E4F07B09900000161200B8B8A982AA83C0018550B3
:20E3600083855182759308E0FEA3E0FF7C007D0E1200B384744C2FF9747E3EA801FC7D09BF
:20E38000D0017E007F0E1200B2A1855083855182759308A3E0FF900000181200B8B8E0FDF3
:20E3A0007B099000001D1200B8B8A982AA83900892E77402F012048B5C85508385518275B9
:20E3C0009308A3E0FF900000181200B8B8E0FD7B09900000191200B8B8A982AA83900892E8
:20E3E000E77401F012048B5C120718DF800C7E007F0380097E007F028003E4FEFF900000BC
:20E40000410200B891EF6402600301E64690084547F0A3F090084544E0FBA3E0FAA3E024C4
:20E4200015F9E43AFA1200B31FB4075390084544A3E0FAA3E02416F9E43AFA74011200B31E
:20E4400054D39405500301FA0C90084544A3E0FAA3E02415F9E43AFAE41200B37090088303
:20E4600040E0FCA3E0FDA3E0FEA3E02401FFE43EFEE43DFDE43CFC900883400200B7579083
:20E48000084544E0FBA3E0FAA3E02415F9E43AFA1200B31FB4052090084544A3E0FAA3E0E8
:20E4A0002416F9E43AFA74011200B354D39405500301FA0C01E63F90084544E0FBA3E0FA1E
:20E4C000A3E02415F9E43AFA1200B31FFF700301FA0C20E40301E5EB90084544A3E0FAA3F9
:20E4E000E02416F9E43AFA74FF1200B354600301FA0C120646E190084544E0FBA3E0FAA3A0
:20E50000E02417F9E43AFA74011200B3356405705990084544E0FBA3E0FAA3E02415F9E41C
:20E520003AFAE41200B37090088340E0FCA3E0FDA3E0FEA3E02401FFE43EFEE43DFDE43C51
:20E54000FC900883401200B757900844377480F0900841D2E0FBA3E0FAA3E0240DF9E43A7F
:20E56000FA74141200B37001F50090084544E0FBA3E0FAA3E02415F9E43AFA1200B31F5470
:20E580000F14700301EFBB24FE603014700301F43924FE700301F43924FE700301F4392429
:20E5A00006600301FA0C900841D2E0FBA3E0FAA3E0240DF9E43AFAE401EFCE9008443774FA
:20E5C00004F090088350E0FCA3E0FDA3E0FEA3E02401FFE43EFEE43DFDE43CFC9008835093
:20E5E0001200B757120718AD01F62690084544E0FBA3E0FAA3E02415F9E43AFA1200B31FD6
:20E60000540F6403600301FA0C90084544A3E0FAA3E02416F9E43AFA74FF1200B35460036B
:20E6200001FA0C90084544A3E0FAA3E02417F9E43AFA74011200B3356405600301FA0C1212
:20E640000646E101E51190087F00E0FBA3E0FAA3E0F990084547E0FEA3E0FFE92FF9EA3EEE
:20E66000FAE41200B370900845447409F0A37444F0A37442F090087F00E0FBA3E0FAA3E073
:20E68000F9900841CCEBF0A3EAF0A3E9F0240EF9E43AFA900841D8EBF0A3EAF0A3E9F0122E
:20E6A0000596A3EF6401600301E7D890087EB5E0700301E7B11207339F9008A84BEFF07524
:20E6C000F005A424EEF582E4343EF583759308E09008A84BF090087F00E0FBA3E0FAA3E0ED
:20E6E000F990084541EBF0A3EAF0A3E9F02411F9E43AFA1200B45045F0600301FA0C90089C
:20E700004541E0FBA3E0FAA3E02413F9E43AFA1200B31F600301FA0C90084541E0FBA3E086
:20E72000FAA3E02414F9E43AFA1200B31F705E90084541A3E0FAA3E0240CF9E43AFA1200F0
:20E74000B450C39403FFE5F09400FEC3EF9423EE9400500301FA0C90084541E0FBA3E0FA3A
:20E76000A3E02415F9E43AFA1200B31FFF64806010EF6481600BEF64016006EF600301FA4F
:20E780000C9008A84BE0FF12057710804B90084541E0FBA3E0FAA3E02414F9E43AFA120046
:20E7A000B31FB480339008A84BE0FF12071BE9802712073C12BF012090087F00E0FBA3E036
:20E7C000FAA3E0F990084541EBF0A3EAF0A3E9F07D347C0012069E3F900841CCE0FBA3E0AC
:20E7E000FAA3E0240CF9E43AFA1200B450FFAEF0BE0807BF06040205495E90087427E0FC55
:20E80000A3E0FDA3E0FEA3E02401FFE43EFEE43DFDE43CFC900874271200B757900841CCFE
:20E82000E0FBA3E0FAA3E0240CF9E43AFA1200B4507004E5F06408602190087437E0FCA3AE
:20E84000E0FDA3E0FEA3E02401FFE43EFEE43DFDE43CFC9008743701E997900841D8E0FB09
:20E86000A3E0FAA3E02402F9E43AFA1200B450FFAEF090084547EEF0A3EFF0D39414EE942D
:20E880000540219008742BE0FCA3E0FDA3E0FEA3E02401FFE43EFEE43DFDE43CFC900874F1
:20E8A0002B01E997900841D8E0FBA3E0FAA3E0F91200B31F644560219008742BE0FCA3E083
:20E8C000FDA3E0FEA3E02401FFE43EFEE43DFDE43CFC9008742B01E997E92406F9E43AFADD
:20E8E0001200B450E5F0543F602190087463E0FCA3E0FDA3E0FEA3E02401FFE43EFEE43DE5
:20E90000FDE43CFC9008746301E9971207375E900841D8E0FBA3E0FAA3E02410F9E43AFA6F
:20E920001200B6D0C31200B6346042900841D8E0FBA3E0FAA3E02410F9E43AFA1200B66BDA
:20E9400074FFFBFAF9F8C31200B63460209008742FE0FCA3E0FDA3E0FEA3E02401FFE43E3E
:20E96000FEE43DFDE43CFC9008742F802A120582D3EFF47002EEF460259008742BE0FCA39C
:20E98000E0FDA3E0FEA3E02401FFE43EFEE43DFDE43CFC9008742B1200B75701F1769008C1
:20E9A00041D8E0FBA3E0FAA3E0240CF9E43AFA1200B66B900841CCE0FBA3E0FAA3E0240645
:20E9C000F9E43AFA120494CB9008743FE0FCA3E0FDA3E0FEA3E02401FFE43EFEE43DFDE4C0
:20E9E0003CFC9008743F1200B757900841D8E0FBA3E0FAA3E02409F9E43AFA1200B31FB412
:20EA000001491200B31FFF90084544E0FBA3E0FAA3E02414F9E43AFAEF1200B37090084187
:20EA2000D8E0FBA3E0FAA3E0240CF9E43AFA1200B66B90084544E0FBA3E0FAA3E02404F992
:20EA4000E43AFA1200B6880206CFDC900841D8E0FBA3E0FAA3E02409F9E43AFA1200B31FED
:20EA60006411600301EB7790089350E0FCA3E0FDA3E0FEA3E02401FFE43EFEE43DFDE43CFE
:20EA8000FC900893501200B757900841D8E0FBA3E0FAA3E02414F9E43AFA900841D5EBF081
:20EAA000A3EAF0A3E9F090087F00E0FBA3E0FAA3E0F91206DE2F900841D8E0FBA3E0FAA3A1
:20EAC000E02409F9E43AFA1200B31FFF90084544E0FBA3E0FAA3E02414F9E43AFAEF1200EF
:20EAE000B370900841D5E0FBA3E0FAA3E02402F9E43AFA1200B450FF90084544E0FBA3E09F
:20EB0000FAA3E0F9E5F08FF01200B4CA900841D5E0FBA3E0FAA3E0F91200B450FF90084527
:20EB200044E0FBA3E0FAA3E02402F9E43AFAE5F08FF01200B4CA900841D8E0FBA3E0FAA3EF
:20EB4000E0240CF9E43AFA1200B66B90084544E0FBA3E0FAA3E02404F9E43AFA1200B688DC
:20EB600090084544E0FBA3E0FAA3E0F91200B450FFAEF0020654D6900841D8E0FBA3E0FAB2
:20EB8000A3E02409F9E43AFA1200B31F64066043E4FFFEFDFC9008743FE0F8A3E0F9A3E0C7
:20EBA000FAA3E0FBD31200B63440259008743FE0FCA3E0FDA3E0FEA3E024FFFFEE34FFFEBD
:20EBC000ED34FFFDEC34FFFC9008743F1200B75701F176900841D8E0FBA3E0FAA3E0241466
:20EBE000F9E43AFA900841D2EBF0A3EAF0A3E9F090088348E0FCA3E0FDA3E0FEA3E024019D
:20EC0000FFE43EFEE43DFDE43CFC900883481200B75712073AE1900841D2E0FBA3E0FAA33E
:20EC2000E02402F9E43AFA1200B4506F7003EE65F0600301F1769008A849E4F0A304F09033
:20EC400008A849E0FEA3E0FFC39405EE9400400301ED1D7C007D331200B38474422FF97468
:20EC6000443EFA7B0990084544EBF0A3EAF0A3E9F02415F9E43AFA1200B31F700301ED0A06
:20EC8000900841D2E0FBA3E0FAA3E02402F9E43AFA1200B450FFAEF090084544E0FBA3E085
:20ECA000FAA3E0F91200B4506F7003EE65F0705AE92402F9E43AFA1200B450FFAEF090086E
:20ECC00041D2E0FBA3E0FAA3E0F91200B450B50739E5F0B5063490084544E0FBA3E0FAA362
:20ECE000E02404F9E43AFA1200B66B900841D8E0FBA3E0FAA3E0240CF9E43AFA1200B6D063
:20ED0000C31200B634700301F0D19008A84AE004F070079008A849E004F001EC3F900841C8
:20ED2000D2E0FBA3E0FAA3E0240DF9E43AFA1200B31F6402600301F1769008A849E4F0A3CF
:20ED400004F09008A849E0FEA3E0FFC39405EE9400502D9008445775F033EF1200B774EE96
:20ED600075F033A42583F583759308E0605E9008A84AE004F070CB9008A849E004F080C251
:20ED80009008A849E4F0A304F09008A849E0FEA3E0FFC39405EE9400502F9008445775F0A1
:20EDA00033EF1200B774EE75F033A42583F583759308E0640760159008A84AE004F070C943
:20EDC0009008A849E004F080C001F1769008A849E0FEA3E0FF7C007D331200B38474422FEB
:20EDE000F974443EFA900845447409F0A3EAF0A3E9F0900841D8E0FBA3E0FAA3E02409F9F1
:20EE0000E43AFA1200B31FFF90084544E0FBA3E0FAA3E02414F9E43AFAEF1200B3709008F6
:20EE20004544E0FBA3E0FAA3E02416F9E43AFA74021200B37090084544E0FBA3E0FAA3E07C
:20EE40002417F9E43AFAE41200B370900841D2E0FBA3E0FAA3E02402F9E43AFA1200B4507A
:20EE6000FF90084544E0FBA3E0FAA3E0F9E5F08FF01200B4CA900841D2E0FBA3E0FAA3E034
:20EE8000F91200B450FF90084544E0FBA3E0FAA3E02402F9E43AFAE5F08FF01200B4CA90BD
:20EEA0000841D8E0FBA3E0FAA3E0240CF9E43AFA1200B66B90084544E0FBA3E0FAA3E024C2
:20EEC00004F9E43AFA1200B68890084544E0FBA3E0FAA3E02415F9E43AFA74111200B370CD
:20EEE00090088338E0FCA3E0FDA3E0FEA3E02401FFE43EFEE43DFDE43CFC9008833812007C
:20EF0000B7579008443EE0FCA3E0FDA3E0FEA3E0FF90084544E0FBA3E0FAA3E0240CF9E461
:20EF20003AFA1200B688EF2401FFE43EFEE43DFDE43CFC90084544E0FBA3E0FAA3E02410B0
:20EF4000F9E43AFA1200B688900841D2E0FBA3E0FAA3E02404F9E43AFA1200B66BEF24014A
:20EF6000FFE43EFEE43DFDE43CFC90084544E0FBA3E0FAA3E02408F9E43AFA1200B688901F
:20EF8000084544E0FBA3E0FAA3E0242AF9E43AFAC003C002C00190084544A3E0FAA3E0241B
:20EFA00028F9E43AFA9008A7C2EBF0A3EAF0A3E9F0D001D002D00312070063900841D2E0C6
:20EFC000FBA3E0FAA3E0240DF9E43AFA74101200B370900841D2E0FBA3E0FAA3E0240DF98B
:20EFE000E43AFA1200B31F44021200B370900841D2E0FBA3E0FAA3E02414F9E43AFA900833
:20F00000A84CEBF0A3EAF0A3E9F074021200B3709008A84CE0FBA3E0FAA3E02401F9E43ADA
:20F02000FA74041200B3709008A84CE0FBA3E0FAA3E02402F9E43AFA74041200B370900846
:20F04000A84CE0FBA3E0FAA3E02403F9E43AFA74B01200B3709008A84CE0FBA3E0FAA3E0E9
:20F060002404F9E43AFA74011200B3709008A84CE0FBA3E0FAA3E02405F9E43AFA74011285
:20F0800000B3709008A84CE0FBA3E0FAA3E02406F9E43AFA74041200B3709008A84CE0FB97
:20F0A000A3E0FAA3E02407F9E43AFA74021200B37090084547E4F0A37430F0900841D2E0AF
:20F0C000FBA3E0FAA3E0240CF9E43AFA747001F8D5E490084437F0900841D2E0FBA3E0FA58
:20F0E000A3E0240DF9E43AFA1200B31F30E26F90084544E0FBA3E0FAA3E02415F9E43AFAA0
:20F100001200B31FB401229008833CE0FCA3E0FDA3E0FEA3E02401FFE43EFEE43DFDE43CFB
:20F12000FC9008833C1200B757E41200B37090088340E0FCA3E0FDA3E0FEA3E02401FFE480
:20F140003EFEE43DFDE43CFC900883401200B757900844377420F0120718AD01F797900822
:20F1600041D2E0FBA3E0FAA3E0240DF9E43AFA1200B31F20E40301F797900841D2E0FBA3BC
:20F18000E0FAA3E0240CF9E43AFA1200B31FC4540F25E025E0FF7E009008A849EEF0A3EF46
:20F1A000F02414FFEE33FEC390084548E09FFF90084547E09EFEF0A3EFF0D39400EE9400A8
:20F1C000403490084544E0FBA3E0FAA3E02408F9E43AFA1200B66B900841D2E0FBA3E0FA4C
:20F1E000A3E02404F9E43AFA1200B6D0C31200B634600301F8A190084544E0FBA3E0FAA3E3
:20F20000E02410F9E43AFA1200B66B900841D2E0FBA3E0FAA3E02408F9E43AFA1200B6D03B
:20F22000C31200B634706690084544E0FBA3E0FAA3E02410F9E43AFA1200B66B90084544A4
:20F24000A3E0FAA3E0240CF9E43AFA1200B68890084544E0FBA3E0FAA3E02415F9E43AFAD7
:20F260001200B31FFF30E425900844377401F0EF54EF1200B37090084544E0FBA3E0FAA377
:20F28000E02416F9E43AFA74021200B37090084544E0FBA3E0FAA3E02415F9E43AFA120040
:20F2A000B31F540F14B40800400301F89D9000F2BC75F004A4C58325F0C583730200F2DC3D
:20F2C0000200F2F80200F37B0200F6B20200F79A0200F8680200F8A10200F66C9008443721
:20F2E000E030E01174031200B370900844377440F0120718AD01F79790084437E030E078C2
:20F30000900841D2E0FBA3E0FAA3E0240DF9E43AFA1200B31F6412705F90084544E0FBA35D
:20F32000E0FAA3E02415F9E43AFA74031200B370900841D2E0FBA3E0FAA3E02404F9E43AB5
:20F34000FA1200B66B90084544E0FBA3E0FAA3E02408F9E43AFA1200B6881200B66BEF24B1
:20F3600001FFE43EFEE43DFDE43CFC1200B6887442120718A001F4A901F79790088344E0F0
:20F38000FCA3E0FDA3E0FEA3E02401FFE43EFEE43DFDE43CFC900883441200B75790084117
:20F3A000D2E0FBA3E0FAA3E0240DF9E43AFA1200B31F20E00301F43C90084548E02401FF1D
:20F3C00090084547E03400FEE4FCFD90084544E0FBA3E0FAA3E02408F9E43AFA1200B68891
:20F3E0007410120718A090084544E0FBA3E0FAA3E02410F9E43AFA1200B66BEF2401FFE44D
:20F400003EFEE43DFDE43CFC1200B68890084544E0FBA3E0FAA3E02415F9E43AFA74181242
:20F4200000B37090084544E0FBA3E0FAA3E02417F9E43AFAE41200B37001F580D390084522
:20F4400048E0940090084547E09400404590084437E04402F090084544E0FBA3E0FAA3E0AE
:20F460002408F9E43AFAC003C002C0011200B6D090084547E0FEA3E0FFE4FCFDEB2FFFEA0D
:20F480003EFEED39FDEC38FCD001D002D0031200B68890084437E05403700301F6691207F1
:20F4A00018ADEF4E700301F8A190084437E030E57490084544E0FBA3E0FAA3E02415F9E4AF
:20F4C0003AFAE41200B370900841D2E0FBA3E0FAA3E0240DF9E43AFA74141200B3709008C2
:20F4E0008340E0FCA3E0FDA3E0FEA3E02401FFE43EFEE43DFDE43CFC900883401200B757F0
:20F5000090088358E0FCA3E0FDA3E0FEA3E02401FFE43EFEE43DFDE43CFC90088358120015
:20F52000B75701F8B890084437E030E46990084544E0FBA3E0FAA3E02410F9E43AFA120049
:20F54000B66BEF2401FFE43EFEE43DFDE43CFC1200B68890084544E0FBA3E0FAA3E0241598
:20F56000F9E43AFA74141200B37090084544E0FBA3E0FAA3E02417F9E43AFAE41200B3705C
:20F58000900841D2E0FBA3E0FAA3E0240DF9E43AFA741101F8B4D390084548E0940090086D
:20F5A0004547E09400407790084544E0FBA3E0FAA3E02415F9E43AFA1200B31F20E45F12F5
:20F5C00000B31F44101200B37090084544E0FBA3E0FAA3E02417F9E43AFAE41200B37090DF
:20F5E000084544E0FBA3E0FAA3E02410F9E43AFAC003C002C0011200B6D090084547E0FE7A
:20F60000A3E0FFE4FCFDEB2FFFEA3EFEED39FDEC38FCD001D002D0031200B6888008E49047
:20F62000084547F0A3F0D390084548E0940090084547E09400500890084437E030E12A9099
:20F64000084548E02428F090084547E03400F0900841D2E0FBA3E0FAA3E0240DF9E43AFA09
:20F6600074181200B37001F8C201F79790084437E020E00301F89D90084544E0FBA3E0FA7A
:20F68000A3E02415F9E43AFAE41200B37090088340E0FCA3E0FDA3E0FEA3E02401FFE43E83
:20F6A000FEE43DFDE43CFC900883401200B75701F89DD390084548E0940090084547E094FD
:20F6C00000403D90084544E0FBA3E0FAA3E02408F9E43AFAC003C002C0011200B6D09008FE
:20F6E0004547E0FEA3E0FFE4FCFDEB2FFFEA3EFEED39FDEC38FCD001D002D0031200B688F9
:20F70000900841D2E0FBA3E0FAA3E0240DF9E43AFA1200B31F30E04990084437E090084514
:20F720004430E027E0FBA3E0FAA3E02415F9E43AFA74071200B37090084544E0FBA3E0FA00
:20F74000A3E02416F9E43AFAE4800FE0FBA3E0FAA3E02415F9E43AFA74161200B37001F88B
:20F760002D90084437E030E01A90084544E0FBA3E0FAA3E02415F9E43AFA74051200B3704B
:20F7800001F89DD390084548E0940090084547E09400400301F8A101F89DD390084548E084
:20F7A000940090084547E09400403D90084544E0FBA3E0FAA3E02408F9E43AFAC003C002E2
:20F7C000C0011200B6D090084547E0FEA3E0FFE4FCFDEB2FFFEA3EFEED39FDEC38FCD0011C
:20F7E000D002D0031200B688900841D2E0FBA3E0FAA3E0240DF9E43AFA1200B31F30E05503
:20F8000090084544E0FBA3E0FAA3E02415F9E43AFA74071200B37090084544E0FBA3E0FA79
:20F82000A3E02416F9E43AFAE41200B37090084544E0FBA3E0FAA3E02408F9E43AFA120096
:20F84000B66BEF2401FFE43EFEE43DFDE43CFC1200B688804CD390084548E09400900845B5
:20F8600047E09400503B803590084437E030E02D90084544E0FBA3E0FAA3E02415F9E43A11
:20F88000FA74071200B37090084544E0FBA3E0FAA3E02416F9E43AFAE41200B37002073D18
:20F8A000B0900841D2E0FBA3E0FAA3E0240DF9E43AFA74101200B37090084547E4F0A37408
:20F8C00028F0900841D2E0FBA3E0FAA3E0240CF9E43AFA74501200B37090084544E0FBA3B1
:20F8E000E0FAA3E02408F9E43AFA1200B66B900841D2E0FBA3E0FAA3E02408F9E43AFA1266
:20F9000000B68890084544E0FBA3E0FAA3E0240CF9E43AFA1200B66B900841D2E0FBA3E030
:20F92000FAA3E02404F9E43AFA1200B68890084544E0FBA3E0FAA3E0F91200B450FF90081F
:20F9400041D2E0FBA3E0FAA3E0F9E5F08FF01200B4CA90084544E0FBA3E0FAA3E02402F9C1
:20F96000E43AFA1200B450FF900841D2E0FBA3E0FAA3E02402F9E43AFAE5F08FF01200B483
:20F98000CA900841D2E0FBA3E0FAA3E0240EF9E43AFA740475F0B01200B4CA9008834CE070
:20F9A000FCA3E0FDA3E0FEA3E02401FFE43EFEE43DFDE43CFC9008834C1200B757900883A7
:20F9C0004CE0FCA3E0FDA3E0FEA3E0FFA3E0F8A3E0F9A3E0FAA3E0FBC3EF9BFFEE9AFEEDCB
:20F9E00099FDEC98FC9008834C1200B7577F027E001202EE6F90084544E0FBA3E0FAA3E0FE
:20FA00002416F9E43AFA74021200B37022900899B4EFF0A3EDF0A3EBF05D900899B5F09049
:20FA20000899B7E0FFA3E0FEEF5E900899B7F0900899BBE0FEA3E0FF900899B9E05EF0A3E2
:20FA4000E05FF09008DD961200B6C0900899BD1200B757E4FFFEFDFC900899C11200B757EA
:20FA6000900899BDE0FCA3E0FDA3E0FEA3E0FF900895A31200B757E4900895A7F0A304F00A
:20FA8000900899C1E0FCA3E0FDA3E0FEA3E0FF900895A91200B757900899B4E0FF12057ACA
:20FAA0000BEF60037F17229008DD9A1200B6C0900899BD1200B757900899BBE0FEA3E0FF40
:20FAC000E4FCFD900899C11200B757900899C1E0FCA3E0FDA3E0FEA3E0FF780C1200B65842
:20FAE000900899C11200B757900899C1E0F8A3E0F9A3E0FAA3E0FB900899B9E0FEA3E0FF69
:20FB0000EB4FFFEA4EFEE9FDE8FC900899C11200B757900899BDE0FCA3E0FDA3E0FEA3E04C
:20FB2000FF900895A31200B757900895A77408F0A37418F0900899C1E0FCA3E0FDA3E0FEA8
:20FB4000A3E0FF900895A91200B757900899B4E0FF12057A0BEF60037F17229008DD9E129E
:20FB600000B6C0900899BD1200B757900899B8E05401FFE4FCFDFE900899C11200B7579067
:20FB80000899C1E0FCA3E0FDA3E0FEA3E0FF78011200B658900899C11200B757900899C107
:20FBA000E0F8A3E0F9A3E0FAA3E0FB900899B7E05401FFEB4FFFEAFEE9FDE8FC900899C1FD
:20FBC0001200B757900899C1E0FCA3E0FDA3E0FEA3E0FF78011200B658900899C11200B760
:20FBE00057900899C1E0F8A3E0F9A3E0FAA3E0FB900899B6E0541FFFEB4FFFEAFEE9FDE845
:20FC0000FC900899C11200B757900899C1E0FCA3E0FDA3E0FEA3E0FF78051200B658900850
:20FC200099C11200B757900899C1E0F8A3E0F9A3E0FAA3E0FB900899B5E0541FFFEB4FFF98
:20FC4000EAFEE9FDE8FC900899C11200B757900899BDE0FCA3E0FDA3E0FEA3E0FF90089566
:20FC6000A31200B757E4900895A7F0A3740CF0900899C1E0FCA3E0FDA3E0FEA3E0FF90081D
:20FC800095A91200B757900899B4E0FF12057A0BEF60037F17229008DD961200B6C0900871
:20FCA00099BD1200B757E47F05FEFDFC900899C11200B757900899BDE0FCA3E0FDA3E0FE92
:20FCC000A3E0FF900895A31200B757900895A77402F0A304F0900899C1E0FCA3E0FDA3E010
:20FCE000FEA3E0FF900895A91200B757900899B4E0FF12057A0BEF60037F1722E47F03FEC0
:20FD0000FDFC900899C11200B757900899BDE0FCA3E0FDA3E0FEA3E0FF900895A31200B7F2
:20FD200057E4900895A7F0A37402F0900899C1E0FCA3E0FDA3E0FEA3E0FF900895A9120082
:20FD4000B757900899B4E0FF12057A0BEF60037F1722E47F18FEFD7C06900899BD1200B77C
:20FD600057900899BDE0FCA3E0FDA3E0FEA3E0FF900897921200B757900897967404F0A32E
:20FD80007401F0A37409F0A37499F0A374C1F0900899B4E0FF12063ECEEF60037F17229004
:20FDA0000899C1E0FCA3E0FDA3E0FEA3E0FFEC4D4E4F60AD9008DD961200B6C0900899BD1E
:20FDC0001200B757E47F03FEFDFC900899C11200B757900899BDE0FCA3E0FDA3E0FEA3E046
:20FDE000FF900895A31200B757E4900895A7F0A37402F0900899C1E0FCA3E0FDA3E0FEA3F1
:20FE0000E0FF900895A91200B757900899B4E0FF12057A0BEF60037F1722E47F18FEFD7CB1
:20FE200006900899BD1200B757900899BDE0FCA3E0FDA3E0FEA3E0FF900897921200B75780
:20FE4000900897967404F0A37401F0A37409F0A37499F0A374C1F0900899B4E0FF12063EDB
:20FE6000CEEF60037F1722900899C1E0FCA3E0FDA3E0FEA3E0FFEC4D4E4F60AD9008DD966B
:20FE80001200B6C0900899BD1200B757E4FFFEFDFC900899C11200B757900899BDE0FCA373
:20FEA000E0FDA3E0FEA3E0FF900895A31200B757E4900895A7F0A304F0900899C1E0FCA3C2
:20FEC000E0FDA3E0FEA3E0FF900895A91200B757900899B4E0FF12057A0BEF60037F1722E2
:20FEE0009008DD9E1200B6C0900899BD1200B757900899BDE0FCA3E0FDA3E0FEA3E0FF907C
:20FF00000895A31200B757E4900895A7F0A3740CF0900899C1E0FCA3E0FDA3E0FEA3E0FF75
:20FF2000900895A91200B757900899B4E0FF12057A0BEF60037F17229008DD9A1200B6C0CA
:20FF4000900899BD1200B757900899BDE0FCA3E0FDA3E0FEA3E0FF900895A31200B75790C6
:20FF60000895A77408F0A37418F0900899C1E0FCA3E0FDA3E0FEA3E0FF900895A91200B7C2
:20FF800057900899B4E0FF12057A0BEF60037F1722E47F01FEFDFC900899C11200B75790A3
:20FFA00008DD961200B6C0900899BD1200B757900899BDE0FCA3E0FDA3E0FEA3E0FF90084B
:20FFC00095A31200B757E4900895A7F0A37405F0900899C1E0FCA3E0FDA3E0FEA3E0FF9034
:20FFE0000895A91200B757900899B4E0FF12057A0BEF7F0060027F1722E4FFFE0207314256
:020000040001F9
:20000000E49008ABF3F0229000FFFD1200B891EBF0A3EAF0A3E9F09000FFBB1200B8911242
:20002000073B69EF64014E7006FE7F022115639000004B1200B8B8E0FBA3E0FAA3E0F912A2
:2000400000B450FDACF0C3940DEC64809480500321155A900000481200B8B8E0FBA3E0FA26
:20006000A3E0F9C003C002C001C3ED9401FDEC9400FC900000451200B8B8E0F9A3E0FAA3B0
:20008000E090089F19C9F0A3EAF0A3E9F0900000451200B8B8E0FBA3E0FAA3E02434F9E417
:2000A0003AFA1200B450C39401FEE5F0940090089F1CF0A3CEF0D001D002D0031206054BB5
:2000C000EF4E600321155A7C007D029000004B1200B8B8E0FBA3E0FAA3E0F91200B4502589
:2000E000E0FFE5F033FE900000481200B8B8E0FBA3E0FAA3E02FF9EA3EFAC3E99DF9EA9CD4
:20010000FA1200B450FFAEF0855083855182759308EEF0A3EFF0855083855182759308E072
:20012000FEA3E0FFC39401EE94004009D3EF94FEEE940F400321155A7E007F047D007B0962
:200140009000001E1200B8B8A982AA831200BBFD900000451200B8B8E0FBA3E0FAA3E024F7
:2001600037F9E43AFA1200B450FFAEF0E5F07013EF24FD60111470032107D9147003210D6E
:20018000D9240321155A900000041200B8B8E0FEA3E0FF900848D575F00D1200B774EE7592
:2001A000F00DA42583F583759308E0FD900000441200B8B8EDF0900848D575F00DEF120036
:2001C000B774EE75F00DA42583F583759308ED54FDF0900000511200B8B8E0FEA3E0D39467
:2001E00004EE648094804039900000441200B8B8E020E103211554900000041200B8B8E0E2
:20020000FEA3E0900848D575F00D1200B774EE75F00DA42583F583759308E04402F0211579
:20022000547E007F047D007B099000001A1200B8B8A982AA831200BBFD900000511200B86F
:20024000B8E0FEA3E0FF9000004E1200B8B8E0FBA3E0FAA3E0F9C003C002C0017B099000F8
:20026000001A1200B8B8A982AA83A801AC02AD03D001D002D0031200B2A17B099000001A7A
:200280001200B8B8A982AA837D047C001205A5B2EFF47002EEF47036900000441200B8B8E6
:2002A000E030E127900000041200B8B8E0FEA3E0900848D575F00D1200B774EE75F00DA447
:2002C0002583F583759308E04402F0211554855083855182759308E0FEA3E0FF7B0990001A
:2002E00000041200B8B8A982AA83C003C002C0017B09900000371200B8B8A982AA8390081D
:20030000A5BDEBF0A3EAF0A3E9F0D001D002D0031206D0EAEF4E7036900000441200B8B826
:20032000E030E127900000041200B8B8E0FEA3E0900848D575F00D1200B774EE75F00DA4C6
:200340002583F583759308E04402F02115547B099000001A1200B8B8A982AA83C003C00240
:20036000C0017B09900000261200B8B8A982AA839008A5B3EBF0A3EAF0A3E9F0D001D00241
:20038000D00312060754855083855182A3A3759308E4F0A3F0C390087ED4E09401FF9008F1
:2003A0007ED3E09400FE855083855182A3A3759308E0FCA3E0FDC39FEE6480F8EC64809884
:2003C00040032104AEEDAE047803CEA2E713CE13D8F8FF900000261200B8B8E5822FF5828E
:2003E000E5833EF583759308E0FF855083855182A3A3759308A3E05407FE7401A806088063
:2004000002C333D8FCFD5F6003210498855083855182A3A3759308E0FEA3E07803CEA2E75B
:2004200013CE13D8F8FF9000003D1200B8B8E5822FF582E5833EF583759308E0FC5D60587E
:20044000855083855182A3A3759308E0FEA3E07803CEA2E713CE13D8F8FF9000003D1200C1
:20046000B8B8E5822FF582E5833EF583C083C082759308855083855182A3A3759308A3E0C3
:200480005407FF7401A807088002C333D8FCF45C759308D082D083F0855083855182A3A39F
:2004A000759308E475F0011200B424210395855083855182A3A3759308E4F0A3F0C3900877
:2004C0007ED4E09401FF90087ED3E09400FE855083855182A3A3759308E0FCA3E0FDC39F37
:2004E000EE6480F8EC64809840032105B0EDAE047803CEA2E713CE13D8F8FF9000003D129E
:2005000000B8B8E5822FF582E5833EF583759308E0FF855083855182A3A3759308A3E05474
:2005200007FE7401A806088002C333D8FCFD5F6069855083855182A3A3759308E0FEA3E0B3
:200540007803CEA2E713CE13D8F8FF900000261200B8B8E5822FF582E5833EF58375930893
:20056000E05D7036900000441200B8B8E030E127900000041200B8B8E0FEA3E0900848D5FE
:2005800075F00D1200B774EE75F00DA42583F583759308E04402F021155485508385518228
:2005A000A3A3759308E475F0011200B4242104BD900000371200B8B8E0FEA3E0FF90000096
:2005C0000E1200B8B8EEF0A3EFF07B09900000261200B8B8A982AA83C003C002C0017B094D
:2005E000900000101200B8B8A982AA83A801AC02AD03D001D002D0037E007F041200B2A19E
:200600007B099000003D1200B8B8A982AA83C003C002C0017B09900000141200B8B8A98294
:20062000AA83A801AC02AD03D001D002D0037E007F041200B2A1855083855182A3A37593AC
:2006400008E4F0A3F0C390087ED4E09401FD90087ED3E09400FC855083855182A3A37593B5
:2006600008E0FEA3E0FFC39DEC6480F8EE64809840032107477B09900000181200B8B8A977
:2006800082AA831207191C9000000E1200B8B8E0FEA3E0FF900000181200B8B8E0540FFC74
:2006A000A3E06F7002EE6C6003210731855083855182A3A3759308E0FEA3E07803CEA2E787
:2006C00013CE13D8F8FF900000101200B8B8E5822FF582E5833EF583759308E0FF855083C3
:2006E000855182A3A3759308A3E05407FE7401A806088002C333D8FC5F703690000044120E
:2007000000B8B8E030E127900000041200B8B8E0FEA3E0900848D575F00D1200B774EE7513
:20072000F00DA42583F583759308E04402F0211554855083855182A3A3759308E475F001F8
:200740001200B4242106457B099000000E1200B8B8A982AA83C003C002C00190000004125B
:2007600000B8B8E0FEA3E0FF7C007D0D1200B38474C92FF974483EA801FC7D09D001D0022D
:20078000D0037E007F0A1200B2A1900000041200B8B8E0FEA3E0FF900848D575F00D12006B
:2007A000B774EE75F00DA42583F583759308E04402F0900848D375F00DEF1200B774EE7510
:2007C000F00DA42583F583759308E0FEA3E064014E6003211560210DAF900000041200B800
:2007E000B8E0FEA3E0FF900848D575F00D1200B774EE75F00DA42583F583759308E0FD90DC
:200800000000441200B8B8EDF0900848D575F00DEF1200B774EE75F00DA42583F5837593B6
:2008200008ED54FBF0900000511200B8B8E0FEA3E0D39404EE648094804036900000441213
:2008400000B8B8E030E227900000041200B8B8E0FEA3E0900848D575F00D1200B774EE75D1
:20086000F00DA42583F583759308E04404F02115547E007F047D007B099000001A1200B88F
:20088000B8A982AA831200BBFD900000511200B8B8E0FEA3E0FF9000004E1200B8B8E0FB80
:2008A000A3E0FAA3E0F9C003C002C0017B099000001A1200B8B8A982AA83A801AC02AD03EA
:2008C000D001D002D0031200B2A17B099000001A1200B8B8A982AA837D047C001205A5B2CA
:2008E000EFF47002EEF47036900000441200B8B8E030E227900000041200B8B8E0FEA3E035
:20090000900848D575F00D1200B774EE75F00DA42583F583759308E04404F02115548550C8
:2009200083855182759308E0FEA3E0FF7B09900000041200B8B8A982AA83C003C002C00134
:200940007B09900000371200B8B8A982AA839008A5BDEBF0A3EAF0A3E9F0D001D002D0032E
:200960001206D0EAEF4E7036900000441200B8B8E030E227900000041200B8B8E0FEA3E0DC
:20098000900848D575F00D1200B774EE75F00DA42583F583759308E04404F02115547B0999
:2009A0009000001A1200B8B8A982AA83C003C002C0017B09900000221200B8B8A982AA835D
:2009C0009008A5B3EBF0A3EAF0A3E9F0D001D002D00312060754855083855182A3A375936C
:2009E00008E4F0A3F0C390087ED4E09401FF90087ED3E09400FE855083855182A3A375930E
:200A000008E0FCA3E0FDC39FEE6480F8EC6480985075EDAE047803CEA2E713CE13D8F8FFE5
:200A2000900000221200B8B8E5822FF582E5833EF583759308E0FD855083855182A3A375FF
:200A40009308A3E05407FC7401A804088002C333D8FCFC5D601B900000391200B8B8E58226
:200A60002FF582E5833EF583759308E04C759308F0855083855182A3A3759308E475F00126
:200A80001200B4242109E5855083855182A3A3759308E4F0A3F0C390087ED4E09401FF903F
:200AA000087ED3E09400FE855083855182A3A3759308E0FCA3E0FDC39FEE6480F8EC64800D
:200AC000984003210B89EDAE047803CEA2E713CE13D8F8FF900000221200B8B8E5822FF593
:200AE00082E5833EF583759308E0FF855083855182A3A3759308A3E05407FE7401A806085A
:200B00008002C333D8FCFD5F6069855083855182A3A3759308E0FEA3E07803CEA2E713CE4A
:200B200013D8F8FF900000391200B8B8E5822FF582E5833EF583759308E05D7036900000DA
:200B4000441200B8B8E030E227900000041200B8B8E0FEA3E0900848D575F00D1200B774DB
:200B6000EE75F00DA42583F583759308E04404F0211554855083855182A3A3759308E47540
:200B8000F0011200B424210A96900000371200B8B8E0FEA3E0FF9000000E1200B8B8EEF012
:200BA000A3EFF07B09900000391200B8B8A982AA83C003C002C0017B09900000101200B858
:200BC000B8A982AA83A801AC02AD03D001D002D0037E007F041200B2A17B099000002212DA
:200BE00000B8B8A982AA83C003C002C0017B09900000141200B8B8A982AA83A801AC02ADE1
:200C000003D001D002D0037E007F041200B2A1855083855182A3A3759308E4F0A3F0C39035
:200C2000087ED4E09401FD90087ED3E09400FC855083855182A3A3759308E0FEA3E0FFC366
:200C40009DEC6480F8EE6480984003210D207B09900000181200B8B8A982AA831207191CE0
:200C60009000000E1200B8B8E0FEA3E0FF900000181200B8B8E0540FFCA3E06F7002EE6CCD
:200C80006003210D0A855083855182A3A3759308E0FEA3E07803CEA2E713CE13D8F8FF902D
:200CA0000000101200B8B8E5822FF582E5833EF583759308E0FF855083855182A3A375938A
:200CC00008A3E05407FE7401A806088002C333D8FC5F7036900000441200B8B8E030E22745
:200CE000900000041200B8B8E0FEA3E0900848D575F00D1200B774EE75F00DA42583F583F5
:200D0000759308E04404F0211554855083855182A3A3759308E475F0011200B424210C1E9C
:200D20007B099000000E1200B8B8A982AA83C003C002C001900000041200B8B8E0FEA3E0FA
:200D4000FF7C007D0D1200B38474C92FF974483EA801FC7D09D001D002D0037E007F0A122C
:200D600000B2A1900000041200B8B8E0FEA3E0FF900848D575F00D1200B774EE75F00DA442
:200D80002583F583759308E04404F0900848D375F00DEF1200B774EE75F00DA42583F58396
:200DA000759308E0FEA3E064014E6003211560900000041200B8B8E0FEA3E0FF7C007D0D9A
:200DC0001200B38474C92FF974483EFA7B09900000041200B8B8210FCA9000004E1200B835
:200DE000B8E0FBA3E0FAA3E0F91200B66B1200B8480E13000000010FD2000000020FD50039
:200E0000000004119B0000000512DA0000000600001554855083855182759308E0FEA3E0A1
:200E2000FF7B09900000041200B8B8A982AA83C003C002C0017B099000002A1200B8B8A912
:200E400082AA839008A5BDEBF0A3EAF0A3E9F0D001D002D0031206D0EAEF4E700321133BAE
:200E6000900000361200B8B8E0540764066003211554855083855182A3A3759308E4F0A31B
:200E8000F0855083855182A3A3759308E0FEA3E0FFC39440EE64809480504F7B09900000CC
:200EA0000E1200B8B8A982AA831206F578EF4E60399000000E1200B8B8E0FEA3E0FF85509A
:200EC00083855182759308E0FCA3E0B50707ECB5060321145E855083855182A3A3759308C2
:200EE000E475F0011200B4248097855083855182A3A3759308E0FAA3E0FBC39440EA6480E4
:200F0000948040032115547C007D0DAF03AE021200B38474C92FF974483EFA7B09C003C0DF
:200F200002C001900000041200B8B8E0FEA3E0FF7C007D0D1200B38474C92FF974483EA822
:200F400001FC7D09D001D002D0037E007F0D1200B2A1900000341200B8B8E4F0A304F07BFD
:200F6000099000002A1200B8B8A982AA83C001855083855182A3A3759308E0FEA3E0FF7C31
:200F8000007D0D1200B38474C92FF974483EA801FC7D09D0017E007F0D1200B2A18550835C
:200FA000855182A3A3759308E0FEA3E0FF7C007D0D1200B38474C92FF974483EFA7B098572
:200FC0005083855182A3A3759308E0FEA3E0FF211194211554855083855182A3A3759308DA
:200FE000E4F0A3F0855083855182A3A3759308E0FEA3E0FFC39440EE64809480506F7B0964
:201000009000000E1200B8B8A982AA831206F578EF4E701F855083855182A3A3759308E021
:20102000FEA3E0FF900000041200B8B8EEF0A3EFF0803A9000000E1200B8B8E0FEA3E0FF80
:20104000855083855182759308E0FCA3E0B50707ECB50603211554855083855182A3A3750F
:201060009308E475F0011200B424210FE4855083855182A3A3759308E0FEA3E0C39440EEA1
:2010800064809480400321155A855083855182759308E0FEA3E0FF9000000E1200B8B8EE57
:2010A000F0A3EFF0855083855182A3A3759308E4F0A3F0C390087ED4E09401FF90087ED347
:2010C000E09400FE855083855182A3A3759308E0FCA3E0FDC39FEE6480F8EC6480985063F5
:2010E000EDAE047803CEA2E713CE13D8F8FF900000101200B8B8E5822FF582E5833EF5836F
:20110000C083C082759308E0FF855083855182A3A3759308A3E05407FE7401A806088002CC
:20112000C333D8FC4F759308D082D083F0855083855182A3A3759308E475F0011200B424B7
:201140002110B37B09900000101200B8B8A982AA83C003C002C0017B09900000141200B875
:20116000B8A982AA83A801AC02AD03D001D002D0037E007F041200B2A1900000041200B81E
:20118000B8E0FEA3E0FF7B099000000E1200B8B8A982AA8312073A1E21154E855083855118
:2011A00082A3A3759308E4F0A3F0855083855182A3A3759308E0FEA3E0FFC39440EE648021
:2011C0009480502B7B09900000371200B8B8A982AA831206E46AEF4E601585508385518293
:2011E000A3A3759308E475F0011200B42480BB855083855182A3A3759308E0FEA3E0FF4E76
:20120000700E900000041200B8B8E4F0A3F08043C3EF9401FFEE9400FE900000041200B8EC
:20122000B8E0FCA3E0D39FEE6480F8EC648098401F855083855182A3A3759308E0FEA3E02D
:20124000FF900000041200B8B8EEF0A3EFF080032115547E007F0D7D007B09900000371228
:2012600000B8B8A982AA831200BBFD855083855182759308E0FEA3E0FF900000371200B82B
:20128000B8EEF0A3EFF0900000411200B8B8E4F0A37403F07B09900000371200B8B8A9820D
:2012A000AA83C003C002C001900000041200B8B8E0FEA3E0FF7C007D0D1200B38474C92F8A
:2012C000F974483EA801FC7D09D001D002D0037E007F0D1200B2A1211560855083855182C5
:2012E000759308E0FEA3E0FF7B09900000041200B8B8A982AA83C003C002C0017B09900032
:20130000002A1200B8B8A982AA839008A5BDEBF0A3EAF0A3E9F0D001D002D0031206D0EAB3
:20132000EF4E7005FEFF211563855083855182759308E0FEA3E064014E7006FE7F03211565
:2013400063900000041200B8B8E0FEA3E0FF900848D375F00D1200B774EE75F00DA42583A6
:20136000F583759308E0FCA3E064034C702AF58375820DC083C082FDC005FC7D0D1200B32B
:201380008474C92FF974483EFA7B09D005D007D0061200BBFD2115607E007F087D007B0904
:2013A000900000061200B8B8A982AA831200BBFD855083855182A3A3759308E4F0A3F08501
:2013C0005083855182A3A3759308E0FEA3E0FFC39440EE64809480506C7B099000000E12BF
:2013E00000B8B8A982AA831206F578EF4E60409000000E1200B8B8E0FEA3E0FF8550838566
:201400005182759308E0FCA3E0B50723ECB5061F855083855182A3A3759308E0FEA3E0FF7F
:20142000900000041200B8B8EEF0A3EFF08016855083855182A3A3759308E475F00112003E
:20144000B4242113BF855083855182A3A3759308E0FEA3E0C39440EE648094804003211564
:2014600060855083855182A3A3759308E4F0A3F0C390087ED4E09401FD90087ED3E0940023
:20148000FC855083855182A3A3759308E0FEA3E0FFC39DEC6480F8EE648098504C7B0990A8
:2014A0000000181200B8B8A982AA831207191C9000000E1200B8B8E0FEA3E0FF90000018C4
:2014C0001200B8B8E0540FFCA3E0B50707EEB50403211554855083855182A3A3759308E4E7
:2014E00075F0011200B4248087900000041200B8B8E0FEA3E07803CEA2E713CE13D8F8FF89
:20150000900000061200B8B8E5822FF582E5833EF583C083C082759308E0FF90000004126E
:2015200000B8B8A3E05407FE7401A806088002C333D8FC4F759308D082D083F07B099000E0
:2015400000061200B8B8A982AA831205BC01120718DF800C7E007F0380097E007F02800330
:20156000E4FEFF900000530200B891900841D2E0FBA3E0FAA3E02414F9E43AFA900841CFE5
:20158000EBF0A3EAF0A3E9F090084544E0FBA3E0FAA3E0242CF9E43AFA900848C0EBF0A3FC
:2015A000EAF0A3E9F090084544A3E0FAA3E0242BF9E43AFA9008454CEBF0A3EAF0A3E9F057
:2015C00090084544A3E0FAA3E02418F9E43AFA900848ACEBF0A3EAF0A3E9F090084544A379
:2015E000E0FAA3E0241AF9E43AFA90084549EBF0A3EAF0A3E9F090084544A3E0FAA3E02400
:201600001CF9E43AFA900848BDEBF0A3EAF0A3E9F090084544A3E0FAA3E0241EF9E43AFAB8
:20162000900848AFEBF0A3EAF0A3E9F090084544A3E0FAA3E02420F9E43AFA900848B2EB54
:20164000F0A3EAF0A3E9F090084544A3E0FAA3E02422F9E43AFA90084553EBF0A3EAF0A3FE
:20166000E9F090084544A3E0FAA3E02424F9E43AFA900848B6EBF0A3EAF0A3E9F0900845D0
:2016800044A3E0FAA3E02426F9E43AFA90084556EBF0A3EAF0A3E9F090084437E0FD30E69E
:2016A00067900848C0E0FBA3E0FAA3E0F9E41200B370900848C0E0FBA3E0FAA3E02402F99C
:2016C000E43AFAE4F5F01200B4CA900848ACE0FBA3E0FAA3E0F9E475F0011200B4CA9008C7
:2016E00048BDE0FBA3E0FAA3E0F9E475F0011200B4CA900848B2E0FBA3E0FAA3E0F9E4F5F8
:20170000F01200B4CA2127D1ED30E7032127D190084437E020E103212526900848C0E0FB32
:20172000A3E0FAA3E0F91200B31F60032125269008A66B7481F0A374C0F0A3745AF0A3E4C0
:20174000F0A37404F0900841CFE0FBA3E0FAA3E0F91206D8AEEF60032117E890088AB7F039
:20176000900841CFE0FBA3E0FAA3E02405F9E43AFA90088AB7E0FF7C0029F9EC3AFAA3EBA8
:20178000F0A3EAF0A3E9F01200B31FFE64206004EEB43F1174BB2FF582E4348AF5837593AD
:2017A00008E4F0801F90088AB7E0FF04F074BB2FF582E4348AF583759308EEF090088AB74C
:2017C000E0B4209C7B097A8A79BB1200CB03EF4E600321188778BB7C8A7D097B817AC0794F
:2017E0005F1200BA3F2118879008A0737481F0A374C0F0A37469F0900841CFE0FBA3E0FAF8
:20180000A3E0F912065EEB90088AB8EBF0A3EAF0A3E9F090088AB8E0FBA3E0FAA3E04A4BF3
:20182000701C900848B5E064037003211C51900841CFE0FBA3E0FAA3E0F9020369F69008C7
:2018400095057481F0A374C0F0A37469F0A37481F0A374C0F0A37473F0A37409F0A3748A58
:20186000F0A374BBF090088AB8E0FBA3E0FAA3E0F9120585CB900848C0E0FBA3E0FAA3E026
:20188000F974011200B3709008A66B7481F0A374C0F0A37475F0A3E4F0A3740AF07B097A4E
:2018A0008A79BB1206D8AEEF704A90084544E0FBA3E0FAA3E02404F9E43AFA1200B66B902B
:2018C0000848B9E0F8A3E0F9A3E0FAA3E0FBC31200B63470032119DBE4FFFEFDFC900848AF
:2018E000B9E0F8A3A3A3E0C31200B6346003211AD52119DB9008A66B7481F0A374C0F0A34F
:201900007480F0A3E4F0A3740AF07B097A8A79BB1206D8AEEF701078BB7C8A7D097B817A5D
:20192000C0798B1200BA3F9008A66B7481F0A374C0F0A37498F0A3E4F0A37404F07B097A64
:201940008A79BB1206D8AEEF7003211A949008A66B7481F0A374C0F0A3749DF0A3E4F0A3E7
:20196000740BF07B097A8A79BB1206D8AEEF704E900848C0E0FBA3E0FAA3E0F974021200F5
:20198000B3707B007A007900C003C002C001900848C0E0FBA3E0FAA3E02404F9E43AFA12AA
:2019A00000B79D900848C0E0FBA3E0FAA3E02402F9E43AFAE4F5F01200B4CA2126E3900806
:2019C000A3D47409F0A3748AF0A374B2F07B097A8A79BB12061F73EF4E702378BB7C8A7DED
:2019E000097B817AC079A91200BA3F900848B57401F0E4FFFEFDFC900848B9211BFF90083B
:201A000048C0E0FBA3E0FAA3E0F974021200B37090088AB2E0FBA3E0FAA3E0F9C003C00212
:201A2000C001900848C0E0FBA3E0FAA3E02404F9E43AFA1200B79D90088AB5E0FEA3E0FF94
:201A4000900848C0E0FBA3E0FAA3E02402F9E43AFAEE8FF01200B4CA1207373EC004C005C0
:201A6000C006C00712073B60E4FCFD7B587A02F9F81200B4E6D003D002D001D000EB2FFFFD
:201A8000EA3EFEE93DFDE83CFC9008454F1200B7572126E390084544E0FBA3E0FAA3E02447
:201AA00004F9E43AFA1200B66B900848B9E0F8A3E0F9A3E0FAA3E0FBC31200B634603EE4B5
:201AC000FFFEFDFC900848B9E0F8A3A3A3E0C31200B63460289008A3CB7481F0A374C0F0DD
:201AE000A374B9F0A37481F0A374C0F0A374A9F07B817AC079B31206A2152127D1900848FD
:201B0000C0E0FBA3E0FAA3E0F91200B31F64016003211C069008A66B7481F0A374C0F0A34A
:201B200074D1F0A3E4F0A3740AF07B097A8A79BB1206D8AEEF6003211C06900841CFE0FB76
:201B4000A3E0FAA3E0F91206AACEEF4E70289008A3CB7481F0A374C0F0A374DCF0A37481FA
:201B6000F0A374C0F0A374A9F07B817AC079B31206A2152127D11206B9A4EF4E70289008D2
:201B8000A3CB7481F0A374C0F0A374EBF0A37481F0A374C0F0A374A9F07B817AC079B312C6
:201BA00006A2152127D190084544E0FBA3E0FAA3E02404F9E43AFA1200B66B900848B9123C
:201BC00000B757900848B57402F01207373EC004C005C006C00712073B60E4FCFD7B587A7A
:201BE00002F9F81200B4E6D003D002D001D000EB2FFFEA3EFEE93DFDE83CFC9008454F1240
:201C000000B7572123199008A66B7481F0A374C0F0A374A9F0A3E4F0A37409F07B097A8A45
:201C200079BB1206D8AEEF7009900848B504F0212319900848B5E0B4010F78BB7C8A7D098C
:201C40007B817AC079A9212315900848B5E0B4033C9008A3CB7481F0A374C1F0A37405F0AC
:201C6000A37481F0A374C0F0A374A9F07B817AC079B31206A215900848B57401F0E4FFFE59
:201C8000FDFC900848B91200B7572127D1900848C0E0FBA3E0FAA3E0F91200B31F6401605C
:201CA000032123199008A66B7481F0A374C1F0A37413F0A3E4F0A37408F07B097A8A79BB12
:201CC0001206D8AEEF701A900841CFE0FBA3E0FAA3E0F91204E6DEEF4E6003212319212257
:201CE0008F9008A66B7481F0A374C1F0A3741CF0A3E4F0A3740BF07B097A8A79BB1206D8A7
:201D0000AEEF7026900841CFE0FBA3E0FAA3E0F9120534D7EF4E700321228F78BB7C8A7DBA
:201D2000097B817AC179282123159008A66B7481F0A374C1F0A37428F0A3E4F0A37408F05E
:201D40007B097A8A79BB1206D8AEEF701A900841CFE0FBA3E0FAA3E0F9120457B9EF4E6071
:201D60000321231921228F9008A66B7481F0A374C1F0A37431F0A3E4F0A37407F07B097A20
:201D80008A79BB1206D8AEEF701A900841CFE0FBA3E0FAA3E0F912032D0AEF4E60032123C2
:201DA0001921228F9008A66B7481F0A374C1F0A37439F0A3E4F0A3740AF07B097A8A79BB5E
:201DC0001206D8AEEF7026900841CFE0FBA3E0FAA3E0F91206BE3FEF4E700321228F78BB9A
:201DE0007C8A7D097B817AC179312123159008A66B7481F0A374C1F0A37444F0A3E4F0A362
:201E00007409F07B097A8A79BB1206D8AEEF701A900841CFE0FBA3E0FAA3E0F9120445901B
:201E2000EF4E600321231921228F9008A66B7481F0A374C1F0A3744EF0A3E4F0A3740AF0A0
:201E40007B097A8A79BB1206D8AEEF701A900841CFE0FBA3E0FAA3E0F91204529EEF4E6090
:201E60000321231921228F9008A66B7481F0A374C1F0A37459F0A3E4F0A37411F07B097AED
:201E80008A79BB1206D8AEEF701A900841CFE0FBA3E0FAA3E0F91205DB61EF4E60032123BA
:201EA0001921228F9008A66B7481F0A374C1F0A3746BF0A3E4F0A3740DF07B097A8A79BB28
:201EC0001206D8AEEF701A900841CFE0FBA3E0FAA3E0F91204CA26EF4E6003212319212229
:201EE0008F9008A66B7481F0A374C1F0A37479F0A3E4F0A37407F07B097A8A79BB1206D84C
:201F0000AEEF701A900841CFE0FBA3E0FAA3E0F9120228C6EF4E600321231921228F9008B5
:201F2000A66B7481F0A374C1F0A37481F0A3E4F0A37407F07B097A8A79BB1206D8AEEF701D
:201F40001A900841CFE0FBA3E0FAA3E0F91202803EEF4E600321231921228F9008A66B742D
:201F600081F0A374C1F0A37489F0A3E4F0A37408F07B097A8A79BB1206D8AEEF701A9008A7
:201F800041CFE0FBA3E0FAA3E0F91204D6C3EF4E600321231921228F9008A66B7481F0A3AE
:201FA00074C1F0A37492F0A3E4F0A37407F07B097A8A79BB1206D8AEEF701A900841CFE083
:201FC000FBA3E0FAA3E0F91206BF63EF4E600321231921228F9008A66B7481F0A374C1F0AE
:201FE000A3749AF0A3E4F0A37409F07B097A8A79BB1206D8AEEF701A900841CFE0FBA3E0E0
:20200000FAA3E0F912057FEFEF4E600321231921228F9008A66B7481F0A374C1F0A374A5E4
:20202000F0A3E4F0A37407F07B097A8A79BB1206D8AEEF701A900841CFE0FBA3E0FAA3E0D5
:20204000F91205BD46EF4E600321231921228F9008A66B7481F0A374C1F0A374ADF0A3E40D
:20206000F0A37408F07B097A8A79BB1206D8AEEF7013900841CFE0FBA3E0FAA3E0F9120502
:20208000E1262123199008A66B7481F0A374C1F0A374B6F0A3E4F0A37409F07B097A8A7941
:2020A000BB1206D8AEEF7013900841CFE0FBA3E0FAA3E0F91205DFFF2123199008A66B746A
:2020C00081F0A374C1F0A374C0F0A3E4F0A37408F07B097A8A79BB1206D8AEEF7026900803
:2020E00041CFE0FBA3E0FAA3E0F91201547CEF4E700321228F78BB7C8A7D097B817AC17928
:20210000C02123159008A66B7481F0A374C1F0A374C9F0A3E4F0A37407F07B097A8A79BB3F
:202120001206D8AEEF701A900841CFE0FBA3E0FAA3E0F912047F56EF4E60032123192122E1
:202140008F9008A66B7481F0A374C1F0A374D1F0A3E4F0A3740AF07B097A8A79BB1206D88E
:20216000AEEF7026900841CFE0FBA3E0FAA3E0F912052A4DEF4E700321228F78BB7C8A7DEA
:20218000097B817AC179C92123159008A66B7481F0A374C1F0A374DCF0A3E4F0A3740CF0A1
:2021A0007B097A8A79BB1206D8AEEF7026900841CFE0FBA3E0FAA3E0F91204E8D4EF4E7045
:2021C0000321228F78BB7C8A7D097B817AC179282123159008A66B7481F0A374C1F0A374CD
:2021E000E9F0A3E4F0A37408F07B097A8A79BB1206D8AEEF701A900841CFE0FBA3E0FAA30A
:20220000E0F91204F09DEF4E600321231921228F9008A66B7481F0A374C1F0A374F2F0A381
:20222000E4F0A3740AF07B097A8A79BB1206D8AEEF7025900841CFE0FBA3E0FAA3E0F9124D
:20224000025BFFEF4E7002804678BB7C8A7D097B817AC179FD2123159008A66B7481F0A3B7
:2022600074C2F0A37405F0A3E4F0A3740AF07B097A8A79BB1206D8AEEF7026900841CFE03D
:20228000FBA3E0FAA3E0F91204BF80EF4E7004FE7F012278BB7C8A7D097B817AC179FD80B8
:2022A000749008A66B7481F0A374C2F0A37410F0A3E4F0A37409F07B097A8A79BB1206D809
:2022C000AEEF701290087EBFF0A304F0900844377410F02127D19008A66B7481F0A374C27C
:2022E000F0A3741AF0A3E4F0A3740DF07B097A8A79BB1206D8AEEF7020900841CFE0FBA343
:20230000E0FAA3E0F912070B1D78BB7C8A7D097B817AC179131200BA3F9008A66B7481F00B
:20232000A374C1F0A37428F0A3E4F0A37408F07B097A8A79BB1206D8AEEF701812073B6992
:20234000EF4E701078BB7C8A7D097B817AC179FD1200BA3FE490088AB7F09008A66B7481FE
:20236000F0A374C2F0A37428F0A3E4F0A3740BF07B097A8A79BB1206D8AEEF701412047C8D
:20238000EC78BB7C8A7D097B817AC279341200BA3F9008A66B7481F0A374C2F0A37440F004
:2023A000A3E4F0A3740BF07B097A8A79BB1206D8AEEF701A9008ABA5F0A304F078BB7C8A19
:2023C0007D097B817AC2794C1200BA3F8008E49008ABA5F0A3F09008A66B7481F0A374C231
:2023E000F0A37458F0A3E4F0A3740AF07B097A8A79BB1206D8AEEF701078BB7C8A7D097B03
:20240000817AC279631200BA3FE49008ABA1F0A3F09008A66B7481F0A374C1F0A374F2F07E
:20242000A3E4F0A3740AF07B097A8A79BB1206D8AEEF7045900889D87481F0A374C2F0A3CC
:20244000746EF0A37409F0A374ABF0A374A1F07B097A8A79BB1200BD8B78BB7C8A7D097BF0
:20246000817AC179FD1200BA3F9008ABA2E024FFF09008ABA1E034FFF090088AB7E0FD7535
:20248000F017A42459F582E5F03445F583759308E0FBA3E0FAA3E04A4B700A900844377456
:2024A00010F02127D1ED75F017A4245CF9744535F0FA7B091200CB039008A66EEEF0A3EF25
:2024C000F090088AB7E075F017A4245CF9744535F0FA9008A66B7409F0A3EAF0A3E9F07B58
:2024E000097A8A79BB1206D8AEEF7030900848C0E0FBA3E0FAA3E0F974031200B3709008B6
:202500008AB7E0FF900848C0E0FBA3E0FAA3E02401F9E43AFAEF1200B370800A90088AB763
:20252000E004F0212479900848C0E0FBA3E0FAA3E0F91200B31F640360032126E3900845E0
:2025400047F0A3F090084437E0640460032125D790084549E0FBA3E0FAA3E0F91200B450C6
:20256000FF900848ACE0FBA3E0FAA3E0F9E5F08FF01200B4CA900848AFE0FBA3E0FAA3E0AE
:20258000F91200B450FF900848BDE0FBA3E0FAA3E0F9E5F08FF01200B4CA90084553E0FBCD
:2025A000A3E0FAA3E0F91200B450FF900848B2E0FBA3E0FAA3E0F9E5F08FF01200B4CA9033
:2025C000084556E0FBA3E0FAA3E0F91200B450FF900848B621265B900848ACE0FBA3E0FA53
:2025E000A3E0F91200B450FF90084549E0FBA3E0FAA3E0F9E5F08FF01200B4CA900848BDCF
:20260000E0FBA3E0FAA3E0F91200B450FF900848AFE0FBA3E0FAA3E0F9E5F08FF01200B454
:20262000CA900848B2E0FBA3E0FAA3E0F91200B450FF90084553E0FBA3E0FAA3E0F9E5F07C
:202640008FF01200B4CA900848B6E0FBA3E0FAA3E0F91200B450FF90084556E0FBA3E0FA61
:20266000A3E0F9E5F08FF01200B4CA900848C0E0FBA3E0FAA3E02401F9E43AFA1200B31F65
:2026800075F017A42459F582E5F03445F583759308E0FBA3E0FAA3E0F91200B884EF6007D8
:2026A000900844377410F01207373EC004C005C006C00712073B60E4FCFD7B587A02F9F81E
:2026C0001200B4E6D003D002D001D000EB2FFFEA3EFEE93DFDE83CFC9008454F1200B7573A
:2026E0002127D190084437E030E07A900848C0E0FBA3E0FAA3E02402F9E43AFA1200B4507C
:20270000C394B0E5F09404402A74FB75F0501200B49E900848C0E0FBA3E0FAA3E02404F9B7
:20272000E43AFA09E970010A740475F0B01200B49E8032900848C0E0FBA3E0FAA3E02402D0
:20274000F9E43AFAE4F5F01200B4CA900848C0E0FBA3E0FAA3E0F91200B31FB40207900862
:2027600044377410F0900848C0E0FBA3E0FAA3E02402F9E43AFA1200B450FFAEF0D394B0EE
:20278000EE94049008454740097404F0A374B0F08005EEF0A3EFF090084547E0FEA3E0FFBE
:2027A000900848C0E0FBA3E0FAA3E02404F9E43AFA1200B780C003C002900841CFE0FBA371
:2027C000E0FAA3E0F8AC02AD03D002D0031200B2A17E007F01229000FFFD1200B891EBF05A
:2027E000A3EAF0A3E9F09000FFB61200B891900000561200B8B8E0FEA3E0FF900000561280
:2028000000B8B8EEF0A3EFF0900000501200B8B8E0FBA3E0FAA3E0F91200B450FDACF0C340
:20282000940DEC6480948050032139269000004D1200B8B8E0FBA3E0FAA3E0F9C003C00288
:20284000C001C3ED9401FDEC9400FC9000004A1200B8B8E0F9A3E0FAA3E090089F19C9F0BB
:20286000A3EAF0A3E9F09000004A1200B8B8E0FBA3E0FAA3E02434F9E43AFA1200B450C3E6
:202880009401FEE5F0940090089F1CF0A3CEF0D001D002D0031206054BEF4E60032139269A
:2028A0007C007D02900000501200B8B8E0FBA3E0FAA3E0F91200B45025E0FFE5F033FE9037
:2028C00000004D1200B8B8E0FBA3E0FAA3E02FF9EA3EFAC3E99DF9EA9CFA1200B450FFAE7F
:2028E000F0855083855182759308EEF0A3EFF0855083855182759308E0FEA3E0FFC3940150
:20290000EE64809480400BD3EF9404EE64809480400321392685508385518275930874FF50
:20292000F5F01200B4249000004A1200B8B8E0FBA3E0FAA3E02437F9E43AFA1200B450FF10
:20294000AEF0E5F06003213926EF24FEB40D0040032139269001296375F004A4C58325F005
:20296000C583730201299702012AFB02012CC702012EBA0201301D0201316A020133D102D9
:202980000133D1020133D1020133D1020133D1020133D4020135D485508385518275930847
:2029A000E0FEA3E0FF90086E8975F03F1200B774EE75F03FA42583F583759308E0FD900074
:2029C00000431200B8B8EDF090086E8975F03FEF1200B774EE75F03FA42583F58375930890
:2029E000ED54FEF0900000531200B8B8E0FBA3E0FAA3E0F91200CB03D3EF9414EE648094BF
:202A000080403A900000431200B8B8E020E00321391E855083855182759308E0FEA3E0905B
:202A2000086E8975F03F1200B774EE75F03FA42583F583759308E04401F021391E90000033
:202A4000531200B8B8E0FBA3E0FAA3E0F9C001855083855182759308E0FEA3E0FF7C007DF3
:202A60003F1200B384744B2FF9746E3EA801FC7D09D0017E007F151200B2A1855083855126
:202A800082759308E0FEA3E0FF90086E8975F03F1200B774EE75F03FA42583F5837593086E
:202AA000E04401F090086E8775F03FEF1200B774EE75F03FA42583F583759308E0FEA3E0DD
:202AC00064014E600321392C855083855182759308E0FEA3E0FF7C007D3F1200B384744BFA
:202AE0002FF9746E3EFA7B09855083855182759308A3E0FD120730952135CD8550838551A1
:202B000082759308E0FEA3E0FF90086E8975F03F1200B774EE75F03FA42583F583759308ED
:202B2000E0FD900000431200B8B8EDF090086E8975F03FEF1200B774EE75F03FA42583F554
:202B400083759308ED54FDF0900000531200B8B8E0FBA3E0FAA3E0F9120427BDEFF470022C
:202B6000EEF47037900000431200B8B8E030E128855083855182759308E0FEA3E090086E37
:202B80008975F03F1200B774EE75F03FA42583F583759308E04402F021391E9000005312E2
:202BA00000B8B8E0FBA3E0FAA3E0F91200B66B12061987EF4E604D900000411200B8B8E0C9
:202BC000FEA3E0FF855083855182759308E0FCA3E0FD6F7002EC6E602B900000431200B8F6
:202BE000B8E030E11C90086E8975F03FED1200B774EC75F03FA42583F583759308E0440229
:202C0000F021391E900000531200B8B8E0FBA3E0FAA3E0F91200B66B855083855182759328
:202C200008E0FAA3E0FB90086E6075F03F1200B774EA75F03FA42583F5837593081200B7C2
:202C40005790086E8975F03FEB1200B774EA75F03FA42583F583759308E04402F090086E44
:202C60008775F03FEB1200B774EA75F03FA42583F583759308E0FEA3E064014E60032139CE
:202C80002C855083855182759308E0FEA3E090086E6075F03F1200B774EE75F03FA42583C2
:202CA000F583759308E0FCA3E0FDA3E0FEA3E0FF855083855182759308A3E09008A934F085
:202CC00012072FA92135CD855083855182759308E0FEA3E0FF90086E8975F03F1200B77450
:202CE000EE75F03FA42583F583759308E0FD900000431200B8B8EDF090086E8975F03FEF3D
:202D00001200B774EE75F03FA42583F583759308ED54FBF0900000531200B8B8E0FBA3E021
:202D2000FAA3E0F91200CB03C3EE64809480401F900000531200B8B8E0FBA3E0FAA3E0F9FC
:202D40001200CB03D3EF9414EE648094804037900000431200B8B8E030E22885508385512F
:202D600082759308E0FEA3E090086E8975F03F1200B774EE75F03FA42583F583759308E0AA
:202D80004404F021391E855083855182759308E0FEA3E090086E8675F03F1200B774EE7592
:202DA000F03FA42583F583759308E0604F900000531200B8B8E0FBA3E0FAA3E0F91200CB6B
:202DC00003EF4E7037900000431200B8B8E030E228855083855182759308E0FEA3E09008E4
:202DE0006E8975F03F1200B774EE75F03FA42583F583759308E04404F021391E9000005322
:202E00001200B8B8E0FBA3E0FAA3E0F9C001855083855182759308E0FEA3E0FF7C007D3F43
:202E20001200B38474642FF9746E3EA801FC7D09D0017E007F151200B2A185508385518206
:202E4000759308E0FEA3E0FF90086E8975F03F1200B774EE75F03FA42583F583759308E04C
:202E60004404F090086E8775F03FEF1200B774EE75F03FA42583F583759308E0FEA3E06492
:202E8000014E600321392C855083855182759308E0FEA3E0FF7C007D3F1200B38474642F52
:202EA000F9746E3EFA7B09855083855182759308A3E0FD120730782135CD855083855182A7
:202EC000759308E0FEA3E0FF90086E8975F03F1200B774EE75F03FA42583F583759308E0CC
:202EE000FD900000431200B8B8EDF090086E8975F03FEF1200B774EE75F03FA42583F583EE
:202F0000759308ED54F7F0900000531200B8B8E0FBA3E0FAA3E0F91200B66B1200B8482FCC
:202F20002F000000012F3B0000000200002F48900000441200B8B8E4F080449000004412AA
:202F400000B8B87401F08037900000431200B8B8E030E328855083855182759308E0FEA334
:202F6000E090086E8975F03F1200B774EE75F03FA42583F583759308E04408F021391E9077
:202F80000000441200B8B8E0FF855083855182759308E0FCA3E0FD90086E7975F03F12003B
:202FA000B774EC75F03FA42583F583759308EFF090086E8975F03FED1200B774EC75F03FB6
:202FC000A42583F583759308E04408F090086E8775F03FED1200B774EC75F03FA42583F5D5
:202FE00083759308E0FEA3E064014E600321392C90086E7975F03FED1200B774EC75F03F64
:20300000A42583F583759308E0FF855083855182759308A3E0FD1207330F2135CD855083E7
:20302000855182759308E0FEA3E090086E7A75F03F1200B774EE75F03FA42583F583759308
:2030400008E0FCA3E0FDA3E0FEA3E0FF900000451200B8B81200B757900000531200B8B82D
:20306000E0FBA3E0FAA3E0F91200B66B1200B848308000000001309A00000002000030C1C9
:20308000900000451200B8B8C083C082E0FCA3E0FDA3E0FEA3E04401801890000045120030
:2030A000B8B8C083C082E0FCA3E0FDA3E0FEA3E054FEFFEC759308D082D0831200B7578029
:2030C0000321391E900000451200B8B8E0FCA3E0FDA3E0FEA3E0FF855083855182759308FF
:2030E000E0FAA3E0FB90086E7A75F03F1200B774EA75F03FA42583F5837593081200B75795
:2031000090086E8775F03FEB1200B774EA75F03FA42583F583759308E0FEA3E064014E6080
:203120000321392C855083855182759308E0FEA3E090086E7A75F03F1200B774EE75F03FF2
:20314000A42583F583759308E0FCA3E0FDA3E0FEA3E0FF855083855182759308A3E0900861
:20316000A925F012072EF52135CD855083855182759308E0FEA3E090086E8275F03F1200D3
:20318000B774EE75F03FA42583F583759308E0FCA3E0FDA3E0FEA3E0FF900000451200B8A0
:2031A000B81200B757900000531200B8B8E0FBA3E0FAA3E0F91200B66B1200B84831CD00BB
:2031C00000000131E7000000020000320E900000451200B8B8C083C082E0FCA3E0FDA3E0D9
:2031E000FEA3E044028018900000451200B8B8C083C082E0FCA3E0FDA3E0FEA3E054FDFFE4
:20320000EC759308D082D0831200B757800321391E900000451200B8B8E0FCA3E0FDA3E0BC
:20322000FEA3E0FF855083855182759308E0FAA3E0FB90086E8275F03F1200B774EA75F03E
:203240003FA42583F5837593081200B75790086E7E75F03FEB1200B774EA75F03FA4258311
:20326000F583759308E0FCA3E0FDA3E0FEA3E0FF900000451200B8B81200B757900000530D
:203280001200B8B8E0FBA3E0FAA3E0F91200B66B1200B84832A40000000132BE00000002CA
:2032A000000032E5900000451200B8B8C083C082E0FCA3E0FDA3E0FEA3E04401801890004E
:2032C00000451200B8B8C083C082E0FCA3E0FDA3E0FEA3E054FEFFEC759308D082D083123E
:2032E00000B757800321391E900000451200B8B8E0FCA3E0FDA3E0FEA3E0FF8550838551E1
:2033000082759308E0FAA3E0FB90086E7E75F03F1200B774EA75F03FA42583F583759308FC
:203320001200B75790086E8775F03FEB1200B774EA75F03FA42583F583759308E0FEA3E051
:2033400064014E600321392C855083855182759308E0FEA3E090086E8275F03F1200B77447
:20336000EE75F03FA42583F583759308E0FCA3E0FDA3E0FEA3E0FF855083855182759308C8
:20338000A3E09008A92AF012072F31855083855182759308E0FEA3E090086E7E75F03F127B
:2033A00000B774EE75F03FA42583F583759308E0FCA3E0FDA3E0FEA3E0FF8550838551826D
:2033C000759308A3E09008A92FF012072F6D2135CD213926855083855182759308E0FEA361
:2033E000E0FF90086E8975F03F1200B774EE75F03FA42583F583759308E0FD900000431256
:2034000000B8B8EDF090086E8975F03FEF1200B774EE75F03FA42583F583759308ED54EF6A
:20342000F0900000531200B8B8E0FBA3E0FAA3E0F91200B66B1200B848344900000001346C
:20344000560000000200003462900000491200B8B87401F08043900000491200B8B8E4F0CC
:203460008037900000431200B8B8E030E428855083855182759308E0FEA3E090086E8975FF
:20348000F03F1200B774EE75F03FA42583F583759308E04410F021391E900000491200B81B
:2034A000B8E07003213532855083855182759308E0FEA3E0FF7C007D3F1200B38474602FD5
:2034C000F9746E3EFA7B09120427BDEFF47002EEF46028855083855182759308E0FEA3E07B
:2034E000FF7C007D3F1200B38474642FF9746E3EFA7B091200CB03EF4E7037900000431205
:2035000000B8B8E030E428855083855182759308E0FEA3E090086E8975F03F1200B774EEA0
:2035200075F03FA42583F583759308E04410F021391E900000491200B8B8E0FF8550838560
:203540005182759308E0FCA3E0FD90086E8675F03F1200B774EC75F03FA42583F583759363
:2035600008EFF090086E8975F03FED1200B774EC75F03FA42583F583759308E04410F090EF
:20358000086E8775F03FED1200B774EC75F03FA42583F583759308E0FEA3E064014E600385
:2035A00021392C90086E8675F03FED1200B774EC75F03FA42583F583759308E0FF85508390
:2035C000855182759308A3E0FD12073327120718DF21392C900000531200B8B8E0FBA3E037
:2035E000FAA3E0F91200B66B1200B848360E0000000136CF0000000236D20000000436D5AD
:203600000000000537C2000000060000391E1206C5939000003D1200B8B8E060032136AE48
:203620009000003E1200B8B8E0FEA3E04E7006FE7F0321392FE4FFFEFDFC90000017120079
:20364000B8B8E0F8A3E0F9A3E0FAA3E0FBC31200B634606C7B09900000171200B8B8A98248
:20366000AA83120427BDBEFF06BFFF0321391E900000171200B8B8E0FCA3E0FDA3E0FEA37E
:20368000E0FF12061987EF4E6036900000411200B8B8E0FEA3E0FF8550838551827593084D
:2036A000E0FCA3E06F7002EC6E601521391E900000401200B8B8E054066406600321391EB2
:2036C0009000003E1200B8B8E4F0A3042138A621391E21391E1206C593EF4E600321391EA8
:2036E0007E007F3F7D007B09855083855182A3A3759308A982AA831200BBFD9000003E1285
:2037000000B8B8E4F0A37403F07B09855083855182A3A3759308A982AA83855083855182C9
:20372000759308A3E0FD12071B38900000401200B8B8E4F0FFFEFDFC900000171200B8B848
:20374000E0F8A3E0F9A3E0FAA3E0FBC31200B634600C900000401200B8B8E04402F07B0903
:203760009000001B1200B8B8A982AA831200CB03EF4E600C900000401200B8B8E04404F0D1
:203780007B09855083855182A3A3759308A982AA83C001855083855182759308E0FEA3E065
:2037A000FF7C007D3F1200B384744B2FF9746E3EA801FC7D09D0017E007F3F1200B2A121C4
:2037C0003924855083855182759308E0FEA3E0FF90086E8775F03F1200B774EE75F03FA4C8
:2037E0002583F583759308E0FCA3E04C7002802E855083855182759308E0FEA3E0FF900816
:203800006E8775F03F1200B774EE75F03FA42583F583759308E0FCA3E064034C702AF58348
:2038200075823FC083C082FDC005FC7D3F1200B384744B2FF9746E3EFA7B09D005D007D009
:20384000061200BBFD21392C855083855182759308E0FEA3E090086E8775F03F1200B77483
:20386000EE75F03FA42583F583759308E0FEA3E064014E600321391CFE7F3FFD7B098550E3
:2038800083855182A3A3759308A982AA831200BBFD9000003E1200B8B8E4F0A3F09000008E
:2038A000401200B8B8E4F07B09855083855182A3A3759308A982AA83C0018550838551821F
:2038C000759308E0FEA3E0FF7C007D3F1200B384744B2FF9746E3EA801FC7D09D0017E0076
:2038E0007F3F1200B2A1855083855182759308E0FEA3E0FF7C007D3F1200B384744B2FF91D
:20390000746E3EFA7B09855083855182759308A3E0FD1207260D120718DF800880007E00E7
:203920007F03800B80067E007F028003E4FEFF900000580200B8919000FFFD1200B891EB8C
:20394000F0A3EAF0A3E9F09000FFA71200B89112073B69EF4E7006FE7F022148BE90000047
:203960005F1200B8B8E0FBA3E0FAA3E0F91200B450FDACF0C3940DEC6480948050032148DF
:20398000B59000005C1200B8B8E0FBA3E0FAA3E0F9C003C002C001C3ED9401FDEC9400FC2C
:2039A000900000591200B8B8E0F9A3E0FAA3E090089F19C9F0A3EAF0A3E9F09000005912C6
:2039C00000B8B8E0FBA3E0FAA3E02434F9E43AFA1200B450C39401FEE5F0940090089F1C0B
:2039E000F0A3CEF0D001D002D0031206054BEF4E60032148B57C007D029000005F1200B826
:203A0000B8E0FBA3E0FAA3E0F91200B45025E0FFE5F033FE9000005C1200B8B8E0FBA3E02E
:203A2000FAA3E02FF9EA3EFAC3E99DF9EA9CFA1200B450FFAEF0855083855182A3A375934C
:203A400008EEF0A3EFF0855083855182A3A3759308E0FEA3E0FFC39401EE64809480400B0F
:203A6000D3EF9410EE6480948040032148B5855083855182A3A375930874FFF5F01200B475
:203A800024900000591200B8B8E0FBA3E0FAA3E02437F9E43AFA1200B450FFAEF0E5F06068
:203AA000032148B5EF24FD7003213D0024FE70032140D8240360032148B5855083855182DE
:203AC000A3A3759308A3E0C4F8540FC868FF0582D5820215831582E0C454F048FE74522F8D
:203AE000F58274683EF583759308E0FD900000581200B8B8EDF074522FF58274683EF5838B
:203B0000759308ED54FEF0900000621200B8B8E0FBA3E0FAA3E0F91200CB03D3EF9408EEF2
:203B2000648094804046900000581200B8B8E020E0032148AF855083855182A3A37593089C
:203B4000A3E0C4F8540FC868FF0582D5820215831582E0C454F048FE74522FF58274683ED1
:203B6000F583759308E04401F02148AF855083855182759308E4F0A3F08550838551827544
:203B80009308E0FEA3E0FFC39410EE64809480501B1206CCAAEF4E6013855083855182750F
:203BA0009308E475F0011200B42480CD855083855182759308E0FEA3E0FF4E7010855083A3
:203BC000855182A3A3759308F0A3F08041C3EF9401FFEE9400FE855083855182A3A375932F
:203BE00008E0FCA3E0D39FEE6480F8EC648098401D855083855182759308E0FFA3E0855066
:203C000083855182A3A3759308CFF0A3EFF07E007F217D007B09900000171200B8B8A982BF
:203C2000AA831200BBFD900000651200B8B8E0FEA3E0FF900000621200B8B8E0FBA3E0FAEA
:203C4000A3E0F9C003C002C0017B09900000171200B8B8A982AA83A801AC02AD03D001D0F5
:203C600002D0031200B2A17B09900000171200B8B8A982AA83C001855083855182A3A375D9
:203C80009308A3E0C4F8540FC868FF0582D5820215831582E0C454F048FE74432FF97468C0
:203CA0003EA801FC7D09D0017E007F091200B2A1855083855182A3A3759308A3E0C4F854C6
:203CC0000FC868FF0582D5820215831582E0C454F048FE74522FF58274683EF5837593085B
:203CE000E04401F074502FF58274683EF583759308E0FEA3E064014E60032148BB2140CDDA
:203D0000855083855182A3A3759308A3E0C4F8540FC868FF0582D5820215831582E0C454C5
:203D2000F048FE74522FF58274683EF583759308E0FD900000581200B8B8EDF074522FF531
:203D40008274683EF583759308ED54FDF0900000651200B8B8E0FEA3E0D39404EE64809468
:203D6000804043900000581200B8B8E030E134855083855182A3A3759308A3E0C4F8540F09
:203D8000C868FF0582D5820215831582E0C454F048FE74522FF58274683EF583759308E0C9
:203DA0004402F02148AF855083855182759308E4F0A3F0855083855182759308E0FEA3E06D
:203DC000FFC39410EE64809480501B1206CCAAEF4E6013855083855182759308E475F001E4
:203DE0001200B42480CD855083855182759308E0FEA3E0FF4E7010855083855182A3A37533
:203E00009308F0A3F08041C3EF9401FFEE9400FE855083855182A3A3759308E0FCA3E0D3C5
:203E20009FEE6480F8EC648098401D855083855182759308E0FFA3E0855083855182A3A33C
:203E4000759308CFF0A3EFF07E007F047D007B09900000041200B8B8A982AA831200BBFDD7
:203E6000900000651200B8B8E0FEA3E0FF900000621200B8B8E0FBA3E0FAA3E0F9C003C0A0
:203E800002C0017B09900000041200B8B8A982AA83A801AC02AD03D001D002D0031200B22C
:203EA000A17B09900000041200B8B8A982AA837D047C001205A5B2EFF47002EEF47043908A
:203EC0000000581200B8B8E030E134855083855182A3A3759308A3E0C4F8540FC868FF0507
:203EE00082D5820215831582E0C454F048FE74522FF58274683EF583759308E04402F02145
:203F000048AF7B09900000041200B8B8A982AA83C003C002C0017B099000000C1200B8B8D0
:203F2000A982AA839008A5B3EBF0A3EAF0A3E9F0D001D002D003120607547E007F047D00FE
:203F40007B09900000101200B8B8A982AA831200BBFD7B09900000101200B8B8A982AA839B
:203F6000C003C002C0017B099000000C1200B8B8A982AA83A801AC02AD03D001D002D00384
:203F80007E007F041200BB73EF7043900000581200B8B8E030E134855083855182A3A37544
:203FA0009308A3E0C4F8540FC868FF0582D5820215831582E0C454F048FE74522FF5827478
:203FC000683EF583759308E04402F02148AF855083855182A3A3759308E0FEA3E0FF7B099B
:203FE0009000000C1200B8B8A982AA8312046948EF4E7043900000581200B8B8E030E13405
:20400000855083855182A3A3759308A3E0C4F8540FC868FF0582D5820215831582E0C454C2
:20402000F048FE74522FF58274683EF583759308E04402F02148AF7B099000000C1200B824
:20404000B8A982AA83C001855083855182A3A3759308A3E0C4F8540FC868FF0582D58202D8
:2040600015831582E0C454F048FE744C2FF974683EA801FC7D09D0017E007F041200B2A17F
:20408000855083855182A3A3759308A3E0C4F8540FC868FF0582D5820215831582E0C45442
:2040A000F048FE74522FF58274683EF583759308E04402F074502FF58274683EF5837593A2
:2040C00008E0FEA3E064014E60032148BB855083855182A3A32142A1900000621200B8B8CF
:2040E000E0FBA3E0FAA3E0F91200B66B1200B84841120000000142E70000000242EA0000FC
:20410000000444EC00000005460500000006000042E7855083855182A3A3759308E0FEA365
:20412000E0FF900000381206CCAE900000471200B8B8E020E1032148AF85508385518275CC
:204140009308E4F0A3F0855083855182759308E0FEA3E0FFC39410EE6480948050777B09A5
:204160009000000C1200B8B8A982AA83C003C002C0017B09900000141200B8B8A982AA8381
:204180009008A27BEBF0A3EAF0A3E9F0D001D002D00312069131EF4E603B855083855182BE
:2041A000759308E0FEA3E0FF855083855182A3A3759308E0FCA3E0B50707ECB50603214755
:2041C000BE855083855182759308E475F0011200B424214146855083855182759308E0FCE9
:2041E000A3E0FDC39410EC6480948040032148AFEDC4F8540FC868FFECC454F048FE74436D
:204200002FF974683EFA7B09C003C001855083855182A3A3759308A3E0C4F8540FC868FF83
:204220000582D5820215831582E0C454F048FE74432FF974683EA801FCAD03D001D0037ED1
:20424000007F101200B2A1900000451200B8B8E4F0A304F07B09900000381200B8B8A982AF
:20426000AA83C001855083855182759308A3E0C4F8540FC868FF0582D5820215831582E0D0
:20428000C454F048FE74432FF974683EA801FC7D09D0017E007F101200B2A185508385513B
:2042A00082759308E0FEA3E0FFC006C4F8540FC868FDEEC454F048FC744C2DF974683CFAC8
:2042C0007B09C003C002C00174432DF974683CFA90088F1FEBF0A3EAF0A3E9F0D001D00268
:2042E000D003D0062144E52148AF855083855182759308E4F0A3F0855083855182759308CC
:20430000E0FEA3E0FFC39410EE6480948040032143AF7B099000000C1200B8B8A982AA83A0
:20432000C003C002C0017B09900000141200B8B8A982AA839008A27BEBF0A3EAF0A3E9F0AC
:20434000D001D002D00312069131EF4E701F855083855182759308E0FFA3E08550838551F1
:2043600082A3A3759308CFF0A3EFF08042855083855182A3A3759308E0FEA3E0C39401FFA4
:20438000EE9400FE855083855182759308E0FCA3E0B50707ECB506032148AF8550838551CB
:2043A00082759308E475F0011200B4242142F7855083855182759308E0FEA3E0C39410EE67
:2043C0006480948040032148B5855083855182759308E4F0A3F0C390087ED4E09401FF90AC
:2043E000087ED3E09400FE855083855182759308E0FCA3E0FDC39FEE6480F8EC64809850F2
:204400005FEDAE047803CEA2E713CE13D8F8FF9000000C1200B8B8E5822FF582E5833EF543
:2044200083C083C082759308E0FF855083855182759308A3E05407FE7401A806088002C379
:2044400033D8FC4F759308D082D083F0855083855182759308E475F0011200B4242143D633
:20446000855083855182A3A3759308E0FEA3E0FF7B099000000C1200B8B8A982AA831204C6
:204480006948EF4E70032148307E007F217D007B09900000171200B8B8A982AA831200BBB5
:2044A000FD855083855182A3A3759308E0FEA3E0FF7B099000000C1200B8B8A982AA83C0DF
:2044C00003C002C0017B09900000171200B8B8A982AA8390088F1FEBF0A3EAF0A3E9F0D067
:2044E00001D002D00312034A0A2148A9855083855182759308E4F0A3F0855083855182754F
:204500009308E0FEA3E0FFC39410EE64809480501B1206CCAAEF4E60138550838551827585
:204520009308E475F0011200B42480CD855083855182759308E0FEA3E0FF4E701085508319
:20454000855182A3A3759308F0A3F08046C3EF9401FFEE9400FE855083855182A3A37593A0
:2045600008E0FCA3E0D39FEE6480F8EC648098401F855083855182759308E0FFA3E08550DA
:2045800083855182A3A3759308CFF0A3EFF080032148AF7E007F107D007B09900000481216
:2045A00000B8B8A982AA831200BBFD900000551200B8B8E4F0A37403F07B099000004812B6
:2045C00000B8B8A982AA83C001855083855182A3A3759308A3E0C4F8540FC868FF0582D51F
:2045E000820215831582E0C454F048FE74432FF974683EA801FC7D09D0017E007F101200C6
:20460000B2A12148BB855083855182759308E4F0A3F0855083855182759308E0FEA3E0FFDC
:20462000C39410EE6480948050217B09900000381206CCB0EF4E6013855083855182759374
:2046400008E475F0011200B42480C7855083855182759308E0FCA3E0FD64014C700321482E
:2046600030ED4C7005FEFF2148BE855083855182759308E0FEA3E0C39401FFEE9400FE85BB
:204680005083855182A3A3759308E0FCA3E0FDD39FEE6480F8EC64809840032147BEEDC47F
:2046A000F8540FC868FFECC454F048FE74502FF58274683EF583759308E0FCA3E064034C18
:2046C000701FF583758210C083C082FD74432FF974683EFA7B09D007D0061200BBFD2148F3
:2046E000BB7E007F047D007B09900000081200B8B8A982AA831200BBFD855083855182759C
:204700009308E4F0A3F0855083855182759308E0FEA3E0FFC39410EE64809480400321477F
:20472000A77B099000000C1200B8B8A982AA83C003C002C0017B09900000141200B8B8A93F
:2047400082AA839008A27BEBF0A3EAF0A3E9F0D001D002D00312069131EF4E6036855083A6
:20476000855182759308E0FEA3E0FF855083855182A3A3759308E0FCA3E0B50716ECB50693
:2047800012855083855182A3A3759308EEF0A3EFF08014855083855182759308E475F00103
:2047A0001200B424214706855083855182759308E0FEA3E0C39410EE648094804003214887
:2047C000BB855083855182A3A3759308E0FEA3E07803CEA2E713CE13D8F8FF900000081278
:2047E00000B8B8E5822FF582E5833EF583C083C082759308E0FF855083855182A3A37593AC
:2048000008A3E05407FE7401A806088002C333D8FC4F759308D082D083F07B09900000082D
:204820001200B8B8A982AA8312059276EF4E7006FE7F032148BE7E007F107D007B09900087
:2048400000381200B8B8A982AA831200BBFD7B09900000381200B8B8A982AA83C0018550C0
:2048600083855182A3A3759308A3E0C4F8540FC868FF0582D5820215831582E0C454F048F7
:20488000FE74432FF974683EA801FC7D09D0017E007F101200B2A17B09900000081200B8CD
:2048A000B8A982AA831205C4C2120718DF800C7E007F0380097E007F028003E4FEFF900033
:2048C00000670200B8919000FFFD1200B891EBF0A3EAF0A3E9F09000FFA81200B891900049
:2048E00000061200B8B8E4F0A3F09000005E1200B8B8E0FBA3E0FAA3E0F91200B450FDACC6
:20490000F0C3940DEC64809480500321546B9000005B1200B8B8E0FBA3E0FAA3E0F9C00328
:20492000C002C001C3ED9401FDEC9400FC900000581200B8B8E0F9A3E0FAA3E090089F19A3
:20494000C9F0A3EAF0A3E9F0900000581200B8B8E0FBA3E0FAA3E02434F9E43AFA1200B431
:2049600050C39401FEE5F0940090089F1CF0A3CEF0D001D002D0031206054BEF4E600321E5
:20498000546B7C007D029000005E1200B8B8E0FBA3E0FAA3E0F91200B45025E0FFE5F033F7
:2049A000FE9000005B1200B8B8E0FBA3E0FAA3E02FF9EA3EFAC3E99DF9EA9CFA1200B4508F
:2049C000FFAEF0855083855182759308EEF0A3EFF0855083855182759308E0FEA3E0FFC337
:2049E0009401EE64809480400BD3EF9414EE64809480400321546B855083855182759308BE
:204A000074FFF5F01200B4247B09900000381200B8B8A982AA83855083855182759308E08E
:204A2000FCA3E0FD1207165C900000581200B8B8E0FBA3E0FAA3E02437F9E43AFA1200B4F8
:204A400050FFAEF0E5F0600321546BEF24FD7003214E5F147003214FA91470032151D22471
:204A600003600321546B855083855182759308E0FEA3E0FF9008704875F00C1200B774EEE4
:204A800075F00CA42583F583759308E0FD9000004D1200B8B8EDF09008704875F00CEF12F6
:204AA00000B774EE75F00CA42583F583759308ED54FDF09000004D1200B8B8E030E128856D
:204AC0005083855182759308E0FEA3E09008704875F00C1200B774EE75F00CA42583F58319
:204AE000759308E04402F0900000641200B8B8E0FEA3E064114E6003214CE3FE7F12FD7B3C
:204B0000099000000E1200B8B8A982AA831200BBFD900000641200B8B8E0FEA3E0FF9000E4
:204B200000611200B8B8E0FBA3E0FAA3E0F9C003C002C0017B099000000E1200B8B8A982A9
:204B4000AA83A801AC02AD03D001D002D0031200B2A17B099000000E1200B8B8A982AA834A
:204B600012058B687B099000000E1200B8B8A982AA8312060220EF4E7003215292900000B0
:204B8000041200B8B8E4F0A3F0855083855182A3A3759308F0A3F07B099000000E1200B8B3
:204BA000B8A982AA831200CB03855083855182A3A3759308E0FCA3E0C39FEE6480F8EC6424
:204BC00080985069855083855182A3A3759308A3E0FF9000000E1200B8B8E5822FF582E46B
:204BE0003583F583759308E0FF643A602A900000041200B8B8E475F0011200B43AADF0FC75
:204C0000900000201200B8B8E5822DF582E5833CF583759308EFF0855083855182A3A375E1
:204C20009308E475F0011200B424214B97900000041200B8B8A3E0FF900000201200B8B8D8
:204C4000E5822FF582E43583F583759308E4F07B09900000201200B8B8A982AA83C003C0BE
:204C600002C0017B09900000081200B8B8A982AA839008A3DDEBF0A3EAF0A3E9F0D001D0EE
:204C800002D0031206E021855083855182759308E0FEA3E09008704475F00C1200B774EE1D
:204CA00075F00CA42583F583759308E0FCA3E0FD7B09900000081200B8B8A982AA83120645
:204CC000D27FEF60032154657B09900000081200B8B8A982AA8312071D07EF7003214D99BB
:204CE000215465900000641200B8B8E0FEA3E064064E6003214D96FE7F06FD7B0990000050
:204D0000321200B8B8A982AA831200BBFD900000641200B8B8E0FEA3E0FF900000611200E4
:204D2000B8B8E0FBA3E0FAA3E0F9C003C002C0017B09900000081200B8B8A982AA83A8014A
:204D4000AC02AD03D001D002D0031200B2A1900000081200B8B8E020E0397B0990000032A1
:204D60001200B8B8A982AA83C003C002C0017B09900000081200B8B8A982AA83A801AC02C6
:204D8000AD03D001D002D0037E007F061200BB73EF70062154652154657B09900000081263
:204DA00000B8B8A982AA83C001855083855182759308E0FEA3E0FF7C007D0C1200B3847488
:204DC0003D2FF974703EA801FC7D09D0017E007F061200B2A1855083855182759308E0FE4A
:204DE000A3E0FF9008704875F00C1200B774EE75F00CA42583F583759308E04402F0900852
:204E0000704675F00CEF1200B774EE75F00CA42583F583759308E0FEA3E064014E60032174
:204E20005471855083855182759308A3E0FF1206FCD7855083855182759308E0FEA3E0FF60
:204E40007C007D0C1200B384743D2FF974703EFA7B091205F7ADEF600321545F2152928520
:204E60005083855182759308E0FEA3E0FF9008704875F00C1200B774EE75F00CA42583F5F9
:204E800083759308E0FD9000004D1200B8B8EDF09008704875F00CEF1200B774EE75F00C1A
:204EA000A42583F583759308ED54FEF0900000611200B8B8E0FBA3E0FAA3E0F91200B66B75
:204EC000E47B01FAF9F8D31200B6345021900000611200B8B8E0FBA3E0FAA3E0F91200B638
:204EE0006BE47B10FAF9F8C31200B6345003215465900000611200B8B8E0FBA3E0FAA3E0B3
:204F0000F91200B66B855083855182759308E0FCA3E0FD9008704375F00C1200B774EC75EF
:204F2000F00CA42583F583759308EFF09008704875F00CED1200B774EC75F00CA42583F539
:204F400083759308E04401F09008704675F00CED1200B774EC75F00CA42583F5837593088F
:204F6000E0FEA3E064014E6003215471855083855182759308A3E0FF1206FCD785508385CA
:204F80005182759308E0FEA3E0FF7C007D0C1200B384743D2FF974703EFA7B091205F7AD4C
:204FA000EF700321529221545F855083855182759308E0FEA3E0FF9008704875F00C1200C3
:204FC000B774EE75F00CA42583F583759308E0FD9000004D1200B8B8EDF09008704875F0A5
:204FE0000CEF1200B774EE75F00CA42583F583759308ED54FBF0900000611200B8B8E0FBCC
:20500000A3E0FAA3E0F91200B66BE47B01FAF9F8D31200B6345022900000611200B8B8E085
:20502000FBA3E0FAA3E0F91200B66BE47BFE7A0FF9F8C31200B634500321546512073B69C9
:20504000EF4E60032150CA900000041200B8B8E4F0A3F0900000041200B8B8E0FEA3E0FF82
:20506000C39440EE6480948050607B099000004E1200B8B8A982AA831206F578EF4E604A5B
:20508000900000611200B8B8E0FBA3E0FAA3E0F91200B6D09000004E1200B8B8E0FEA3E070
:2050A000FFE4FCFDC31200B634700D900000061200B8B8E4F0A304F0900000041200B8B83F
:2050C000E475F0011200B424808912073B69EF64014E7031900000611200B8B8E0FBA3E0C2
:2050E000FAA3E0F91200B66BE47B01FAF9F8C31200B6346003215465900000061200B8B8A8
:20510000E4F0A304F0900000061200B8B8E0FEA3E04E7003215292900000611200B8B8E092
:20512000FBA3E0FAA3E0F91200B66B855083855182759308E0FCA3E0FD9008704475F00C6F
:205140001200B774EC75F00CA42583F583759308EEF0A3EFF09008704875F00CED1200B70A
:2051600074EC75F00CA42583F583759308E04404F09008704675F00CED1200B774EC75F038
:205180000CA42583F583759308E0FEA3E064014E6003215471855083855182759308A3E08F
:2051A000FF1206FCD7855083855182759308E0FEA3E0FF7C007D0C1200B384743D2FF9744A
:2051C000703EFA7B091205F7ADEF700321529221545F900000611200B8B8E0FBA3E0FAA33F
:2051E000E0F91200B66B1200B848520C00000001529B00000002529B00000004529E000062
:2052000000055331000000060000529B1206C9F79000004C1200B8B8E054076407600321B2
:2052200054659000004A1200B8B8E4F0A304F07B09900000411200B8B8A982AA83C0018579
:205240005083855182759308E0FEA3E0FF7C007D0C1200B384743D2FF974703EA801FC7D48
:2052600009D0017E007F0C1200B2A1855083855182759308E0FEA3E0FF7C007D0C1200B3FC
:2052800084743D2FF974703EFA7B091205F7ADEF7006FE7F0321547421545F2154651206C2
:2052A000C9F7EF4E60032154657E007F0C7D007B09900000411200B8B8A982AA831200BB32
:2052C000FD12073B69EF64014E7019900000481200B8B8E4F0A304F09000004C1200B8B8C6
:2052E000E04404F09000004A1200B8B8E4F0A37403F07B09900000411200B8B8A982AA832D
:20530000C001855083855182759308E0FEA3E0FF7C007D0C1200B384743D2FF974703EA8BB
:2053200001FC7D09D0017E007F0C1200B2A1215471855083855182759308E0FEA3E0FF9015
:2053400008704675F00C1200B774EE75F00CA42583F583759308E0FCA3E04C7002802E855E
:205360005083855182759308E0FEA3E0FF9008704675F00C1200B774EE75F00CA42583F5F6
:2053800083759308E0FCA3E064034C702AF58375820CC083C082FDC005FC7D0C1200B3843E
:2053A000743D2FF974703EFA7B09D005D007D0061200BBFD21547185508385518275930882
:2053C000E0FEA3E09008704675F00C1200B774EE75F00CA42583F583759308E0FEA3E06478
:2053E000014E6003215465FE7F0CFD7B09900000411200B8B8A982AA831200BBFD90000012
:205400004A1200B8B8E4F0A3F09000004C1200B8B8E4F07B09900000411200B8B8A982AA7B
:2054200083C001855083855182759308E0FEA3E0FF7C007D0C1200B384743D2FF974703EBF
:20544000A801FC7D09D0017E007F0C1200B2A1855083855182759308A3E0FF1206FCD712A3
:205460000718DF800C7E007F0380097E007F028003E4FEFF900000660200B891900851FB91
:20548000EBF0A3EAF0A3E9F07E007FF07D007B097A5179FE1200BBFD7E007FF07D007B0950
:2054A0007A5279EE1200BBFD90088B077481F0A37488F0A37470F07B097A5379E612008C8C
:2054C0003374FF9008541AF0A3F0E49008540EF0A3F09008540EE0FEA3E0FFC39404EE6435
:2054E000809480502A7C007D3C1200B38474EE2FF974523EFA7B09E0FD12071B38900854DF
:205500000FE004F070CC9008540EE004F080C3900851FBE0F9A3E0FAA3E090085408C9F0F1
:20552000A3EAF0A3E9F0E49008540EF0A3F09008540EE0FAA3E0FBC39404EA648094804042
:2055400003215EA0E49008541CF0A3F0FFFEFDFC900854261200B7577C007D3CAF03AE02FB
:205560001200B38474FE2FF974513EFA7B09C002C00174EE2FF974523EFA90088B07740915
:20558000F0A3EAF0A3E9F0D001D00212008C33E490085410F0A3F090088B077481F0A37425
:2055A00088F0A37470F07B097A5379DE12008C339008A0737481F0A37483F0A37404F090CE
:2055C0000851FBE0FBA3E0FAA3E0F912065EEB90085408EBF0A3EAF0A3E9F09008950574D4
:2055E00081F0A37483F0A37404F0A37481F0A37481F0A37490F0A37409F0A37453F0A3747D
:20560000DEF0120585CB78DE7C537D097B097A5379E61200B995EF702290085411E025E037
:20562000FF90085410E033FE74122FF58274543EF583759308E4F0A3F0802F7B097A5379C4
:20564000DE120630DBAC06AD0790085411E025E0FF90085410E033FE74122FF58274543EC3
:20566000F583759308ECF0A3EDF090085409E475F0031200B42490085408E0F9A3E0FAA32E
:20568000E0900851FBC9F0A3EAF0A3E9F090085411E004F0700790085410E004F0C3900821
:2056A0005411E0940490085410E064809480500321559790085412E07002A3E060519008BD
:2056C000540EE0FEA3E0FF7C007D3C1200B38474132FF974523EFA90089EE77409F0A3EAC6
:2056E000F0A3E9F07B097A547912120551ABEF4E70459008A3CB7481F0A37488F0A3747E4D
:20570000F0A37481F0A37488F0A37494215F8BE4FFFEFDFC9008540EE0FAA3E0900852139E
:2057200075F03C1200B774EA75F03CA42583F5837593081200B75790088B077481F0A374E6
:2057400088F0A374A5F09008540EE0FFA3E090088B0ACFF0A3EFF07B097A5379EA12008C09
:20576000339008A0737409F0A37453F0A374EAF090085408E0FBA3E0FAA3E0F912065EEB6A
:2057800090085408EBF0A3EAF0A3E9F0C002C001900895057409F0A37453F0A374EAF0A331
:2057A0007481F0A37481F0A37490F09008540EE0FEA3E0FF7C007D3C1200B38474172FF95A
:2057C00074523EFA9008950B7409F0A3EAF0A3E9F0D001D002120585CB9008540EE0FEA3A8
:2057E000E0FF7C007D3C1200B38474172FF974523EFA90088B077409F0A3EAF0A3E9F07B90
:20580000097A5379EA12008C337B097A5379EA12058B687B097A5379EA1200CB03D3EF94D6
:2058200014EE64809480403D90088B077481F0A37488F0A374ADF0A3E4F0A37414F07B0989
:205840007A54792A12008C339008A3CB7409F0A37454F0A3742AF0A37481F0A37488F0A34D
:2058600074D4215F8B90088B077481F0A37488F0A374DDF09008540EE0FFA3E090088B0ACA
:20588000CFF0A3EFF07B097A5379EA12008C339008A0737409F0A37453F0A374EAF0900847
:2058A0005408E0FBA3E0FAA3E0F912065EEB90085408EBF0A3EAF0A3E9F0900895057409E0
:2058C000F0A37453F0A374EAF0A37481F0A37481F0A37490F0A37409F0A37454F0A3741E46
:2058E000F0120585CB781E7C547D097B817A8879E41200B995EF9008540E701FE0FEA3E0D1
:205900009008522C75F03C1200B774EE75F03CA42583F583759308E4F0801EE0FEA3E090CD
:2059200008522C75F03C1200B774EE75F03CA42583F5837593087401F09008540EE07002EF
:20594000A3E06003215A3D90085408E0F9A3E0FAA3E0A3C9F0A3EAF0A3E9F09008A0737468
:2059600081F0A37488F0A374E6F0900851FBE0FBA3E0FAA3E0F912065EEB9008540BEBF04F
:20598000A3EAF0A3E9F09008540BE0FBA3E0FAA3E04A4B7003215A3D9008A0737481F0A349
:2059A0007488F0A374EDF0900851FBE0FBA3E0FAA3E0F912065EEBC003C002C001900854BC
:2059C0000BA3E0FAA3E0F9D3D082D083D0E0E99582EA958340249008A0737481F0A3748806
:2059E000F0A374EDF0900851FBE0FBA3E0FAA3E0F912065EEBE94A4B7043900889D874818B
:205A0000F0A37488F0A374F3F0A37409F0A37454F0A3741AF09008540BE0FBA3E0FAA3E0AF
:205A2000F91200BD8B7B817A8879E61200CB03900851FCEE8FF01200B42421595B900854D9
:205A400008E0F9A3E0FAA3E0900851FBC9F0A3EAF0A3E9F07B817A8879FC9008540EE0FF83
:205A6000A3E090088B07CFF0A3EFF09008541AE0FFA3E090088B09CFF0A3EFF012008C398C
:205A80009008541AE0F47003A3E0F46019E47F01FEFDFC9008541BE0F9F81200B6589008DE
:205AA00054261200B75790085408E0F9A3E0FAA3E0A3C9F0A3EAF0A3E9F090088B0774810B
:205AC000F0A37489F0A3740CF09008540EE0FFA3E090088B0ACFF0A3EFF07B097A5379EAB5
:205AE00012008C339008A0737409F0A37453F0A374EAF0900851FBE0FBA3E0FAA3E0F912A8
:205B0000065EEB90085408EBF0A3EAF0A3E9F090085408E0FBA3E0FAA3E04A4B7003215C1A
:205B20003B9008A0737481F0A37488F0A374EDF0900851FBE0FBA3E0FAA3E0F912065EEBFE
:205B4000C003C002C00190085408A3E0FAA3E0F9D3D082D083D0E0E99582EA9583402790F1
:205B600008A0737481F0A37488F0A374EDF0900851FBE0FBA3E0FAA3E0F912065EEBE94A56
:205B80004B6003215C3B90088B077481F0A37489F0A37412F0A37409F0A37453F0A374EA7C
:205BA000F07B097A5379DE12008C33900889D87409F0A37453F0A374DEF0A37409F0A374B0
:205BC00054F0A3741CF090085408E0FBA3E0FAA3E0F91200BD8B90085426E0F8A3E0F9A333
:205BE000E0FAA3E0FBC000C001E47F01FEFDFC9008541DE0F9F81200B658D001D000EB4F9C
:205C0000FFEA4EFEE94DFDE84CFC900854261200B7577B097A5379EA1200CB039008540832
:205C2000E0FBA3E0FAA3E02FF9EA3EFA900851FBEBF0A3EAF0A3E9F0215AE49008540BE051
:205C4000F9A3E0FAA3E0900851FBC9F0A3EAF0A3E9F09008540BE0F9A3A3E090085408C902
:205C6000F0A3EAF0A3E9F090085426E0FCA3E0FDA3E0FEA3E0FF9008540EE0FAA3E09008DB
:205C8000522D75F03C1200B774EA75F03CA42583F5837593081200B75790085426A3A3A32D
:205CA000E05404FFE4FEFDFC7B04FAF9F8C31200B6349008540E7073E0FAA3E0FB90085389
:205CC0002575F03C1200B774EA75F03CA42583F583759308E0FCA3E0FDA3E0FEA3E04402BC
:205CE000FF9008523575F03CEB1200B774EA75F03CA42583F5837593081200B75790085452
:205D00000EE0FAA3E0FB9008532175F03C1200B774EA75F03CA42583F583759308E0FCA355
:205D2000E0FDA3E0FEA3E044018071E0FAA3E0FB9008532575F03C1200B774EA75F03CA4D7
:205D40002583F583759308E0FCA3E0FDA3E0FEA3E054FDFF9008523575F03CEB1200B7747B
:205D6000EA75F03CA42583F5837593081200B7579008540EE0FAA3E0FB9008532175F03CA5
:205D80001200B774EA75F03CA42583F583759308E0FCA3E0FDA3E0FEA3E054FEFF900852CC
:205DA0003175F03CEB1200B774EA75F03CA42583F5837593081200B75790088B077481F05B
:205DC000A37489F0A37418F09008540EE0FFA3E090088B0ACFF0A3EFF07B097A5379EA1284
:205DE000008C339008A0737409F0A37453F0A374EAF090085408E0FBA3E0FAA3E0F91206A1
:205E00005EEB90085408EBF0A3EAF0A3E9F0900895057409F0A37453F0A374EAF0A37481EF
:205E2000F0A37481F0A37490F0A37409F0A37454F0A37422F0120585CB78227C547D097BED
:205E4000817A8879E41200B995EF9008540E7020E0FEA3E09008523975F03C1200B774EE39
:205E600075F03CA42583F5837593087401F0801DE0FEA3E09008523975F03C1200B774EE5B
:205E800075F03CA42583F583759308E4F09008540FE004F070079008540EE004F021552E01
:205EA000E49008540EF0A3F09008540EE0FEA3E0FFC39404EE648094804003215FC09008CB
:205EC000521375F03CEF1200B774EE75F03CA42583F583759308E0FCA3E0FDA3E0FEA3E0CD
:205EE000FFE4FBFAF9F8C31200B6347003215FAD9008540FE02401FE9008540EE0340090DE
:205F0000085410F0A3CEF090085410E0FEA3E0FFC39404EE648094804003215FAD900852CD
:205F20001375F03CEF1200B774EE75F03CA42583F583759308E0FCA3E0FDA3E0FEA3E0FFBF
:205F40009008540EE0FAA3E09008521375F03C1200B774EA75F03CA42583F583759308E0D0
:205F6000F8A3E0F9A3E0FAA3E0FBC31200B63470299008A3CB7481F0A37489F0A37421F0B7
:205F8000A37481F0A37488F0A374D4F07B817A8879711206A215E4FEFF2290085411E00474
:205FA000F0700790085410E004F0215F079008540FE004F070079008540EE004F0215EA8E8
:205FC000E49008540EF0A3F09008540EE0FEA3E0FFC39404EE64809480502A7C007D3C1204
:205FE00000B38474FE2FF974513EFA7B09E0FD1207260D9008540FE004F070CC9008540E21
:20600000E004F080C3120718DF7E007F0122E0FBA3E0FAA3E0F97E007F009000FFFD1200CA
:20602000B891EBF0A3EAF0A3E9F09000FFFE1200B891EEF0A3EFF09000FFEF1200B8919092
:2060400000000B1200B8B8E4F0A3F0900000191200B8B8E0FBA3E0FAA3E04A4B701690009B
:2060600000161200B8B8E0FBA3E0FAA3E0F91200B7808010900000191200B8B8E0FBA3E052
:20608000FAA3E0F9900000191200B8B8EBF0A3EAF0A3E9F07B097A98794A9000000312008D
:2060A000B8B8EBF0A3EAF0A3E9F0900000161200B8B8E0FBA3E0FAA3E024072161D1855046
:2060C00083855182759308E0FBA3E0FAA3E0F9EB8A8389827B097A98794A6409700A744A00
:2060E000658270047498658370032161FD9000000B1200B8B8E0FEA3E04E60032161FD852C
:206100005083855182759308E0FBA3E0FAA3E0F9900000031200B8B8EBF0A3EAF0A3E9F087
:20612000855083855182759308E0FBA3E0FAA3E0240BF9E43AFA1200B7809000FFFD12009D
:20614000B891EBF0A3EAF0A3E9F0900000161200B8B8E0FBA3E0FAA3E0F9C003C002C001E0
:206160009000001C1200B8B8E0FBA3E0FAA3E0F5828A838B93D001D002D0031200B88A901A
:206180000000091200B8B8EEF0A3EFF0900000091200B8B8E0FEA3E0FFC3EE6480948050A0
:2061A00013855083855182759308E0FBA3E0FAA3E0F98021D3EF9400EE64809480402E8568
:2061C0005083855182759308E0FBA3E0FAA3E02403F9E43AFA1200B7808550838551827503
:2061E0009308EBF0A3EAF0A3E9F02160BE9000000B1200B8B8E4F0A304F02160BE9000009A
:206200000B1200B8B8E0FEA3E04E6011900000111200B8B8E0FEA3E04E6002807B90000012
:20622000111200B8B8E0FEA3E04E700C855083855182759308216A9A900000161200B8B893
:20624000E0FBA3E0FAA3E02405F9E43AFA1200B450FFAEF0EE3395E0FDFC7B0990000006CD
:206260001200B8B8A982AA83120711F99000000D1200B8B81200B75774FFFFFEFDFC9000E9
:20628000000D1200B8B8E0F8A3E0F9A3E0FAA3E0FBC31200B63470097B097A98794A216A04
:2062A000A2900000131200B8B8E0FBA3E0FAA3E0F9C003C002C001900000061200B8B8E005
:2062C000FBA3E0FAA3E0240BF9E43AFA1200B79D900000031200B8B8E0FBA3E0FAA3E0F934
:2062E000C003C002C001900000061200B8B8E0FBA3E0FAA3E02406F9E43AFA1200B79D9034
:206300000000031200B8B8E0FBA3E0FAA3E0F9EB8A8389827B097A98794A6409700A744A23
:206320006582700474986583702E900000061200B8B8E0FBA3E0FAA3E0F9C003C002C0013E
:20634000900000161200B8B8E0FBA3E0FAA3E02407F9E43AFA21642D900000031200B8B837
:20636000E0FBA3E0FAA3E0240BF9E43AFA1200B7809000FFFD1200B891EBF0A3EAF0A3E9EE
:20638000F0900000091200B8B8E0FBA3E0FAA3E0240BF9E43AFA1200B780C003C002C00148
:2063A0009000001C1200B8B8E0FBA3E0FAA3E0F5828A838B93D001D002D0031200B88A90D8
:2063C0000000091200B8B8EEF0A3EFF0900000091200B8B8E0FEC3EE64809480900000069A
:2063E00050241200B8B8E0FBA3E0FAA3E0F9C003C002C001900000031200B8B8E0FBA3E01A
:20640000FAA3E0F980271200B8B8E0FBA3E0FAA3E0F9C003C002C001900000031200B8B8AE
:20642000E0FBA3E0FAA3E02403F9E43AFA1200B79D7B097A98794AC003C002C001900000B4
:20644000061200B8B8E0FBA3E0FAA3E0F91200B79D7B097A98794AC003C002C0019000004B
:20646000061200B8B8E0FBA3E0FAA3E02403F9E43AFA1200B79D900000061200B8B8E0FB28
:20648000A3E0FAA3E02409F9E43AFAE475F0011200B4CA900000061200B8B8E0F9A3E0FA76
:2064A000A3E0855083855182759308C92168FC900000161200B8B8E0FBA3E0FAA3E024071D
:2064C000F9E43AFA1200B780C003C002C001855083855182759308E0FBA3E0FAA3E0F9D0B8
:2064E00082D083D0E06B7008E965827003EA65837003216A6B855083855182759308E0FB1B
:20650000A3E0FAA3E02406F9E43AFA1200B780E92409F9E43AFA1200B450640145F06003BD
:20652000216A6B855083855182759308E0FBA3E0FAA3E02406F9E43AFA1200B780E9240633
:20654000F9E43AFA1200B7801200B780C003C002C001855083855182759308E0FBA3E0FA3A
:20656000A3E02406F9E43AFA1200B780D082D083D0E06B7008E965827003EA658360032143
:2065800067FA855083855182759308E0FBA3E0FAA3E02406F9E43AFA1200B780E92406F96F
:2065A000E43AFA1200B780E92403F9E43AFA1200B780900000031200B8B8EBF0A3EAF0A300
:2065C000E9F0900000031200B8B8E0FBA3E0FAA3E02409F9E43AFA1200B450640145F060A4
:2065E0000321668E855083855182759308E0FBA3E0FAA3E02406F9E43AFA1200B780E92457
:2066000009F9E43AFAE4F5F01200B4CA900000031200B8B8E0FBA3E0FAA3E02409F9E43AD3
:20662000FAE4F5F01200B4CA855083855182759308E0FBA3E0FAA3E02406F9E43AFA12001F
:20664000B780E92406F9E43AFA1200B780E92409F9E43AFAE475F0011200B4CA85508385B8
:206660005182759308E0FBA3E0FAA3E02406F9E43AFA1200B780E92406F9E43AFA1200B7EB
:2066800080855083855182759308EB2168FC855083855182759308E0FBA3E0FAA3E0240685
:2066A000F9E43AFA1200B780E92403F9E43AFA1200B780C003C002C00185508385518275AB
:2066C0009308E0FBA3E0FAA3E0F9D082D083D0E06B7008E965827003EA65837068855083CE
:2066E000855182759308E0FBA3E0FAA3E02406F9E43AFA1200B78085508385518275930813
:20670000EBF0A3EAF0A3E9F0900000161200B8B8E0FBA3E0FAA3E02407F9E43AFAC002C0E4
:2067200001855083855182759308E0F9A3E0FAA3E09008A488C9F0A3EAF0A3E9F0D001D0A8
:20674000021204C618855083855182759308E0FBA3E0FAA3E02406F9E43AFA1200B780E93B
:206760002409F9E43AFAE4F5F01200B4CA855083855182759308E0FBA3E0FAA3E02406F9C4
:20678000E43AFA1200B780E92406F9E43AFA1200B780E92409F9E43AFAE475F0011200B4F4
:2067A000CA900000161200B8B8E0FBA3E0FAA3E02407F9E43AFAC003C002C00185508385AD
:2067C0005182759308E0FBA3E0FAA3E02406F9E43AFA1200B780E92406F9E43AFA1200B78A
:2067E000809008A491EBF0A3EAF0A3E9F0D001D002D0031204BB612164AF855083855182EC
:20680000759308E0FBA3E0FAA3E02406F9E43AFA1200B780E92406F9E43AFA1200B780128A
:2068200000B780900000031200B8B8EBF0A3EAF0A3E9F0900000031200B8B8E0FBA3E0FACB
:20684000A3E02409F9E43AFA1200B450640145F06003216906855083855182759308E0FB39
:20686000A3E0FAA3E02406F9E43AFA1200B780E92409F9E43AFAE4F5F01200B4CA90000084
:20688000031200B8B8E0FBA3E0FAA3E02409F9E43AFAE4F5F01200B4CA85508385518275DC
:2068A0009308E0FBA3E0FAA3E02406F9E43AFA1200B780E92406F9E43AFA1200B780E92464
:2068C00009F9E43AFAE475F0011200B4CA855083855182759308E0FBA3E0FAA3E02406F906
:2068E000E43AFA1200B780E92406F9E43AFA1200B780855083855182759308EBF0A3EAF0B2
:20690000A3E9F02164AF855083855182759308E0FBA3E0FAA3E02406F9E43AFA1200B780A8
:206920001200B780C003C002C001855083855182759308E0FBA3E0FAA3E0F9D082D083D0BF
:20694000E06B7008E965827003EA65837068855083855182759308E0FBA3E0FAA3E02406C2
:20696000F9E43AFA1200B780855083855182759308EBF0A3EAF0A3E9F0900000161200B8B9
:20698000B8E0FBA3E0FAA3E02407F9E43AFAC002C001855083855182759308E0F9A3E0FA8F
:2069A000A3E09008A491C9F0A3EAF0A3E9F0D001D0021204BB61855083855182759308E060
:2069C000FBA3E0FAA3E02406F9E43AFA1200B780E92409F9E43AFAE4F5F01200B4CA8550E3
:2069E00083855182759308E0FBA3E0FAA3E02406F9E43AFA1200B780E92406F9E43AFA1217
:206A000000B780E92409F9E43AFAE475F0011200B4CA900000161200B8B8E0FBA3E0FAA31B
:206A2000E02407F9E43AFAC003C002C001855083855182759308E0FBA3E0FAA3E02406F936
:206A4000E43AFA1200B780E92406F9E43AFA1200B7809008A488EBF0A3EAF0A3E9F0D001FF
:206A6000D002D0031204C6182164AF900000161200B8B8E0FBA3E0FAA3E02407F9E43AFA0A
:206A80001200B780E92409F9E43AFAE4F5F01200B4CA900000061200B8B8E0FBA3E0FAA31A
:206AA000E0F99000001C0200B89112073B27EF4E7003FEFF2290083666E025E0FF900836D6
:206AC00065E033FE74B32FF58274333EF583759308E0FFA3E090087ADDCFF0A3EFF09008DC
:206AE00031D8E0FEA3E0FFC390087ADEE09F90087ADDE09E4003217527E0FFA3E090087A1A
:206B0000E1CFF0A3EFF07E007F647D007B097A7A79E91200BBFD7B097A44794290084544B3
:206B2000EBF0A3EAF0A3E9F02414F9E43AFA74111200B37090084544E0FBA3E0FAA3E0F989
:206B4000740475F0001200B4CA90084544E0FBA3E0FAA3E02402F9E43AFAE475F0A2120098
:206B6000B4CA90084544E0FBA3E0FAA3E0242AF9E43AFAE41200B370120646E1900841D536
:206B8000E0FBA3E0FAA3E02408F9E43AFA90087B4DEBF0A3EAF0A3E9F090087ADDE475F071
:206BA000011200B43AFEE5F025E0FFEE33FE74CD2FF58274333EF583759308E0FFA3E09098
:206BC000087AE3CFF0A3EFF0E4FFFEFDFC90087B5C1200B75790087AE3E0FEA3E0FFC394FA
:206BE000D0EE648094874003216E8EEF64EA7003EE6403705590087ADEE025E0FF90087AC8
:206C0000DDE033FE74CD2FF58274333EF583759308E0FCA3E0FDA3E0FEA3E0FF90087B6060
:206C20001200B75790087ADEE02402F090087ADDE03400F0C390087AE4E094E8FF90087A35
:206C4000E3E09403CFC39401806590087AE3E064037004A3E064ED6003216D8190087ADEE8
:206C6000E025E0FF90087ADDE033FE74CD2FF58274333EF583759308E0FCA3E0FDA3E0FEFF
:206C8000A3E0FF90087B601200B75790087ADEE02402F090087ADDE03400F0C390087AE44D
:206CA000E094E8FF90087AE3E09403CFC39403CF9400FE900833AA75F003EF1200B774EE8C
:206CC00075F003A42583F583759308E0F9A3E0FAA3E090088B07C9F0A3EAF0A3E9F090082B
:206CE0007B60E0FCA3E0FDA3E0FEA3E0FF78181200B645E490088B0AF0A3EFF090087B60C7
:206D0000E0FCA3E0FDA3E0FEA3E0FF78101200B645E490088B0CF0A3EFF090087B60E0FCAB
:206D2000A3E0FDA3E0FEA3E0FF78081200B645E490088B0EF0A3EFF090087B60E0FCA3E0EA
:206D4000FDA3A3E0FEE490088B10F0A3CEF07B097A7A79E912008C3390087AE5EEF0A3EF98
:206D6000F078587C7B7D097B097A3279A67E007F041200B2A190087B52E4F0A3740421703C
:206D80002D90087AE3E064037004A3E064EB7075C390087AE4E094E8FF90087AE3E09403DF
:206DA000CFC39403CF9400FE900833AA75F003EF1200B774EE75F003A42583F58375930816
:206DC000E0F9A3E0FAA3E090088B07C9F0A3EAF0A3E9F07B097A7A79E912008C3390087A41
:206DE000E5EEF0A3EFF078587C7B7D097B097A3279AC7E007F041200B2A1E490087B52F00D
:206E0000A3F02171F290087AE3E064037004A3E064EC600321726DC390087AE4E094E8FF61
:206E200090087AE3E09403CFC39404CF9400FE900833AA75F003EF1200B774EE75F003A458
:206E40002583F583759308E0F9A3E0FAA3E090088B07C9F0A3EAF0A3E9F07B097A7A79E973
:206E600012008C3390087AE5EEF0A3EFF078587C7B7D097B097A3379C77E007F041200B267
:206E8000A190087B52E4F0A304F0E42171F290087AE3E0FEA3E0FFC394B8EE6480948B4084
:206EA000032170A3C3EF94D0FFEE9407CFC39401CF9400FE9008359575F003EF1200B7747F
:206EC000EE75F003A42583F583759308E0F9A3E0FAA3E090088B07C9F0A3EAF0A3E9F09043
:206EE000087ADEE025E0FF90087ADDE033FE74CD2FF58274333EF583759308E0FFA3E09008
:206F0000088B0ACFF0A3EFF07B097A7A79E912008C3390087AE5EEF0A3EFF090087B52E448
:206F2000F0A37406F090087AE3E0FEA3E08EF01200B8196F4F07D16F6D07D26FD307D370C6
:206F40003807D46F8F07D56FAF07D60000726D78587C7B7D097B097A3179DA7E007F041288
:206F600000B2A190087B54E4F0A304801D78587C7B7D097B097A3179707E007F041200B215
:206F8000A190087B54E4F0A37402F0E42171F678587C7B7D097B097A3379BB7E007F0412DB
:206FA00000B2A190087B54E4F0A3740321718F78587C7B7D097B097A3379BF7E007F04123F
:206FC00000B2A190087B54E4F0A37404F0E47F0821726290087ADEE025E0FF90087ADDE015
:206FE00033FE74CD2FF58274333EF583759308E0FFA3E090087B56CFF0A3EFF090087ADE10
:20700000E004F0700790087ADDE004F012072E0378587C7B7D097B097A36794D7E007F04D0
:207020001200B2A190087B52E4F0A37403F0E4A3F0A3F07F0221726290087ADEE025E0FF54
:2070400090087ADDE033FE74CD2FF58274333EF583759308E0FFA3E090087B56CFF0A3EFC0
:20706000F090087ADEE004F0700790087ADDE004F07B097A3279B012072E0978587C7B7D35
:20708000097B097A3379C37E007F041200B2A190087B52E4F0A37402F0E4A3F0A3F07F0247
:2070A000217262C390087AE4E094B8FF90087AE3E0940BCFC39401CF9400FE9008363D757B
:2070C000F003EF1200B774EE75F003A42583F583759308E0F9A3E0FAA3E090088B07C9F0AB
:2070E000A3EAF0A3E9F090087ADEE025E0FF90087ADDE033FE74CD2FF58274333EF583750A
:207100009308E0FFA3E090088B0ACFF0A3EFF07B097A7A79E912008C3390087AE5EEF0A3E1
:20712000EFF090087B52E4F0A37406F090087AE3E0FEA3E08EF01200B819714E0BB971720D
:207140000BBA71960BBB71FA0BBC0000726D78587C7B7D097B097A3379BB7E007F041200C7
:20716000B2A190087B54E4F0A37405F0E47F0221726278587C7B7D097B097A3379BF7E00E7
:207180007F041200B2A190087B54E4F0A37406F0E47F0421726290087ADEE025E0FF9008F7
:2071A0007ADDE033FE74CD2FF58274333EF583759308E0FFA3E090087B56CFF0A3EFF09077
:2071C000087ADEE004F0700790087ADDE004F012072E0378587C7B7D097B097A36794D7E32
:2071E000007F041200B2A190087B52E4F0A37403F0E4A3F0A3F07F01806890087ADEE025FD
:20720000E0FF90087ADDE033FE74CD2FF58274333EF583759308E0FFA3E090087B56CFF0B1
:20722000A3EFF090087ADEE004F0700790087ADDE004F07B097A3279B012072E0978587CD9
:207240007B7D097B097A3379C37E007F041200B2A190087B52E4F0A37402F0E4A3F0A3F00E
:207260007F01FEFDFC90087B5C1200B757E490087AE7F0A3F090083665E0FEA3E0FF90087D
:207280007ADFEEF0A3EFF090087ADDE0FCA3E0FDEF25E0FFEE33FE74B32FF58274333EF531
:2072A00083759308ECF0A3EDF090087AE0E0FF12071166EF4E7003FEFF2290087AE0E0FFDE
:2072C00012073CDB90084544E0FBA3E0FAA3E02404F9E43AFA1200B688C390087AE4E094CC
:2072E000D090087AE3E064809487503590087AE0E0FF12073CCC90087B5CE0F8A3E0F9A30D
:20730000E0FAA3E05FFFEA5EFEE95DFDE85CFCE4FBFAF9F8C31200B634600321742F216AAE
:20732000DE90087AE3E0FEA3E0FF64BB7003EE640B6006BE0B38BFBC3590087AE0E0FF1231
:20734000073CD690087B5CE0F8A3E0F9A3E0FAA3E05FFFEA5EFEE95DFDE85CFCE4FBFAF958
:20736000F8C31200B634600321742F216ADE90087AE3E0FEA3E0FF64D37003EE6407600608
:20738000BE0735BFD43290087AE0E0FF12073CD190087B5CE0F8A3E0F9A3E0FAA3E05FFF16
:2073A000EA5EFEE95DFDE85CFCE4FBFAF9F8C31200B634707A216ADEC390087AE4E094B843
:2073C00090087AE3E06480948B503290087AE0E0FF12073CD190087B5CE0F8A3E0F9A3E016
:2073E000FAA3E05FFFEA5EFEE95DFDE85CFCE4FBFAF9F8C31200B6347035216ADE90087A40
:20740000E0E0FF12073CD690087B5CE0F8A3E0F9A3E0FAA3E05FFFEA5EFEE95DFDE85CFC98
:20742000E4FBFAF9F8C31200B6347003216ADE12073B69EF64014E90087AE0700EE0FF1227
:20744000073D2FAC06AD07E4FF800CE0FF12073D2FAC06AD077F0112071C5D90087B4DE0C8
:20746000F9A3E0FAA3E09008369CC9F0A3EAF0A3E9F0A37409F0A3747BF0A37450F0A374F7
:2074800009F0A3747AF0A374E9F090087B52E0FFA3E0900836A5CFF0A3EFF090087B54E0C0
:2074A000FFA3E0900836A7CFF0A3EFF090087ADFE0FFA3E0900836A9CFF0A3EFF07B097A8B
:2074C0007B79581206108290087AE7EEF0A3EFF0BEFF2FBFFF2C90087AE1E0FCA3E0FD90A8
:2074E000083666E025E0FF90083665E033FE74B32FF58274333EF583759308ECF0A3EDF02A
:20750000802590087CB3E0FCA3E0FDA3E0FEA3E02401FFE43EFEE43DFDE43CFC90087CB35A
:207520001200B757216ADE90087AE7E0FEA3E0FF229000FFFD1200B891EBF0A3EAF0A3E97C
:20754000F09000FED61200B8919000012A1200B8B8E0FBA3E0FAA3E0F9C003C002C00185A0
:207560005083855182759308A982AA839008A5AB7409F0A3EAF0A3E9F09000012A1200B8A5
:20758000B8E0FBA3E0FAA3E02434F9E43AFA1200B45025E0FEE5F0339008A5AEF0A3CEF092
:2075A000D001D002D0031206FBB79000012A1200B8B8E0FBA3E0FAA3E02434F9E43AFA12F8
:2075C00000B45025E0FFE5F033FE9000012A1200B8B8E0FBA3E0FAA3E02FF9EA3EFA120029
:2075E000B450FFAEF0900000821200B8B8EEF0A3EFF0900000801200B8B8E4F0A304F09069
:207600000000821200B8B8E0FEA3E0FF900000801200B8B8E0FCA3E0FDD39FEE6480F8ECF0
:20762000648098400321776E9000012A1200B8B8E0FBA3E0FAA3E02434F9E43AFA1200B43E
:2076400050C39401FFE5F09400FEEF25E0FFEE33FE759308E5512FF582E5503EF58375932B
:2076600008ECF0A3EDF0900000821200B8B8E0FEA3E0B5052FECB5062B1200B450C3940188
:20768000FFE5F09400FEEF25E0FFEE33FE759308E5512FF582E5503EF5837593087402F025
:2076A000A3745CF09000012D1200B8B8E0FBA3E0FAA3E0F9C003C002C0019000013012003A
:2076C000B8B8E0FBA3E0FAA3E0F91200B450FDACF0855083855182759308A982AA83900807
:2076E0009F197409F0A3EAF0A3E9F09000012A1200B8B8E0FBA3E0FAA3E02434F9E43AFAEB
:207700001200B450FF90089F1CE5F0F0A3EFF0D001D002D0031206054B900000841200B8FE
:20772000B8EEF0A3EFF0900001331200B8B8E0FEA3E0FF4E600F900000841200B8B8E0FC5C
:20774000A3E04C6029EF4E7012900000841200B8B8E0FEC3EE648094804013900000801280
:2077600000B8B8E475F0011200B4242175FF900000821200B8B8E0FEA3E0FF9000008012BA
:2077800000B8B8E0FCA3E0D39FEE6480F8EC6480984003217F167B09855083855182759341
:2077A00008A982AA83C003C002C0019000012D1200B8B8E0F9A3E0FAA3E09008A5ABC9F069
:2077C000A3EAF0A3E9F09000012A1200B8B8E0FBA3E0FAA3E02434F9E43AFA1200B45025F4
:2077E000E0FEE5F0339008A5AEF0A3CEF0D001D002D0031206FBB79000012A1200B8B8E00A
:20780000FBA3E0FAA3E02434F9E43AFA1200B450FFAEF0900001301200B8B8E0FBA3E0FAB6
:20782000A3E0F9EE8FF01200B4CA900001381200B8B8E0FBA3E0FAA3E0F9E4F5F01200B421
:20784000CA9000012A1200B8B8E0FBA3E0FAA3E02437F9E43AFA1200B450FFAEF0E5F060F2
:207860000321798CEF24F9607714600E24F2400321792A2411600321798C9000008212007B
:20788000B8B8E0FEA3E0FF900000801200B8B8E0FCA3E0B50727ECB5062390000080120058
:2078A000B8B8A3E0C39401FF7B09900000861200B8B8A982AA831207246B21798C900000AC
:2078C000801200B8B8A3E0C39401FF7B09900000861200B8B8A982AA8312073D1321798CC9
:2078E000900000821200B8B8E0FEA3E0FF900000801200B8B8E0FCA3E0C39FEE6480F8EC8B
:20790000648098400321798C900000801200B8B8A3E0C39401FF7B09900001281200B8B857
:20792000A982AA831204A07D8062900000821200B8B8E0FEA3E0FF900000801200B8B8E074
:20794000FCA3E0B50726ECB50622900000801200B8B8A3E0C39401FF7B09900000881200E3
:20796000B8B8A982AA831207249A8020900000801200B8B8A3E0C39401FF7B0990000088C0
:207980001200B8B8A982AA831206B3C79000012A1200B8B8E0FBA3E0FAA3E02437F9E43AF1
:2079A000FA1200B450FFAEF0E5F06003217F16EF24FCB412004003217F16900179C975F026
:2079C00004A4C58325F0C5837302017A1102017A7602017ADC02017B5802017BBB02017F7C
:2079E0001602017C0302017C3902017C6F02017CC202017CF802017DA202017DCA02017EA4
:207A00000002017E3602017E8902017EBE02017DA2900001351200B8B8E0FBA3E0FAA3E021
:207A2000F9E475F0041200B4CA900000821200B8B8E0FEA3E0FF900000801200B8B8E0FC0E
:207A4000A3E0B50716ECB50612E47F147E05FDFC9008570F1200B757217F0E900000801237
:207A600000B8B8A3E0C39401FF7B097A57790F1206AB6A217F0E900001351200B8B8E0FBE1
:207A8000A3E0FAA3E0F9E475F0041200B4CA900000861200B8B8E0C4F854F0C8A3E0C45435
:207AA0000F48540F601914600C14600924FE600304701680147F007EE17DF57C0580127F11
:207AC000007ECA7D9A7C3B80087F807E967D987C009008570F1200B757217F0E9000008286
:207AE0001200B8B8E0FEA3E0FF900000801200B8B8E0FCA3E0B50728ECB50624900001353E
:207B00001200B8B8E0FBA3E0FAA3E0F9E475F0061200B4CA7B097A56790F12072845802F1F
:207B2000900001351200B8B8E0FBA3E0FAA3E0F9E4F5F01200B4CA900000801200B8B8A39B
:207B4000E0C39401FF7B097A56790F120726677B097A56790F217F1C900001351200B8B88C
:207B6000E0FBA3E0FAA3E0F9E475F0041200B4CA900000821200B8B8E0FEA3E0FF900000D0
:207B8000801200B8B8E0FCA3E0B50709ECB50605E47F018018900001281200B8B8A3E05405
:207BA0000F64066005E47F018003E47F02FEFDFC9008570F1200B757217F0E900001351200
:207BC00000B8B8E0FBA3E0FAA3E0F9E475F0041200B4CA900000861200B8B8E0C4F854F00C
:207BE000C8A3E0C4540F48540F64076005E47F018003E47F02FEFDFC9008570F1200B75737
:207C0000217F0E900001351200B8B8E0FBA3E0FAA3E0F9E475F0041200B4CA900000C41257
:207C200000B8B8E0FCA3E0FDA3E0FEA3E0FF9008570F1200B757217F0E900001351200B819
:207C4000B8E0FBA3E0FAA3E0F9E475F0041200B4CA900001081200B8B8E0FCA3E0FDA3E0C1
:207C6000FEA3E0FF9008570F1200B757217F0E900001351200B8B8E0FBA3E0FAA3E0F9E4B8
:207C800075F0041200B4CA900001101200B8B8E0FCA3E0FDA3E0FEA3E0FF9000010C1200BA
:207CA000B8B8E0F8A3E0F9A3E0FAA3E02FFFEA3EFEE93DFDE83CFC9008570F1200B757212A
:207CC0007F0E900001351200B8B8E0FBA3E0FAA3E0F9E475F0041200B4CA90000104120077
:207CE000B8B8E0FCA3E0FDA3E0FEA3E0FF9008570F1200B757217F0E900001351200B8B8A1
:207D0000E0FBA3E0FAA3E0F9E475F0041200B4CA900000F81200B8B8E0FCA3E0FDA3E0FECB
:207D2000A3E0FF900000F41200B8B8E0F8A3E0F9A3E0FAA3E02FFFEA3EFEE93DFDE83CFCD0
:207D4000900001181200B8B8E0F8A3E0F9A3E0FAA3E02FFFEA3EFEE93DFDE83CFC9000007D
:207D6000EC1200B8B8E0F8A3E0F9A3E0FAA3E02FFFEA3EFEE93DFDE83CFC900000F0120018
:207D8000B8B8E0F8A3E0F9A3E0FAA3E02FFFEA3EFEE93DFDE83CFC9008570F1200B7572149
:207DA0007F0E900001351200B8B8E0FBA3E0FAA3E0F9E475F0041200B4CAE4FFFEFDFC90D3
:207DC00008570F1200B757217F0E900001351200B8B8E0FBA3E0FAA3E0F9E475F0041200EC
:207DE000B4CA900000881200B8B8E0FCA3E0FDA3E0FEA3E0FF9008570F1200B757217F0E40
:207E0000900001351200B8B8E0FBA3E0FAA3E0F9E475F0041200B4CA9000009C1200B8B8BB
:207E2000E0FCA3E0FDA3E0FEA3E0FF9008570F1200B757217F0E900001351200B8B8E0FBF4
:207E4000A3E0FAA3E0F9E475F0041200B4CA900000941200B8B8E0FCA3E0FDA3E0FEA3E046
:207E6000FF900000981200B8B8E0F8A3E0F9A3E0FAA3E02FFFEA3EFEE93DFDE83CFC9008D6
:207E8000570F1200B757217F0E900001351200B8B8E0FBA3E0FAA3E0F9E475F0041200B47F
:207EA000CA900000901200B8B8E0FCA3E0FDA3E0FEA3E0FF9008570F1200B7578050900079
:207EC00001351200B8B8E0FBA3E0FAA3E0F9E475F0041200B4CA900000B01200B8B8E0FC9B
:207EE000A3E0FDA3E0FEA3E0FF900000B41200B8B8E0F8A3E0F9A3E0FAA3E02FFFEA3EFE91
:207F0000E93DFDE83CFC9008570F1200B7577B097A57790F80067B007A0079009000013B63
:207F20000200B89178047C627D097B817A9079FD7E007F3D1200B2A178417C627D097B81E2
:207F40007A91793A7E007F2F1200B2A1900848ACE0FBA3E0FAA3E0F9E475F0011200B474EE
:207F6000AFF0FE60032188AFEF24FE700321804D1470032183671470032186552403600398
:207F80002188AF9008A0737489F0A374B3F0A374D7F0900841CFE0FBA3E0FAA3E0F91206C5
:207FA0005EEB90086310EBF0A3EAF0A3E9F090086310E0FBA3E0FAA3E04A4B70037F012209
:207FC000900889D87489F0A374B3F0A374DFF0A37409F0A37463F0A37413F090086310E09C
:207FE000FBA3E0FAA3E0F91200BD8B90088B077489F0A374B3F0A374E9F090086313E0FE86
:20800000A3E0FF90088B0AEEF0A3EFF02401FFE43EA3F0A3EFF0900841CFE0FBA3E0FAA353
:20802000E0F912008C3390084547EEF0A3EFF090086313E0F9A3E0FF900848BDE0FBA3E0AE
:20804000FAA3E0C98FF01200B4CA2188B290087EFFE02401FF90087EFEE03400FE90087E1B
:20806000CCE02FFF90087ECBE03EFE900848BDE0FBA3E0FAA3E0F91200B4502401FDE43567
:20808000F0FCC3ED9FEC9E401812073CA4EF4E7010FE7FA0FD7B097A6279701200BBFD8060
:2080A0001B900848BDE0FBA3E0FAA3E0F91200B450FF7B097A6279701206B3C790088B071A
:2080C0007409F0A37462F0A37404F0A37489F0A374B5F0A37460F090086270E0FCA3E0FD46
:2080E000A3E0FEA3E0FF90088B0D1200B757900841CFE0FBA3E0FAA3E0F912008C33900848
:208100004547EEF0A3EFF0900841CFE0FBA3E0FAA3E0F990084547E0FEA3E0FFE92FF9EA78
:208120003EFAC00390088B077489F0A374B5F0A37463F090086284E0FCA3E0FDA3E0FEA309
:20814000E0FF90088B0A1200B75790086278E0FCA3E0FDA3E0FEA3E0FF90088B0E1200B728
:2081600057D00312008C3390084548E02FF090084547E03EF090086313E4F0A304F090089D
:208180006313E0FEA3E0FFD39404EE6480948040032188B2EE60032182B0EF24FE604F14A2
:2081A0007003218229147003218264240360032182B0900863157489F0A374B5F0A374C77E
:2081C000F090086280E0FCA3E0FDA3E0FEA3E0FF9008631B1200B757900863187489F0A3FD
:2081E00074B5F0A374D5F0900862A421829D900863157489F0A374B5F0A374DFF090086213
:208200007CE0FCA3E0FDA3E0FEA3E0FF9008631B1200B757900863187489F0A374B5F0A3EE
:2082200074EDF0900862A08074900863157489F0A374B5F0A374F9F090086294E0FCA3E0B9
:20824000FDA3E0FEA3E0FF9008631B1200B757900863187489F0A374B6F0A3740AF0900882
:2082600062888039900863157489F0A374B6F0A37414F090086298E0FCA3E0FDA3E0FEA374
:20828000E0FF9008631B1200B757900863187489F0A374B6F0A37422F09008629CE0FCA3CE
:2082A000E0FDA3E0FEA3E0FF9008631F1200B757900841CFE0FBA3E0FAA3E0F99008454704
:2082C000E0FEA3E0FFE92FF9EA3EFAC003C002C00190088B077409F0A37462F0A37441F07D
:2082E00090086315E0F9A3E0FAA3E090088B0AC9F0A3EAF0A3E9F09008631BE0FCA3E0FD44
:20830000A3E0FEA3E0FF90088B0D1200B75790086318E0F9A3E0FAA3E090088B11C9F0A38E
:20832000EAF0A3E9F09008631FE0FCA3E0FDA3E0FEA3E0FF90088B141200B757D001D00274
:20834000D00312008C3390084548E02FF090084547E03EF090086314E004F07007900863CE
:2083600013E004F021817E90087EFFE02401FF90087EFEE03400FE90087ECCE02FFF90082F
:208380007ECBE03EFE900848BDE0FBA3E0FAA3E0F91200B4502401FDE435F0FCC3ED9FEC8F
:2083A0009E401812073CA4EF4E7010FE7FA0FD7B097A6279701200BBFD801B900848BDE0CC
:2083C000FBA3E0FAA3E0F91200B450FF7B097A6279701206B3C790088B077409F0A37462A9
:2083E000F0A37404F0A37489F0A374B6F0A37435F0900862ACE0FCA3E0FDA3E0FEA3E0FFF4
:2084000090088B0D1200B757900841CFE0FBA3E0FAA3E0F912008C3390084547EEF0A3EF2B
:20842000F090086313E4F0A304F090086313E0FEA3E0FFC39406EE6480948040032188B284
:20844000EE600321859EEF24FE60551470032184DC1470032185171470032185522404606E
:208460000321859E900863157489F0A374B6F0A37438F0900862F0E0FCA3E0FDA3E0FEA352
:20848000E0FF9008631B1200B757900863187489F0A374B6F0A37444F0900862EC21858BA8
:2084A000900863157489F0A374B5F0A374C7F0900862F4E0FCA3E0FDA3E0FEA3E0FF900850
:2084C000631B1200B757900863187489F0A374B5F0A374D5F0900862B821858B9008631573
:2084E0007489F0A374B5F0A374DFF0900862F8E0FCA3E0FDA3E0FEA3E0FF9008631B120074
:20850000B757900863187489F0A374B6F0A3744DF0900862B48074900863157489F0A37486
:20852000B6F0A3745BF0900862D8E0FCA3E0FDA3E0FEA3E0FF9008631B1200B757900863D1
:20854000187489F0A374B6F0A37463F0900862D48039900863157489F0A374B6F0A3747027
:20856000F0900862E0E0FCA3E0FDA3E0FEA3E0FF9008631B1200B757900863187489F0A3F9
:2085800074B6F0A3747AF090086300E0FCA3E0FDA3E0FEA3E0FF9008631F1200B757900814
:2085A00041CFE0FBA3E0FAA3E0F990084547E0FEA3E0FFE92FF9EA3EFAC003C002C001904A
:2085C000088B077409F0A37462F0A37441F090086315E0F9A3E0FAA3E090088B0AC9F0A371
:2085E000EAF0A3E9F09008631BE0FCA3E0FDA3E0FEA3E0FF90088B0D1200B757900863184D
:20860000E0F9A3E0FAA3E090088B11C9F0A3EAF0A3E9F09008631FE0FCA3E0FDA3E0FEA301
:20862000E0FF90088B141200B757D001D002D00312008C3390084548E02FF090084547E095
:208640003EF090086314E004F0700790086313E004F021842A90087EFFE02401FF90087EB2
:20866000FEE03400FE90087ECCE02FFF90087ECBE03EFE900848BDE0FBA3E0FAA3E0F9127A
:2086800000B4502401FDE435F0FCC3ED9FEC9E401812073CA4EF4E7010FE7FA0FD7B097AB0
:2086A0006279701200BBFD801B900848BDE0FBA3E0FAA3E0F91200B450FF7B097A6279703B
:2086C0001206B3C790086313E4F0A304F090086313E0FEA3E0FFD39403EE6480948040038E
:2086E000218871EE60032187BAEF24FE604514607D240260032187BA900863157489F0A37B
:2087000074B6F0A37484F0900862BCE0FCA3E0FDA3E0FEA3E0FF9008631B1200B7579008D1
:2087200063187489F0A374B6F0A37490F0900862C08074900863157489F0A374B6F0A374FE
:20874000A3F0900862C4E0FCA3E0FDA3E0FEA3E0FF9008631B1200B757900863187489F033
:20876000A374B6F0A374B7F0900862C88039900863157489F0A374B6F0A374CBF09008627D
:20878000CCE0FCA3E0FDA3E0FEA3E0FF9008631B1200B757900863187489F0A374B6F0A318
:2087A00074E0F0900862D0E0FCA3E0FDA3E0FEA3E0FF9008631F1200B757900841CFE0FB8F
:2087C000A3E0FAA3E0F990084547E0FEA3E0FFE92FF9EA3EFAC003C002C00190088B077405
:2087E00009F0A37462F0A37441F090086315E0F9A3E0FAA3E090088B0AC9F0A3EAF0A3E9F7
:20880000F09008631BE0FCA3E0FDA3E0FEA3E0FF90088B0D1200B75790086318E0F9A3E034
:20882000FAA3E090088B11C9F0A3EAF0A3E9F09008631FE0FCA3E0FDA3E0FEA3E0FF9008C4
:208840008B141200B757D001D002D00312008C3390084548E02FF090084547E03EF0900824
:208860006314E004F0700790086313E004F02186CD900841CFE0FBA3E0FAA3E0F990084587
:2088800047E0FEA3E0FFE92FF9EA3EFA90088B077489F0A374B6F0A374F6F012008C3390CC
:2088A000084548E02FF090084547E03EF080037F01227F002290088D7DEDF090088D7AEB23
:2088C000F0A3EAF0A3E9F02404F9E43AFA1200B31FFFE4FCFDFE90088D861200B757900855
:2088E0008D86E0FCA3E0FDA3E0FEA3E0FF78081200B65890088D861200B75790088D86E010
:20890000F8A3E0F9A3E0FAA3E0FBC001C002C00390088D7AE0FBA3E0FAA3E02405F9E43AE8
:20892000FA1200B31FFFD003D002D001EB4FFFEAFEE9FDE8FC90088D861200B75790088D09
:2089400086E0FCA3E0FDA3E0FEA3E0FF78101200B65890088D861200B75790088D86E0FC38
:20896000A3E0FDA3E0FEA3E04402FFEC90088D861200B75790088D7AE0FBA3E0FAA3E0F904
:208980001200B31FFFE4FCFDFE90088D8A1200B75790088D8AE0FCA3E0FDA3E0FEA3E0FF3C
:2089A00078081200B65890088D8A1200B75790088D8AE0F8A3E0F9A3E0FAA3E0FBC001C0C9
:2089C00002C00390088D7AE0FBA3E0FAA3E02401F9E43AFA1200B31FFFD003D002D001EBDE
:2089E0004FFFEAFEE9FDE8FC90088D8A1200B75790088D8AE0FCA3E0FDA3E0FEA3E0FF7822
:208A0000081200B65890088D8A1200B75790088D8AE0F8A3E0F9A3E0FAA3E0FBC001C002DE
:208A2000C00390088D7AE0FBA3E0FAA3E02402F9E43AFA1200B31FFFD003D002D001EB4F2F
:208A4000FFEAFEE9FDE8FC90088D8A1200B75790088D8AE0FCA3E0FDA3E0FEA3E0FF780808
:208A60001200B65890088D8A1200B75790088D8AE0F8A3E0F9A3E0FAA3E0FBC001C002C0C6
:208A80000390088D7AE0FBA3E0FAA3E02403F9E43AFA1200B31FFFD003D002D001EB4FFF8F
:208AA000EAFEE9FDE8FC90088D8A1200B75790088D7DE0B40111E4FFFEFD7C8090088D925C
:208AC0001200B757218E57E47F01FEFDFC90088D921200B75790088D92E0FCA3E0FDA3E0A8
:208AE000FEA3E0FF78041200B65890088D921200B75790088D92E0FCA3E0FDA3E0FEA3E06C
:208B0000FFEC90088D921200B75790088D92E0FCA3E0FDA3E0FEA3E0FF78031200B6589052
:208B2000088D921200B75790088D92E0F8A3E0F9A3E0FAA3E0FBC001C002C00390088D7A03
:208B4000E0FBA3E0FAA3E0240CF9E43AFA1200B31FFFD003D002D001EB4FFFEAFEE9FDE8B1
:208B6000FC90088D921200B75790088D92E0FCA3E0FDA3E0FEA3E0FF78021200B6589008DA
:208B80008D921200B75790088D92E0F8A3E0F9A3E0FAA3E0FBC001C002C00390088D7AE0CB
:208BA000FBA3E0FAA3E0240BF9E43AFA1200B31FFFD003D002D001EB4FFFEAFEE9FDE8FC36
:208BC00090088D921200B75790088D92E0FCA3E0FDA3E0FEA3E0FF78011200B65890088DEA
:208BE000921200B75790088D92E0FCA3E0FDA3E0FEA3E0FF90088D7AE0FBA3E0FAA3E0240F
:208C000013F9E43AFA1200B31FB40105E47B018002E4FBFAF9F8EF4BFFEE4AFEED49FDEC58
:208C200048FC90088D921200B75790088D92E0FCA3E0FDA3E0FEA3E0FF78011200B65890DA
:208C4000088D921200B75790088D92E0FCA3E0FDA3E0FEA3E0FFEC90088D921200B7579064
:208C6000088D92E0FCA3E0FDA3E0FEA3E0FF78011200B65890088D921200B75790088D9247
:208C8000E0FCA3E0FDA3E0FEA3E0FF90088D7AE0FBA3E0FAA3E02412F9E43AFA1200B31FD0
:208CA000B40105E47B018002E4FBFAF9F8EF4BFFEE4AFEED49FDEC48FC90088D921200B7FC
:208CC0005790088D92E0FCA3E0FDA3E0FEA3E0FF78011200B65890088D921200B75790081F
:208CE0008D92E0FCA3E0FDA3E0FEA3E0FF90088D80E0B40105E47B018002E4FBFAF9F8EF1C
:208D00004BFFEE4AFEED49FDEC48FC90088D921200B75790088D92E0FCA3E0FDA3E0FEA362
:208D2000E0FF78031200B65890088D921200B75790088D92E0F8A3E0F9A3E0FAA3E0FBC01C
:208D400001C002C00390088D7AE0FBA3E0FAA3E0240AF9E43AFA1200B31F5403FFD003D0F7
:208D600002D001EB4FFFEAFEE9FDE8FC90088D921200B75790088D92E0FCA3E0FDA3E0FECA
:208D8000A3E0FF78031200B65890088D921200B75790088D92E0F8A3E0F9A3E0FAA3E0FBD9
:208DA000C001C002C00390088D7AE0FBA3E0FAA3E02409F9E43AFA1200B31F5403FFD003A8
:208DC000D002D001EB4FFFEAFEE9FDE8FC90088D921200B75790088D92E0FCA3E0FDA3E098
:208DE000FEA3E0FF780C1200B65890088D921200B75790088D92E0F8A3E0F9A3E0FAA3E06D
:208E0000FBC000C001C002C00390088D7EE0FEA3E07802CEC313CE13D8F9547FFFD003D008
:208E200002D001D000EB4FFFEAFEE9FDE8FC90088D921200B7577B817ACA79BB90088D92A2
:208E4000E0FCA3E0FDA3E0FEA3E0FF90088B071200B75712008C39E490088D81F090088DF3
:208E600081E0FFC3940140032192261207327EEF700321921C90088D7DE064016003218F2A
:208E80003090088D81E0541FFFE4FCFDFE90088D8E1200B75790088D8EE0FCA3E0FDA3E06A
:208EA000FEA3E0FF78041200B65890088D8E1200B75790088D8EE0FCA3E0FDA3E0FEA3E0B0
:208EC0004401FFEC90088D8E1200B75790088D8EE0FCA3E0FDA3E0FEA3E0FF780C1200B631
:208EE0005890088D8E1200B75790088D8EE0F8A3E0F9A3E0FAA3E0FBC001C002C003900867
:208F00008D7AE0FBA3E0FAA3E02407F9E43AFA1200B450FFD003D002D001EB4FFFEA45F050
:208F2000FEE9FDE8FC90088D8E1200B75721916490088D7AE0FBA3E0FAA3E02406F9E43AC5
:208F4000FA1200B31FFF7E0030E7027E01EE601BEF547F90088D83F090088D857401F090BC
:208F6000088D81E090088D84F080161200B31FFE541F90088D83F0EEC4135403A3F0E4A3A9
:208F8000F090088D7AE0FBA3E0FAA3E0F91200B31F20E01AE92412F9E43AFA1200B31F64F8
:208FA00001600B90088D7E7401F0A374FFF07B817ACA79C890088D7EE0FFA3E090088B0787
:208FC000CFF0A3EFF012008C397E0090088D7FE05403FFE4FCFD90088D8E1200B7579008D9
:208FE0008D8EE0FCA3E0FDA3E0FEA3E0FF78061200B65890088D8E1200B75790088D8EE0F3
:20900000F8A3E0F9A3E0FAA3E0FB90088D83E0541FFFEB4FFFEAFEE9FDE8FC90088D8E1237
:2090200000B75790088D8EE0FCA3E0FDA3E0FEA3E0FF78081200B65890088D8E1200B7579D
:2090400090088D8EE0F8A3E0F9A3E0FAA3E0FB90088D84E0541FFFEB4FFFEAFEE9FDE8FC28
:2090600090088D8E1200B75790088D8EE0FCA3E0FDA3E0FEA3E0FF78021200B65890088D4C
:209080008E1200B75790088D8EE0F8A3E0F9A3E0FAA3E0FB90088D85E0FFEB4FFFEAFEE98D
:2090A000FDE8FC90088D8E1200B75790088D8EE0FCA3E0FDA3E0FEA3E0FF78011200B65851
:2090C00090088D8E1200B75790088D8EE0FCA3E0FDA3E0FEA3E04401FFEC90088D8E1200B5
:2090E000B75790088D8EE0FCA3E0FDA3E0FEA3E0FF780D1200B65890088D8E1200B7579048
:20910000088D8EE0F8A3E0F9A3E0FAA3E0FBC001C002C00390088D7AE0FBA3E0FAA3E024F9
:2091200007F9E43AFA1200B450FFD003D002D001EB4FFFEA45F0FEE9FDE8FC90088D8E12A7
